:020000040800F2
:1000000000000220F9B70B087DB80B08118C060818
:100010007DB80B087DB80B087DB80B080000000008
:100020000000000000000000000000007DB80B0888
:100030007DB80B08000000007DB80B088D2705086F
:100040007DB80B087DB80B087DB80B087DB80B0890
:100050007DB80B087DB80B08D9EB0408DDEB04086C
:10006000E1EB0408E5EB0408E9EB0408CD400408E3
:10007000E1400408F5400408094104081D41040852
:1000800031410408454104087DB80B087DB80B08D0
:100090007DB80B087DB80B087DB80B08EDEB0408A4
:1000A0007DB80B087DB80B087DB80B08F54A04082D
:1000B000094B04081D4B0408314B04087133040834
:1000C00065330408A5330408993304087DB80B0888
:1000D0007DB80B08515504085D550408695504089E
:1000E000F1EB04087DB80B08000000006D4B04081C
:1000F000BD4B0408E54B0408594B0408594104085A
:100100007DB80B0829680408454B04087DB80B0826
:10011000755504087DB80B087DB80B08D97904081B
:100120006D4104088141040895410408A94104086F
:10013000BD4104087DB80B087DB80B087DB80B08DD
:1001400000000000000000000000000000000000AF
:10015000D1410408E5410408F94104088155040827
:10016000D9330408CD3304087DB80B087DB80B08DB
:100170007DB80B087DB80B087DB80B0800000000A7
:100180007DB80B087DB80B088D55040899550408F7
:100190007DB80B087DB80B087DB80B087DB80B083F
:1001A0007DB80B087DB80B087DB80B087DB80B082F
:1001B0007DB80B087DB80B087DB80B087DB80B081F
:1001C0007DB80B087DB80B087DB80B087DB80B080F
:1001D0007DB80B085D6804087DB80B087DB80B0876
:1001E0007DB80B087DB80B087DB80B087DB80B08EF
:1001F0007DB80B087DB80B087DB80B087DB80B08DF
:100200007DB80B087DB80B087DB80B087DB80B08CE
:10021000814B0408954B0408A94B04087DB80B08D2
:100220007DB80B087DB80B087DB80B0800000000F6
:100230002D6804087DB80B08000000007DB80B088D
:100240007DB80B087DB80B087DB80B087DB80B088E
:100250007DB80B087DB80B087DB80B087DB80B087E
:100260007DB80B087DB80B087DB80B087DB80B086E
:100270007DB80B087DB80B087DB80B0800000000A6
:100280007DB80B08000000007DB80B0800000000DE
:08029000000000007DB80B081E
:080298009CA70B00010000000F
:1002A000F4A501240207000005003F0014A6012464
:1002B0000207000206033D0034A6012401100000DD
:1002C0000001760054A601240114000000001E0065
:1002D00074A60124011A000000000D0094A6012458
:1002E0000115000000000C00B4A601240116000056
:1002F00000000C00D4A60124011B000000000E0029
:10030000F4A60124011C000000001E0014A7012413
:100310000117000000000C0034A7012401180000A0
:1003200000000E0054A701240119000000000C0079
:1003300074A70124011E000000000C0094A70124F2
:10034000011F000000000C00B4A7012401280100D7
:1003500000011800D4A7012401200000000148007A
:10036000F4A70124012100000001490014A8012480
:100370000122000000014A0034A8012401230000EA
:1003800000014B0054A801240124000000014C008E
:1003900074A801240125000000014D0094A8012447
:1003A0000126000000014E00B4A80124012700002E
:1003B00000014F00D4A80124012B000000002900F7
:1003C000F4A80124012C01000000290014A9012433
:1003D000012D01000000700034A90124012F00004C
:1003E0000000310054A90124012E01000000520038
:1003F00074A90124013001000001280094A90124FE
:100400000131010000012800B4A9012402290500DE
:1004100000012C00D4A901240134000000003C009C
:0C042000F4A901240137000000002000B6
:020000040804EE
:10000000836B5A6D12F0500F5A6D1AD1196842F471
:1000100000725A650A6812F0080FCA6816D012F406
:10002000406F15D1CA68920412D45A6D22F48072BE
:100030005A655A6DD1040BD45A6D42F001025A65CB
:100040007047D20604D4DB6CDB6C18479007ECD009
:10005000704700BF704700BF836B5A6D42F040028B
:100060005A659A6D42F004029A65704702685549D4
:1000700038B5554B554D564CAA4218BF9A420CBF45
:10008000012300238A4208BF43F001033031A2421A
:1000900008BF43F0010330348A4208BF43F0010334
:1000A0003031A24208BF43F0010330348A4208BF16
:1000B00043F0010301F55C71A24208BF43F0010364
:1000C00004F55C748A4208BF43F001033031A24258
:1000D00008BF43F0010330348A4208BF43F00103F4
:1000E0003031A24208BF43F0010330348A4208BFD6
:1000F00043F001033031A24208BF43F001038A42BA
:1001000008BF43F0010313B9324B9A4208D10423CC
:1001100080F83530136823F001031360002038BDE8
:100120002D4B2E4D1168AA4218BF9A422C4C21F03B
:100130000E0105F13C050CBF012300231160A24212
:1001400008BF43F0010311682834AA4208BF43F0F6
:10015000010321F00101A24208BF43F0010314345E
:100160001160A24208BF43F001031E498A4208BF42
:1001700043F0010313B91C4B9A4217D10123856D3B
:10018000D0E91714226801F01F0122F480728B401D
:1001900022606B60C36ED0E91921516033B11A68D7
:1001A000D0E91C1422F480721A604C6000210122F4
:1001B000036D80F8341080F83520002BAED09847BE
:1001C000ACE700BF4000024010000240280002409F
:1001D00058000240B80402401C5402580854025807
:1001E000305402588054025894540258002280F827
:1001F000422090F84130292B04D090F841302A2B2E
:1002000018D070474FF0280C2123016880F841C0B6
:10021000036390F8413003EA0C0363450B6814BF95
:100220006FF0F20C6FF0420C03EA0C030B6080F8E5
:10023000402070474FF0280C2223016880F841C00D
:10024000036390F8413003EA0C0363450B6814BF65
:100250006FF0F40C6FF0440C03EA0C030B6080F8B1
:10026000402070470023202210B4174C4363C4621F
:10027000036380F8412080F842304B07026811D5B3
:10028000526A436A1A70436A028D013343624AB16B
:10029000438D013A013B02859BB24385436C43F099
:1002A000040343640368102490F84120002190F86F
:1002B00041201A6822F0FE021A60DC615DF8044BEE
:1002C00080F84010704700BF0000FFFF70B50023AA
:1002D00090F84120424D044680F84230283AC562E9
:1002E0004385022A406C236840EA0100606439D8E3
:1002F00094F84110282094F8412001F0280102F0E0
:100300002802282914BFF6214621282A1A680CBF82
:10031000C9436FF0F6010A4032491A60002284F89E
:10032000410022631A68616312F4804231D01A6876
:10033000A06B22F480421A6098B100222A4B036518
:1003400084F8402090F83520022A3CD08022426573
:10035000BDE87040184794F84130602B3AD084F8DB
:10036000401070BD94F8412094F841201A6822F0A2
:10037000FE021A6094F84120602A02D0202284F8FC
:1003800041200022114622631A68616312F4804200
:10039000CDD1196811F40041DDD01968E06B21F46A
:1003A000004119600028DCD00F4B036584F8402021
:1003B00090F83520022AC9D1FFF758FE0028D0D086
:1003C000E06B036DC4E7FFF751FE0028C9D0A06BB6
:1003D000036DBDE7202384F8401084F8413070BDE0
:1003E0000000FFFF65040408F106040803689A6929
:1003F000196810B4D40528D50C0606D4416C11F048
:100400000B0F1FD15DF8044B7047416C4FF48074A3
:1004100041F0010141645105DC6120D5416C4FF48C
:100420008064920541F008014164DC61E6D5426CCC
:100430004FF4007142F002024264D961416C11F044
:100440000B0FDFD05DF8044B40E7540502D50906D9
:10045000E4D4D3E79405D1D50906E8D4CEE79205D4
:10046000E5D4CBE72DE9F84390F84030C76A012B7B
:1004700000F0D780012304460D46164680F8403030
:10048000880601D591065FD4EA0621D5F3061FD56B
:10049000638D9BB2002B40F0AA8094F84130B7F1F5
:1004A000007FDBB202D1282B00F0198194F8413093
:1004B00017F5803F2268DBB202D0292B00F0D380F1
:1004C0001023D3610023184684F84030BDE8F88338
:1004D0006A071BD4280702D5310700F19880AA07C4
:1004E000F0D5B307EED5638D9BB2002B00F0A4804E
:1004F000616A236811F8010B228D9862638D013ABD
:100500006162013B22859BB26385DBE77307E1D51E
:10051000638D9BB26BB12268636A526A1A70638DF5
:10052000616A228D013B0131013A9BB261622285F1
:100530006385638D17F5803F9BB2C3D0002BC1D17B
:100540002046FFF753FEBDE723682022664819685E
:10055000DA6194F8412094F841201A6822F0FE02F2
:100560001A605A6842F400425A605A6802405A605F
:100570009A69920701D500229A629A69D00703D43A
:100580009A6942F001029A614A044DD5A26B1AB1F0
:1005900011684A6892B2628569074BD55A6A25F09C
:1005A0000409636A1A70636A01336362238D002B46
:1005B00052D1638D9BB21BB1636C43F0040363643F
:1005C0000023236384F84230D4F844806363B8F195
:1005D000000F58D1E36ADFF814914B4531D194F8FC
:1005E0004130202384F8408084F841304CE7236870
:1005F0001022DA61636C43F00403636437F08073A4
:100600007FF460AF616C2046FFF760FE5AE794F814
:100610004130226803F02803282B42D00823D361FD
:1006200050E70220BDE8F8830804B5D5E26B002A44
:10063000AED1B1E7A946BCE737F080737FF442AF93
:100640007EE72046FFF7D2FD2023C4F82C9084F8E3
:10065000408084F8413017E7013B2385638D013BDF
:100660009BB26385A5E71023D3619369980701D5F1
:10067000002393629369D9073FF562AF936943F012
:10068000010393615CE7616C2046FFF71FFE94F85D
:100690004130282B7FF4F8AE49462046FFF7E2FDB3
:1006A000F2E6E1689369022990699368D56811D1EF
:1006B000C3F3C21383EA104313F006030AD1A16CFB
:1006C0000131A164A16C02297FF4FCAE0821A3646E
:1006D000D161F7E6136823F0B8031360F2E6294608
:1006E0002046FFF7BFFDEDE600E800FE0000FFFF3B
:1006F000836B0022D3E90E0102650A6593F841205D
:10070000602A02D1202283F841207047026870B429
:10071000D4072DD597490B69896A03F03803102B4C
:1007200000F0F180182B00F0E9804368B3F5803FBA
:1007300000F05581002B00F05B81B3F5A02F8D4BAD
:10074000196800F02C8221F480311960196821F4B5
:1007500080211960884B41F2883C864C1D6804E07A
:100760001968491B614500F2408121688E03F7D565
:1007700091072DD57F490B69896A13F0380300F082
:10078000A680182B00F0A080C3687A4C002B00F0E4
:100790006381216821F019011943774B21601D689D
:1007A00004E01968491B022900F21F8121684907EA
:1007B000F7D5724B01691D6841F20303B3EB154F86
:1007C000636880F0958023F0FE4343EA0163636031
:1007D000D5064CD4150713D54369664C002B00F0A1
:1007E0009E80616F644B41F0010161671D6804E008
:1007F0001968491B022900F2F880616F8907F7D553
:10080000940613D583695B4C002B00F007812168A7
:10081000594B41F4805121601D6804E01968491B5F
:10082000022900F2E28021688904F7D5540700F11B
:10083000A780426AC2B14F490B6903F03803182BF5
:1008400000F07F81022A0A684B4B22F080720A6016
:1008500000F01881186804E01A68121A022A00F2DF
:10086000C4800A689201F7D4002070BC70474149E7
:100870000B69896A03F03803082B63D0182B5DD00D
:10088000C3693C4C002B00F0D88021683A4B41F002
:10089000800121601D6804E01968491B022900F2EB
:1008A000A4802168C905F7D5344B056A196841F25F
:1008B0000303B3EB114FC0F09081636823F0F8435A
:1008C00043EA8563636085E78D077FF45DAF294B5D
:1008D0001B685C0701D5C368F3B1284C41F20303E0
:1008E00001692468B3EB144F224C6368FFF46BAFCB
:1008F00023F47C3343EA0133636069E701F00301C9
:1009000002297FF412AF1B4B1B689B037FF530AFAE
:100910004368002B7FF42CAF012070BC7047616FDF
:10092000154B21F0010161671D6803E01968491B3F
:1009300002295AD8616F8E07F8D461E701F00301EC
:1009400001299DD10B4B1B68DC0502D5C369802BA7
:10095000E2D10A4941F20303046A0968B3EB114F7B
:100960000449C0F088804B6823F0F84343EA84636D
:100970004B602FE700440258002F00240010005C59
:100980009C499D4B0A6842F480720A601C6803E02F
:100990001A68121B642A28D80A68D505F8D5826817
:1009A000012A00F02181002A00F00181052A934AE2
:1009B000116F00F0278121F001011167116F21F003
:1009C000040111671D6841F288348C4903E01A68FC
:1009D000521BA24209D80A6F9207F8D529E7874926
:1009E0000B6843F480330B60B4E6032070BC70479F
:1009F000824C41F28835804B216821F4803121609E
:100A0000216821F4802121601E6803E01968891B98
:100A1000A942EAD821688903F8D4A9E62168764B6F
:100A200021F4805121601D6803E01968491B0229E7
:100A3000DBD821688E04F8D4F8E621686E4B21F0EB
:100A4000800121601D6803E01968491B0229CCD888
:100A50002168CE05F8D4BDE62168674B21F001017D
:100A600021601D6803E01968491B0229BDD821686F
:100A70004E07F8D4ACE6CB6823F07C5343EA04631A
:100A8000CB60A7E61C6803E01A68121B022AACD8E8
:100A90000A689501F8D48C6A594A2240846A224334
:100AA000C46A42EA04128A62D0E90D24013A013C88
:100AB0005202240492B204F4FE042243046B013C6B
:100AC000C4F308042243C46B013C240604F0FE4432
:100AD00022430A63CA6A22F00102CA624A6B846C2A
:100AE0006FF3CF0242EAC4024A63CA6A046C22F07E
:100AF0000C022243414CCA62CA6A406C22F00202D4
:100B00000243CA62CA6A42F48032CA62CA6A42F4C2
:100B10000032CA62CA6A42F48022CA62CA6A42F0D9
:100B20000102CA620A6842F080720A60196804E031
:100B30001A68521A022A3FF658AF22689001F7D578
:100B400092E6012A8C6A0B6B3FF4E6AE04F00302D6
:100B5000816A8A427FF4E0AEC4F30514C26A94420B
:100B60007FF4DAAE026BC3F30801013A91427FF4DD
:100B7000D3AE426BC3F34621013A91427FF4CCAE2F
:100B8000826BC3F30641013A91427FF4C5AEC26B5A
:100B9000C3F30663013A981A18BF0120BDE641F479
:100BA00080211960196841F480311960D2E5134938
:100BB00041F288350A6F22F001020A670A6F22F0BB
:100BC00004020A671C6804E01A68121BAA423FF676
:100BD0000CAF0A6F9607F7D42BE6E36823F07C533B
:100BE00043EA0563E360F5E504490A6F42F0010258
:100BF0000A67E7E600480258002F00240044025824
:100C00000CFCFFFF41F004011167116F41F001017D
:100C10001167D7E6334B30B4996A9C6ADD6A14F4E5
:100C20007C7F5A6BC4F3051036D0C2F3CC0205F0BA
:100C3000010501F0030107EE900A05FB02F201290C
:100C4000B8EEE77A06EE902AFAEEE96A02D00229B7
:100C500042D019B3DFED247A87EE876A1B6BC3F3AA
:100C6000080307EE903AF7EE005AF8EEE77A77EECF
:100C7000A67A77EEA57A67EE867A1A4B1B6BC3F3DA
:100C80004623013307EE103AF8EEC76A87EEA67ADC
:100C9000FCEEC77A17EE900A30BC70471A689206CD
:100CA0001DD51968F7EE005A104A1B6BC1F3C1013C
:100CB000C3F30803CA4007EE903A06EE102AF8EE96
:100CC000E77AB8EEC66A77EEA66AC6EE077A36EE1F
:100CD000A57A67EE877AD0E7DFED057ABCE7DFED2E
:100CE000057AB9E7004402580024744A0090D00302
:100CF0000024F44A0024744CF0B5344AB0F1804F1B
:100D0000334CA0EB02020368A0EB040E4F69B2FA69
:100D100082F28E68BEFA8EFE0D684FEA52124FEADA
:100D20005E1E20D0FAB9DFF8B4C0604532D00CF5B1
:100D3000806C60452ED00CF5806C604513D0BEF100
:100D4000000F10D1234C244A904218BFA04225D056
:100D500002F58062904221D023F080033B43036080
:100D6000C662856213E04C6823F070032343CC68AD
:100D700023F44073234323F080033B430360C662A4
:100D8000856212B9BEF1000F12D00B690363012313
:100D90004361F0BD23F070034A681343CA6823F42B
:100DA0004073134323F080033B430360C6628562B4
:100DB000084A094B984218BF9042E6D003F5806379
:100DC0009842E2D001234361F0BD00BF0000014022
:100DD0000004014000400140004401400004004084
:100DE000836ADA0710B406D50168C46A4A6822F437
:100DF000003222434A609C0706D50168046B4A68AA
:100E000022F4803222434A60590706D50168446BB8
:100E10004A6822F4802222434A601A0706D50168F4
:100E2000846B4A6822F4004222434A60DC0606D5FD
:100E30000168C46B8A6822F4805222438A60990652
:100E400006D50168046C8A6822F4005222438A6045
:100E50005A060AD50168446C4A68B4F5801F22F42A
:100E6000801242EA04024A600BD01B0606D50268D3
:100E7000C16C536823F400230B4353605DF8044BAB
:100E800070474A68846C22F4C00222434A60ECE74F
:100E90000022836BA3F85E20A3F85620704700BFA2
:100EA000124B41F2883C124A01461B68A2FB032305
:100EB0005B0A0CFB03F33BB14A6B12F0450F01D008
:100EC000920404D5013BF7D14FF0004070474B6BC3
:100ED0005B0707D4486B10F0010014BF0123054BDA
:100EE0008B637047042318468B637047000000240F
:100EF000D34D6210C5002000036942681F2B70B4F7
:100F000030D9A3F1200520215468A940214227D0DF
:100F10008169087C022835D048681F2BC9681B4DA1
:100F20004E680169C1F30324194951F8244015F8AA
:100F300004C0056856F80C4024F0010446F80C4043
:100F4000407901EB4001088CE96800F4F05021EA97
:100F50000001E96010D9A3F1200120238B40D36068
:100F600070BC70472021146899402142F8D08169F3
:100F7000087C0228D0D105E0202101FA03F370BCDF
:100F80009360704700200874C6E700BFF8460C085D
:100F900018450C08436BDA692DE9F04197060446C1
:100FA00013D5586AE36AC0B2002B79D0216B9847F9
:100FB000636B1A6822F480721A609A6822F0010248
:100FC0009A609A6942F008029A61DA69D60701D5F7
:100FD00001221A62DA69950701D502221A62DA69DA
:100FE000500701D504221A62DA69110701D50822D7
:100FF0001A62DA69120612D5D4F8B420212A0ED06A
:10100000D4E909128A4257D0A169895C0132C9B278
:1010100099622169B2FBF1F001FB1022A262DA6948
:10102000570601D4BDE8F081DA6940F60F0C1D685F
:1010300004F1340012EA0C0F996823D0724E0E406E
:1010400042D1724F3D4240F0CD80D60202D54F02D0
:1010500000F1D080160606D501F4000105F08006E7
:101060000E4340F0BA805106DCD56A06DAD51A681C
:101070002020002122F040021A60C4F8B400C4F815
:10108000A410CFE79606E0D505F0200601F08057C2
:101090003E43DAD0D4F8A030002B40F08E80C1E778
:1010A000E3696269D054E369E2680133B3FBF2F1AA
:1010B00002FB1133E3617BE70022A4F88A201A685F
:1010C00022F080021A60AAE7D70709D5EF0507D5F5
:1010D00001271F62D4F8BC7047F00107C4F8BC7048
:1010E00097076DD4570709D5CF0707D504271F6287
:1010F000D4F8BC7047F00207C4F8BC7017070BD5D2
:1011000005F02007374307D008261E62D4F8BC60DC
:1011100046F00806C4F8BC6017050AD56E0108D56C
:101120004FF400661E62D4F8BC6046F02006C4F896
:10113000BC60D4F8BC60002E3FF474AF92060AD5B0
:1011400005F0200501F080510D4304D0D4F8A02013
:101150000AB19047636BD4F8BC109A6801F028017B
:1011600002F040020A434CD019682020284A21F49A
:101170009071196099680A4000219A60C4F8B8001B
:101180009A68C4F8A01057067FF54CAF9A68D4F857
:10119000AC0022F040029A6000283FF443AF90F880
:1011A00035201C4B022A036528D1FEF75FFF00287B
:1011B0003FF438AFD4F8AC00036DBDE8F0411847F8
:1011C000CF079BD502271F62D4F8BC7047F00407F5
:1011D000C4F8BC70570791D588E7D4F8A430002B29
:1011E000EBD11FE7D70789D5EF053FF571AF97071B
:1011F00084D477E74FF480121A6213E780224265A5
:10120000DBE7C4F8BC200DE701000010200100045A
:10121000FEFFFFEF910E0408D0E907239A423CBF7E
:10122000C1685218D01A7047D0E9092300699A4260
:1012300038BF12180138D31AC01A7047D0E9090212
:10124000101AB0FA80F04009704700BF016A0346E7
:1012500040694A1C405CD9688A4228BF00221A6251
:10126000704700BF436A826910B4D154436A416B2E
:10127000046901330A68A34228BF00235DF8044BC8
:1012800042F0800243620A60704700BF436BD86936
:1012900010F0100002D0102201201A62704700BF27
:1012A000B24BD3E9011270B58C0F93F88850100E31
:1012B000C2F3072C83F83040C1F383640001012D91
:1012C00083F83140C1F3016483F83240C1F307442D
:1012D00083F83340C1F30724C9B283F83440C2F322
:1012E000035483F83510D886C2F3C030D98E89B242
:1012F00041EA0401C2F30344D986C2F3403183F8C2
:101300003840C2F3803483F839004FF0000083F88E
:101310003A4083F83B10C2F3003183F83C10D9689F
:1013200083F83D0040F2D480022D00F0B0802A20E6
:101330004FEA4C0C83F84940C1F3C01201F07F0121
:101340000CF07E0C83F84AC04FF0010C93F84A4031
:1013500014431A6983F84A40D40F83F84B10910D57
:1013600083F84C40C2F3417401F00C01C2F3815583
:1013700083F84D40C2F3826483F84E4083F84F10E7
:1013800093F84F105C69294383F84F10C2F3405122
:1013900083F85010002183F85110C2F3004183F804
:1013A0005210C2F3C03183F85310C2F3803183F876
:1013B0005410C2F3403183F85510C2F3003183F862
:1013C0005610C2F3812183F85710C2F30121C2F3F2
:1013D000460283F85810C4F3074183F85920220EBF
:1013E000090283F85AC083F85C20C4F30722A3F8EB
:1013F0005E102406B3F85E1089B21143A3F85E10A4
:1014000099691C660C0E1A6E42EA04421A660A0AB0
:101410001C6E02F47F422243C1F30724C9B21A664C
:101420001D6EDA692C431C6683F86410110E83F874
:101430006510110C0906996611029C6E0A4601F4AA
:101440007F01214392B21C6A9966996E0A439A669B
:10145000C4F30352996E41EA1461996693F86C10D3
:101460001143C4F3072283F86C10210A01F4706160
:10147000A3F86E10B3F86E1089B21143C4F346029C
:10148000A3F86E1083F8702083F871C070BD120449
:10149000C1F3072C0D0E02F47C121A64C1F307424B
:1014A0001C6C44EA05241C641C6C22434FF4007439
:1014B0001A641A6CC3F88040013240F10004A4029F
:1014C00044EA92549202DC67C1F380349A672FE7B2
:1014D0004FEA8C2CC1F3C26594000CF44062C1F356
:1014E000072C04F47F741A641A6C1443CA0B1C642E
:1014F00002F006021C6C44EA91741C64C1F302649D
:1015000083F84450012583F84540C1F3425483F8E1
:101510004640C1F3824483F84740C1F3C03483F8A6
:10152000482093F84820224383F848201C6C93F805
:10153000482093F83860023205FA02F2B540D61717
:10154000A2FB052EC3F8805005FB06EE04FB0EEE51
:101550000134A2FB0424A644520AC1F3803442EAB7
:10156000CE529A674FEA5E22DA67E1E6002F002446
:10157000704700BF704700BF704700BF0120704731
:10158000014BD3F88C007047002F0024044B93F8D4
:101590002C03A0F10300B0FA80F04009704700BFAF
:1015A000002F0024012380F849307047EFF31182A7
:1015B000702383F312880849D2B2D1E9D93182F37A
:1015C0001188581E8B42A0EB01008CBF0023012321
:1015D00000EB0330704700BF002F002401F00F0123
:1015E000D0F8D022C1EBC10102EB8102D0E9AE30CC
:1015F000D2F8142203F5037110B5C468D3F80402BD
:10160000C3F80C22A047002010BD00BFD0F8BC32A8
:1016100083B110B5D0F8B84294F80002FF2807D083
:101620009B68214694F801229847FF2384F80032F2
:10163000002010BD002070470346432201481A8055
:10164000704700BF040000240346432201481A806B
:10165000704700BF480000240346432201481A8017
:10166000704700BF8C00002403460A2201481A80FC
:10167000704700BFD0000024064B4FF0120C064A02
:10168000A3F11400526DA1F800C0022A18BF184639
:10169000704700BFF00000240040005804230148B8
:1016A0000B807047040100241D48D0F80038D0F8A2
:1016B000082830B59B184FF01A040C8001D1194846
:1016C00030BD184A0024D0F8040802F11005114674
:1016D0004FEA137EB3F1204FCC7001F102010EF1FD
:1016E000370C38BF0EF1300C8D424FEA031381F8EE
:1016F00000C0EDD102F108050024010FB0F1204F28
:10170000D47402F1020201F1370338BF01F1300352
:1017100095424FEA00101374EFD1024830BD00BF6C
:1017200000E0F11F0801002400207047212808B5BF
:1017300027D0222818D0202814D199B1072A11D1F6
:10174000184A194B0868B1F804C0D2F86C2389799B
:10175000C3F82401A3F828C183F82A1112B1014665
:1017600000209047002008BD0029FBD0022AF9D1B3
:101770000C4BD3F87033002BF4D009880020984725
:10178000F0E70029EED0072AECD1074BD3F824016B
:10179000B3F8282193F82A31086000208A808B71E1
:1017A00008BD00BF002F002400000024034B93F865
:1017B0009803003818BF0120704700BF002F002495
:1017C000304B0021304A1B683048A2FB032310B580
:1017D000DB0C2F4C82B0013BC4F8DC13C4F8D413EB
:1017E00042F20F7194F80924C4F8CC03C4F8D8135A
:1017F000C4F8D033002A3FD002232649234884F876
:101800000934FFF779FA244B01220621372084F8A6
:101810000924D3F8E82042F02002C3F8E820D3F8E6
:10182000E83003F020030193019B74F06BF9D4F8C6
:10183000CC334FF400001949194A4860D96841F087
:101840000101D96099680A40062A06D0B2F5803FA6
:1018500003D01A6842F001021A600020D4F848331D
:101860001049114AC3F81002C4F87003C4F86C039D
:10187000C3E9812102B010BD02F0FF0084F8080422
:10188000BAE700BF0000002483DE1B4300140040C1
:10189000002F0024D03200240044025800E100E070
:1018A00007000100884D0024883D00242DE9F84FF1
:1018B000234E80468946D6F84833D3F81422002AAE
:1018C000FBD1B9F1000F37D008EB090ADFF874B08B
:1018D00008F1FF3870270AF1FF3AD6F8682318F8A4
:1018E000011F531C0BF80210C3F30B03C6F8683337
:1018F000EFF3118287F31288D6E9D931D2B282F39D
:1019000011888B42A3EB01038CBF0022012203EB61
:101910000233012B0ED110F08BFF04460D4610F060
:1019200087FF001B61EB0501B0F57A7F71F10001C3
:10193000F5D3DDE7D045D0D14846BDE8F88F00BFEC
:10194000002F0024884D0024F8B50C4E96F82C3357
:10195000032B00D0F8BD0D461446D6F80C7408E0F1
:10196000FFF7A4FFD6F80C34241A0544DB1B322BF6
:10197000F0D8002C21462846F2DCF8BD002F0024C8
:10198000F8B590F848305D1C0344EDB280F848503B
:1019900083F8341090F8493053B1132D07D9002340
:1019A00080F848300E4F97F82C33032B05D0F8BD44
:1019B00080F84830002DF5D1F8BDD7F80C6400F15F
:1019C000340429462046FFF771FFD7F80C342D1A4E
:1019D00004449B1B322BEAD8002DF2D1F8BD00BF86
:1019E000002F0024F8B5002390F84850A0F84830A4
:1019F00005B9F8BD0B4F97F82C33032BF9D1D7F865
:101A00000C6400F1340429462046FFF74FFFD7F855
:101A10000C342D1A04449B1B322BEAD8002DF2D132
:101A2000F8BD00BF002F00242DE9F047046982B003
:101A3000C3681C4046D0814688464FF0004501F1FE
:101A4000500701F13806B4FA84F325FA03F21B3B80
:101A5000D2431440C9F81020B8F1000F5FD0042B16
:101A60002ED8DFE803F052483D320300D8F810309A
:101A7000D9F82CA033B19B6823B11FFA8AF108F181
:101A800008009847D8F8283033B19B6823B11FFA73
:101A90008AF108F120009847D8F8403033B19B68AC
:101AA00023B11FFA8AF108F138009847D8F8583066
:101AB00033B19B6823B11FFA8AF108F150009847AF
:101AC000002CC0D102B0BDE8F087D8F8103008F182
:101AD0000800D9F834105B689847002CB3D1F1E7BF
:101AE000D8F8283008F12000D9F838105B689847FA
:101AF000002CA8D1E6E7D8F840303046D9F83C10A1
:101B00005B689847002C9ED1DCE7D8F858303846FF
:101B1000D9F840105B689847002C94D1D2E7042B89
:101B200007D8DFE803F01903140F0A00D9F83C3096
:101B30000193019B002C86D1C4E7D9F82C30019386
:101B4000019BF7E7D9F834300193019BF2E7D9F80C
:101B500038300193019BEDE7D9F840300193019BA8
:101B6000E8E700BF234938B5D1F810346BB1D1F89C
:101B70008C20002AFAD0013A13F8014BC1F88C20CE
:101B8000C1F8103412B1204638BDFEE7D1F8483311
:101B9000002BF8D091F8A000D3F80452D1F86033AC
:101BA000A8B91A690121C3F830024FF40070012A64
:101BB000A3F81812C3F8245203F50671C3F82C02D7
:101BC00014D01868D2B277F0F5FC204638BDC3F8BF
:101BD000302201211A694020A3F8181203F506717A
:101BE000012AC3F82452C3F82C02EAD1C3F82852C0
:101BF000E7E700BF002F0024D0F8B822002A3DD02C
:101C000001EB810300EB830370B5DC69D0F8D0529F
:101C100024B90023C2F81432002070BDC1EBC10CFE
:101C200005EB8C0CDCF84460B4FBF6FC06FB1C44B2
:101C3000002CEED101F07F02DC6101F00F031C21CA
:101C400002EB820201FB035100EB8200C3EBC302F3
:101C50003C31C46105EB82000122846480F83C3091
:101C600080F83D20C0E914442A69012AD2B208BF95
:101C7000C464286823B977F0ADFDCDE70220704732
:101C800077F098FCC8E700BF184B0A68C3F8100447
:101C9000C3F88C200AB100207047D3F848130029FC
:101CA000F9D010B593F8A000D1F80442D3F860330E
:101CB000A0B140200121C3F82442C3E98B021A6974
:101CC0001868012AA3F81812D2B203F5067108BFEA
:101CD000C3F8284277F06EFC002010BD4FF400726C
:101CE0000121C3F82442C3E98B20E8E7002F002438
:101CF00070B5037C0446D0F8D002002B45D14FF4D8
:101D000000730222812177F055FB01214FF400730B
:101D10000222D4F8D002E16277F04CFB01260823BE
:101D200003228221D4F8D002C4F86C6177F042FB20
:101D30004FF40770266481F0E9FD0546C4F8B80247
:101D4000002842D0D4F8BC321B6898470022217C7E
:101D5000C5F81422D4F8D032D5F80402C5F81822F8
:101D600009B3C3F8302240241A6903F50671C3F899
:101D70002402012AA3F81862C3F82C4222D0186862
:101D8000D2B277F017FC002070BD402302228121DF
:101D900077F010FB012140230222D4F8D002E16247
:101DA00077F008FBBAE71A694FF40074C3F83012F1
:101DB00003F50671B242C3F82402A3F81862C3F80F
:101DC0002C42DCD1C3F82802D9E7304670BD00BFF1
:101DD00070B5D0F8D05240F20112044695F8BC33E9
:101DE000A5F85820012B09D001222868114685F852
:101DF000BC2377F0CBFD002385F8BC33D4F8D05258
:101E000000260121E66295F8BC33A5F818128B4232
:101E100007D03246286885F8BC1377F0B7FD85F8FF
:101E2000BC63D4F8D05200264FF48172C4F86C61C0
:101E300095F8BC33A5F87420012B08D001220221AB
:101E4000286885F8BC2377F0A1FD85F8BC630025E0
:101E5000D4F8B83225644BB1D4F8BC325B689847EB
:101E6000D4F8B80281F05AFDC4F8B852002070BD11
:101E70002DE9F0410B7882B000260D4613F0600783
:101E80000446D0F8B8828DF80560ADF8066035D00C
:101E9000202F0DD08021D4F8D00277F031FB002123
:101EA000D4F8D00277F02CFB022002B0BDE8F0811C
:101EB000CA884878002A37D01B064FD5D4F8BC32E0
:101EC00041469B6898470223EA884FF48071C4F822
:101ED0009432D4F8D032C4E907221A651A69998776
:101EE00003F13C01012AC3F848805E6501D1C3F8C3
:101EF0004C80D2B2186877F06DFC19E04D780A2D4D
:101F00001DD00B2D16D0002DC4D190F89C32D0F8E6
:101F1000D002032B55D0802177F0F2FA2946D4F86D
:101F2000D00277F0EDFABFE7D4F8BC329B6898474F
:101F30000020BAE790F89C32032BF9D0AAE790F87A
:101F40009C32D0F8D002032B23D0802177F0D8FA2E
:101F50003946D4F8D00277F0D3FAA5E7032388F8FE
:101F6000000288F80122C4F89432D4F8D032C4E9CF
:101F70005722C3F8102203F5FE711A69C3F80882CC
:101F8000012AC3F81462A3F8FC6108BFC3F80C82ED
:101F9000AFE7022201234FF48071C4F89422026952
:101FA000E3612362012A03650DF10503818700F1D6
:101FB0003C018364476516D0D2B2006877F00AFC12
:101FC000B6E70223026900F13C01C4F89432012A09
:101FD000C4E9073303654FF48073456583870DF1CA
:101FE00006038364E8D1C364E6E700BF08B520B9FF
:101FF000044873F0A3F8044808BD044873F09EF841
:10200000014808BD44EC0C081433002468EC0C08AB
:10201000024808B573F092F8014808BD8CEC0C0832
:1020200014330024024808B573F088F8014808BD4D
:1020300094EC0C0814330024024808B573F07EF8C1
:10204000014808BDA0EC0C081433002470B5124DF3
:10205000124A2B68A2FB03239B09013BB3F1807F4B
:1020600001D3012070BD4FF0E0220D4900240F285C
:1020700053614FF0F003064681F823304FF0070319
:1020800094611361EDD801464FF0FF3073F03AFDD3
:102090002046C5F82C6170BD00000024D34D6210AD
:1020A00000ED00E0034A0130116813685B1A8342B7
:1020B000FBD37047002F00243749024603688B4248
:1020C00033D01831591AB1FA81F1490969BB334843
:1020D000834240D01830834240D01830834236D0FB
:1020E000183083423DD01830834240D018308342AC
:1020F0002CD000F55670834237D029498B4233D01B
:1021000018318B4236D018318B4236D018318B4281
:1021100036D018318B4236D018318B4236D0183138
:102120008B4236D023F0FF0013E0DBB21D491E487E
:10213000103B10B41D4CA4FB03435DF8044B01EBB2
:10214000131393F82810C2E9160170471621184896
:10215000D1659065704710211348F9E716211248A0
:10216000F6E706211248F3E706211248F0E71021AE
:102170000F48EDE710210F48EAE716210D48E7E781
:1021800000210D48E4E706210B48E1E710210A4849
:10219000DEE716210848DBE710000240400002405D
:1021A0002804024018450C0800000240ABAAAAAA65
:1021B0000400024000040240040402400C4A136977
:1021C00003F03803102B0DD0182B09D063B9136816
:1021D0009B060BD513680748C3F3C103D84070476B
:1021E000FEF718BD0448704704487047014870471F
:1021F000004402580090D00300127A0000093D000C
:10220000194A136903F03803102B10B526D0182B88
:1022100009D02BBB13689B0624D513681348C3F35E
:10222000C103D84001E0FEF7F5FC0F49104A8B6965
:10223000104CC3F30323134493F8303003F01F030F
:1022400020FA03F32360896901F00F010A4492F830
:10225000300000F01F0023FA00F010BD0648E4E74C
:102260000648E2E70148E0E7004402580090D00346
:1022700018450C080000002400127A0000093D00F7
:10228000474A70B4946A956AD66A15F47C3FC5F3E0
:102290000533D16B5BD0C1F3CC01C6F3001604F05B
:1022A000030407EE903A06FB01F1012CB8EEE77A41
:1022B00006EE901AFAEEE96A03D0022C6AD0002CDE
:1022C0004AD0DFED387A87EE876A936BC3F3080351
:1022D00007EE903AF7EE005AF8EEE77A77EEA67A34
:1022E00077EEA57A67EE867A2D4AB7EE006A936B91
:1022F000C3F3462307EE103AB8EEC77A70BC37EE48
:10230000067AC7EE876AFCEEE66AC0ED006A936B58
:10231000C3F3064307EE103AB8EEC77A37EE067AF3
:10232000C7EE876AFCEEE66AC0ED016A936BC3F301
:10233000066306EE903AF8EEE66A76EE866A87EE77
:10234000A67AFCEEC77A17EE903A8360704770BCAD
:10235000C0E900338360704713689B061DD514687D
:10236000F7EE005A936B1049C4F3C102C3F308039C
:10237000D14007EE903A06EE101AF8EEE77AB8EE82
:10238000C66A77EEA66AC6EE077A36EEA57A67EEDB
:10239000877AA9E7DFED057A95E7DFED057A92E721
:1023A000004402580024744A0090D0030024F44AE8
:1023B0000024744C474A70B4946A956AD66A15F042
:1023C0007C7FC5F30553516C5BD0C1F3CC01C6F3E0
:1023D000002604F0030407EE903A06FB01F1012CFD
:1023E000B8EEE77A06EE901AFAEEE96A03D0022C0C
:1023F0006AD0002C4AD0DFED387A87EE876A136CFA
:10240000C3F3080307EE903AF7EE005AF8EEE77AC6
:1024100077EEA67A77EEA57A67EE867A2D4AB7EE42
:10242000006A136CC3F3462307EE103AB8EEC77A7E
:1024300070BC37EE067AC7EE876AFCEEE66AC0ED3E
:10244000006A136CC3F3064307EE103AB8EEC77A7E
:1024500037EE067AC7EE876AFCEEE66AC0ED016ADF
:10246000136CC3F3066306EE903AF8EEE66A76EE76
:10247000866A87EEA67AFCEEC77A17EE903A8360FA
:10248000704770BCC0E900338360704713689B06D7
:102490001DD51468F7EE005A136C1049C4F3C1023D
:1024A000C3F30803D14007EE903A06EE101AF8EE97
:1024B000E77AB8EEC66A77EEA66AC6EE077A36EE17
:1024C000A57A67EE877AA9E7DFED057A95E7DFED74
:1024D000057A92E7004402580024744A0090D00321
:1024E0000024F44A0024744CD0E9041283680B439E
:1024F000C16970B513430446056886B0626E0B432C
:1025000028681343A44A666A02401343E2682B60BA
:102510006B6823F440531343A2696B609F4B9D4249
:1025200000F02D82236AA8681A439D4B03401A438A
:10253000AA60EB6A23F00F033343EB62994B9D4291
:1025400028D0994B9D421AD0984B9D4217D0984B5A
:102550009D4214D0974B9D4211D0974B9D4219D06C
:10256000964B9D420BD0964B9D4208D001200023F4
:102570004FF00112C4E91A23236706B070BD914BD6
:102580005B6D03F00703052BF0D8DFE803F0C65FAF
:102590007AAE8D9D8B4B5B6D03F03803282BE5D80D
:1025A00001A252F823F000BF492804086D25040851
:1025B0006D2504086D2504086D2504086D250408A3
:1025C0006D2504086D2504084D2604086D250408B2
:1025D0006D2504086D2504086D2504086D25040883
:1025E0006D2504086D250408832604086D2504085C
:1025F0006D2504086D2504086D2504086D25040863
:102600006D2504086D250408EB2604086D250408D3
:102610006D2504086D2504086D2504086D25040842
:102620006D2504086D250408A92604086D250408F5
:102630006D2504086D2504086D2504086D25040822
:102640006D2504086D250408C9260408B1F5004F5E
:1026500000F0468103A8FFF713FE049B002E40F014
:102660008280626803EB5203B3FBF2F39BB2A3F1E7
:1026700010014FF6EF7291423FF678AFEB60002009
:1026800075E7B1F5004F00F0FD806846FFF792FE58
:10269000019B002EE5D0013E0A2EE2D84A4A52F8AC
:1026A0002620B3FBF2F3DCE7B1F5004F00F03981EF
:1026B000002E56D0013E0A2E53D8444A444B52F8BD
:1026C0002620B3FBF2F3CCE7B1F5004F00F0178101
:1026D000002E43D0013E0A2E40D83E4A4FF400431C
:1026E00052F82620B3FBF2F3BBE7B1F5004F00F040
:1026F0002481344B1A6892063FD51A68364BC2F3D0
:10270000C102D340002EACD0013E0A2EA9D8334AD4
:1027100052F82620B3FBF2F3A3E7B1F5004F67D0E0
:10272000FFF76EFD274A2E4BD269C2F30212134403
:10273000626A93F8303003F01F03D8403AB1013A8F
:102740000A2A04D8274B53F82230B0FBF3F0626812
:1027500000EB5203B3FBF2F39BB288E74FF4004364
:102760007FE71B4B7DE7013E0A2E3FF67AAF1E4AFC
:1027700052F82620B3FBF2F373E7002E00F0FD8041
:10278000013E0A2E00F2F980184A134B52F8262017
:10279000B3FBF2F365E700BFF369FFCF000C00580D
:1027A000FFF4FF11001001400044004000480040C9
:1027B000004C0040005000400014014000780040F0
:1027C000007C00400044025858450C0858450C084D
:1027D00000093D0058450C080090D00358450C08EE
:1027E00018450C0858450C0858450C0858450C0865
:1027F000FFF706FDB34AB44BD269C2F30212134489
:10280000626A93F8303003F01F03D8403AB1013ABE
:102810000A2A04D8AD4B53F82230B0FBF3F06268BB
:10282000530803EB4003B3FBF2F39BB2A3F1100197
:102830004FF6EF7291423FF699AE23F00F02C3F3C9
:1028400042031343EB601AE7B1F5004F2FD0FFF7B7
:10285000D7FC9C4A9C4BD269C2F302221344626AA1
:1028600093F8303003F01F03D840002A3FF46FAFD5
:10287000013A0A2A3FF66BAF954B53F82230B0FB72
:10288000F3F064E76846FFF795FD01993EB1013E1C
:102890000A2E04D88F4B53F82630B1FBF3F162684F
:1028A000530803EB4103B3FBF2F39BB2BEE7FFF720
:1028B000A7FC844A844BD269C2F302221344626AA1
:1028C00093F8303003F01F03D840002AA7D0013A14
:1028D0000A2AA4D8804B53F82230B0FBF3F09EE7CD
:1028E00003A8FFF7CDFC0499002ED8D0013E0A2E94
:1028F000D5D87A4B53F82630B1FBF3F1CFE7002E51
:1029000036D0013E0A2E33D8754B53F82630B1FB32
:10291000F3F35B00626803EB5203B3FBF2F39BB289
:1029200084E746B3013E0A2E25D86E4A6E4B52F814
:102930002620B3FBF2F35B00ECE7624B1A689106CA
:1029400040F1C2811B68694AC3F3C103DA403EB15A
:10295000013E0A2E04D8664B53F82630B2FBF3F240
:1029600061684B0803EB4203B3FBF1F39BB25DE7F5
:102970004FF48033CEE75F4BCCE75C4B71E6A96840
:102980005D4B0B4013434F4AAB60EB6A23F00F03E0
:102990003343EB62936D03F00703052B3FF6E6AD7F
:1029A000DFE803F0D0C1B2776803002E00F0788131
:1029B000013E0A2E00F27481504A4FF40040402339
:1029C00052F82620B0FBF2F000283FF458AE6568BC
:1029D00005EB450282423FF6C9ADB0EB053F3FF63D
:1029E000C5AD202B00F27E81023B1E2B3FF6BEAD13
:1029F00001A252F823F000BF4D2C04086D250408F5
:102A0000272C04086D2504086D2504086D2504088D
:102A1000012C04086D2504086D2504086D250408A3
:102A20006D2504086D2504086D2504086D2504082E
:102A3000C72B04086D2504086D2504086D250408BE
:102A40006D2504086D2504086D2504086D2504080E
:102A50006D2504086D2504086D2504086D250408FE
:102A60006D2504086D2504086D2504086D250408EE
:102A7000772B0408002E00F01781013E0A2E00F289
:102A800013811F4A2023184852F82620B0FBF2F089
:102A90009AE70C4B1A68950640F109811B681348A8
:102AA000C3F3C103D840002E00F0F880013E0A2E87
:102AB00000F2F480134A102352F82620B0FBF2F003
:102AC00082E700BF0044025818450C0858450C081E
:102AD00058450C0858450C0858450C0858450C0832
:102AE00058450C0858450C0800093D000090D003DB
:102AF00058450C0800127A00FFF4FF1158450C08E5
:102B000058450C0858450C086846FFF753FC0198D7
:102B10003EB1013E0A2E04D8864B53F82630B0FB56
:102B2000F3F0082350E703A8FFF7AAFB04983EB18F
:102B3000013E0A2E04D8804B53F82630B0FBF3F048
:102B4000042341E7FFF75CFB7C4B7D491B6A626A0B
:102B5000C3F302130B4493F8303003F01F03D84043
:102B60003AB1013A0A2A04D801EB82010B6CB0FB9E
:102B7000F3F0022328E7616A002900F0CE800139D2
:102B80000A2900F2CF806F4B6F4803EBC103D3E9F2
:102B90000023002178F016FE03460902180241EADC
:102BA00013616B0818182A464FF0000341F1000129
:102BB00078F008FEA0F54072644B9A423FF6D6AC1E
:102BC000634BD8605BE55D4A636A1168880640F133
:102BD0009680126800215F48C2F3C102D0404BB119
:102BE000013B0A2B06D85C4A02EBC303D3E900235E
:102BF00078F0E8FD0902030241EA10616808D1E7B4
:102C00006846FFF7D7FB636A01980021002BF1D0DB
:102C1000013B0A2BEED8514A02EBC303D3E9002350
:102C200078F0D0FDE6E703A8FFF72AFB636A049873
:102C30000021002BDED0013B0A2BDBD8484A02EBF7
:102C4000C303D3E9002378F0BDFDD3E7FFF7D8FA3B
:102C50003A4B3B4D00211B6A626AC3F302132B44BB
:102C600093F8303003F01F03D84042B1013A0A2AEA
:102C700005D805EBC205D5E91C2378F0A3FD6268F1
:102C80000902030241EA1061500818184FF00003CE
:102C900041F1000178F096FD8CE72E48102396E66E
:102CA0004FF40040402392E6274820238FE6002E71
:102CB000F3D0013E0A2EF0D82A4A1023254852F8B4
:102CC0002620B0FBF2F07FE656B1013E0A2E07D86F
:102CD000254A204B52F82620B3FBF2F35B0019E69D
:102CE000224B17E6616AA9B101390A291DD8204B88
:102CF0004FF4004003EBC103D3E9002349E773B16C
:102D0000013B0A2B0BD81B4A124802EBC303D3E941
:102D100000233EE74FF4000043E7174841E7174818
:102D200003213EE7144800213BE74FF40000002157
:102D300037E700BF58450C0858450C0800440258B6
:102D400018450C0888450C0800093D00FFFC0F00E1
:102D5000000C00580090D00388450C0888450C08EA
:102D600088450C0858450C0858450C080020A10758
:102D700088450C0888450C080000093D000090D0EB
:102D8000344A136830B423F08063334C13602568F1
:102D900003E023685B1B022B54D813681B01F8D493
:102DA000936A056823F47C3343EA053393628368AE
:102DB000C568013B013D5B022D049BB205F4FE0595
:102DC0002B434568013DC5F308052B430569013DCB
:102DD0002D0605F0FE452B439363D36A456923F026
:102DE000C0032B43D362D36A856923F020032B43AE
:102DF000D362D36A23F01003D362D36BC0696FF33D
:102E0000CF0343EAC003D363D36A43F01003D36212
:102E1000D36AD1B101290CBF43F4801343F40013EA
:102E2000D3620C4A136843F080631360216803E0A7
:102E300023685B1A022B05D813681B01F8D5002004
:102E400030BC7047032030BC704743F40023D3628A
:102E5000E7E700BF00440258002F0024344A1368FB
:102E600030B423F08053334C1360256803E02368AB
:102E70005B1B022B54D813689B00F8D4936A056837
:102E800023F07C7343EA055393628368C568013B72
:102E9000013D5B022D049BB205F4FE052B43456802
:102EA000013DC5F308052B430569013D2D0605F0DD
:102EB000FE452B431364D36A456923F440632B43D7
:102EC000D362D36A856923F400732B43D362D36A38
:102ED00023F48073D362536CC0696FF3CF0343EA6A
:102EE000C0035364D36A43F48073D362D36AD1B10D
:102EF00001290CBF43F4000343F08073D3620C4AF2
:102F0000136843F080531360216803E023685B1A61
:102F1000022B05D813689B00F8D5002030BC704701
:102F2000032030BC704743F48003D362E7E700BF5F
:102F300000440258002F00244B4B10B41B684B4C2C
:102F4000A4FB03435B0A03FB02F25AB18446531EFF
:102F50004748DCF83420013B024201D0920406D5F8
:102F60005C1CF6D14FF000405DF8044B7047DCF874
:102F700034305C0741D4DCF83430D80709D43D4BF9
:102F8000CCF83830DCF81030DBB2994205D00120A3
:102F9000EAE70123CCF83830F9E7DCF8143036489A
:102FA00018400028E0D0002B2CDB5A002DD49C00C8
:102FB0002DD4D9002DD41A012ED45C012FD4D901DF
:102FC00030D41A0231D45C0232D499023CD4DA02F1
:102FD00037D45C0332D499032DD4DA0340D41C04D3
:102FE0003BD4590436D49A0431D413F0080F0CBFE3
:102FF0004FF480304FF40000B6E704231846CCF8B5
:103000003830B1E74FF00070AEE74020ACE78020E9
:10301000AAE74FF48070A7E74FF40070A4E74FF4DD
:103020008060A1E74FF400609EE74FF480509BE77B
:103030004FF4005098E74FF4802095E74FF40030AC
:1030400092E74FF400408FE74FF480408CE74FF455
:10305000800089E74FF4001086E74FF4801083E783
:103060004FF4002080E700BF00000024D34D621021
:1030700045002000C500200008E0FFFD38B5134DD5
:1030800041F20D13124941F28832D5F85805D5F8AE
:1030900014450004A060E068014020460B430D2168
:1030A000E360FFF749FF38B1D5F848250346002013
:1030B0001343C5F8483538BD606900F4F050A0F5F9
:1030C0000060B0FA80F0400938BD00BF002F002436
:1030D000C0E0FEFF38B5184C0020184941F20D132E
:1030E000D4F85825D4F814551204C4F8940328468B
:1030F000AA60EA68114041F288320B430D21EB606F
:10310000FFF71AFF68B1D4F848350343C4F84835CF
:10311000D4F80C2409230020C4F8882384F89833B9
:1031200038BD6B6903F4F053B3F5006FF0D104239D
:10313000022084F8983338BD002F0024C0E0FEFF41
:1031400070B50D4D04460E4695F89833042B0BD000
:10315000082B07D1D5F8903383420AD0FFF7BAFF86
:10316000022801D0012070BD0823C5E9E44685F896
:103170009833022070BD00BF002F00240A4B013B92
:103180000FD00269002AFADA0369074A43F0010303
:103190000361013A05D0036913F00103F9D1184620
:1031A00070470320704700BF410D03002DE9F84F21
:1031B000066880460C46C6F3100535BB654B9E423B
:1031C00079D903F500339E4274D903F500339E424A
:1031D00040F2B48003F500339E4240F2B18003F523
:1031E00000339E4240F2AE8003F500339E4240F22F
:1031F000AB8003F500339E4240F2A880B6F1016F28
:10320000C0F0A68005200FF085FF534F354697F894
:10321000A435012B00F0898006F178464FF00109B2
:103220000023B6F5801F87F8A495C7F8A83536D3D4
:10323000022072F00BFC002874D1484A4FF00209BA
:10324000D2F80C3143EA0903C2F80C31BFF36F8F97
:10325000BFF34F8F04F1200254F8043B944245F829
:10326000043BF9D1BFF36F8FBFF34F8F484672F025
:10327000EDFBB9F1010F394A5BD0D2F80C3123F0E4
:103280000203C2F80C31002387F8A43500284CD182
:10329000D8F800302033C8F80030BDE8F88F484631
:1032A00072F0D4FB00283DD12C4AD36843F00203CE
:1032B000D360CBE70125284F97F8A435012B0ED01A
:1032C0004FF0010A4FF0000B504687F8A4A5C7F84D
:1032D000A8B572F0BBFB814628B187F8A4B54FF0C2
:1032E000FF30BDE8F88F5046DFF870A0DAF80C30F8
:1032F00023F4E663CAF80C30DAF80C3043EA05230D
:1033000043F0A403CAF80C3072F0A0FBDAF80C20EA
:10331000134B1340CAF80C3087F8A4950028DED16F
:10332000354679E7002387F8A4356FF00100BDE842
:10333000F88FD36823F00203D360A4E70225BAE72D
:103340000325B8E70425B6E70525B4E70625B2E767
:103350000725B0E7FFFF0108002F002400200052DE
:10336000FBF8FFFF0148FDF741B800BFB03400246F
:10337000084810B4D0F8B035D0F8E44599691A6817
:103380002CB1234600F5B6605DF8044B18475DF894
:10339000044B7047002F00240148FDF727B800BFF9
:1033A00000350024084810B4D0F80036D0F8344670
:1033B00099691A682CB1234600F5C0605DF8044B8A
:1033C00018475DF8044B7047002F00240148FDF7B3
:1033D0000DB800BF50350024084810B4D0F850365E
:1033E000D0F8844699691A682CB1234600F5CA6062
:1033F0005DF8044B18475DF8044B7047002F00241C
:103400002DE9F04FDFF8689300EB400583B04300EF
:1034100009EB85050093D5F830310193002B00F0BE
:1034200066818046B5F8360171F0B0FE95F834013A
:103430000BF07AFC044695F835010BF075FC08F1A9
:1034400001030746DBB2002C00F0768140F60C1237
:10345000A1882372E2802268002800F06181037253
:1034600040F60C23C38091613B68BA889A611121B0
:10347000204609260BF014FC112138460BF010FCF5
:103480006525002C00F036812268A38811690B4263
:1034900000F030811B0493610FF0CAF905468B469A
:1034A0000FF0C6F9401B61EB0B01052871F100011B
:1034B000F6D314B12368A2889A610FF0B9F90546D2
:1034C0008B460FF0B5F9401B61EB0B01052871F13C
:1034D0000001F6D3013ED3D11CB1A38822681B049E
:1034E00093610FF0A5F905460E460FF0A1F9401BB8
:1034F00061EB0601052871F10001F6D31FB1BB880D
:103500003A681B0493610FF093F905460E460FF0DD
:103510008FF9401B61EB0601052871F10001F6D31C
:1035200014B12368A2889A610FF082F905460E460D
:103530000FF07EF9401B61EB0601052871F10001D7
:10354000F6D317B13B68BA889A61009B20463E21AA
:103550004FEA8805434409EB830393F83B41224635
:103560000BF0C0FB224638463E210BF0BBFB7B4CE8
:1035700008EB8803019A04EB0313C3F8B025784BDA
:103580009A4200F0C880FEF73BFE764BDA69C2F340
:103590000212754B134493F8303003F01F03D840E8
:1035A000009B434409EB830393F83831022B00F06E
:1035B000BE80032B00F0B680012B14BF4FF4C871FE
:1035C0004FF4487171F070FE034605EB08020021CC
:1035D00004EB0212C2F8B815C2F8C015C2F8C4153F
:1035E000C2F8CC15C2F8D0150121C2F8B435C2F822
:1035F000BC1592F8F11501F0FF00002900F0A4803D
:1036000005EB080123F0706224274FF4004C04EB13
:1036100001115648D1F8B03581F8F1751E6826F0D1
:1036200001061E601A619A6822F400429A60C3F88B
:1036300008C05A681043D1F8C82558601202D868EB
:1036400020F40040D860DA6000221A60186840F068
:10365000010018602020C1F8F42581F8F105C1F8B7
:10366000E02581F8F22591F8F1052028C6B217D19E
:1036700091F8F005012813D081F8F175186820F051
:1036800001001860186820F48050186018681860ED
:10369000186840F00100186081F8F16581F8F025A4
:1036A000009B0221DFF8CCA04544434404EB051401
:1036B00009EB830999F83A71384672F023FA99F8C0
:1036C000396107F01F034FF001097F09304609FAFD
:1036D00003F302214AF8273072F014FA06F01F03B0
:1036E000760909FA03F34AF8263084F8AC9503B05A
:1036F000BDE8F08F013D2AD00FF09AF883468A4644
:103700000FF096F8B0EB0B0061EB0A01052871F1A0
:103710000001F5D3B5E6FEF773FD124B1A6A36E7E2
:103720009161A4E6C82171F0BFFD03464DE7642115
:1037300071F0BAFD034648E700283FF498AE0372E3
:1037400040F60C23C3808FE682F8F00558E7002C82
:103750003FF4A2AEA38822689CE600BF002F00249D
:10376000001C00580044025818450C080080000254
:103770000000002400E100E02DE9F04F441C83B07C
:1037800091469DF8342031D000EB800CC04D0646A8
:10379000870005EB0C104FEA0C1C90F8ACA5BAF1B1
:1037A000000F23D0AC44B9F1FF0F9E464FEA410809
:1037B0000CF5B66400D0FBB9002A40F0B180BA190C
:1037C00005EB021292F8F115202906D1BEF1000F87
:1037D00016D14FF40073C2F8F435B5F89C36304674
:1037E00001339BB2A5F89C36FFF70AFE4FF0000AA2
:1037F000504603B0BDE8F08F90F8F125202AECD1B7
:10380000BA1905EB021292F8F0150129E5D0012151
:10381000D5F800B082F8F015D2F8B01505E02A68A6
:10382000A2EB0B02192A00F2ED80886910F4004027
:10383000F5D1BA194FF0210C0C9B05EB021282F85E
:10384000F1C54FF0400CC2F8D43582F8F2C5C2F889
:10385000E405C2F8F4058F48A2F8DAE54B68019256
:1038600003408D4843EA0803184348605946204600
:1038700072F0C2F8002840F06F81019AD2F8B015BA
:10388000C1F8289005E02B68A3EB0B030A2B00F28C
:1038900056818A6912F08002F5D0BA1905EB02123E
:1038A000B2F8DA359BB2FF2B40F26E814B687B4851
:1038B00003407B4843EA08031843FF23A2F8D835A6
:1038C000486007EB060905EB091905E0B9F8DA3598
:1038D0009BB2002B00F009815946204672F08CF80B
:1038E00000287FF47AAFD9F8D435D9F8B02513F889
:1038F000010BB9F8D8159062C9F8D4350139B9F877
:10390000DA3589B2013BA9F8D8159BB2A9F8DA35A6
:10391000B9F8DA359BB20029D8D1002BD6D0A1E076
:10392000BA1905EB021292F8F11520297FF455AF70
:1039300092F8F01501293FF450AF0121D5F800B0FD
:1039400082F8F015D2F8B01505E02A68A2EB0B0258
:10395000192A00F208818A6912F40042F5D1B819D7
:103960004FF0210C0C9B05EB001080F8F1C54FF0D7
:10397000100CC0F8D43580F8F2C5C0F8F425A0F8D2
:10398000DAE5B0F8DA35C0F8E4259BB2FF2B40F257
:103990000B814B683F4A1340424A43EA08031A43EB
:1039A000FF23A0F8D8354A6007EB060905EB091993
:1039B000B9F8DA35594620469BB2002B00F09780C3
:1039C00072F01AF800287FF408AFD9F8D435D9F886
:1039D000B02513F8010BB9F8D8159062C9F8D435A1
:1039E0000139B9F8DA3589B2013BA9F8D8159BB28B
:1039F000A9F8DA35B9F8DA359BB2002BD8D000290E
:103A0000D6D115E037442021002205EB0717D7F85F
:103A1000F43587F8F0250B43C7F8F43587F8F1152E
:103A200087F8F225D9E62B68A3EB0B030A2B3BD8CA
:103A3000916911F08001F6D0B9F8DA359BB2FF2B0D
:103A40006DD9536815490B40154943EA08031943DA
:103A5000FF23A9F8D8355160AAE72B68A3EB0B0325
:103A60000A2B21D8916911F08001F6D0B9F8DA3526
:103A70009BB2FF2B29D9536808490B40084943EAF8
:103A800008031943FF23A9F8D83551601EE700BF8A
:103A9000002F0024009800FC00200181009C00FC05
:103AA0000000FF010020FF81374405EB0717D7F81E
:103AB000F43587F8F01543F02003C7F8F4352023D8
:103AC00087F8F13587F8F21587E6B9F8DA353E4818
:103AD0009BB25168A9F8D835DBB2014048EA0343EC
:103AE0000B4343F000735360F0E65946204671F0F3
:103AF00059FF00287FF471AED9F8B0352021334C3E
:103B00003744D9615A6822405A60002205EB0713F6
:103B100089F8F11589F8F20583F8F02568E6B9F817
:103B2000DA3529489BB25168A9F8D835DBB2014093
:103B300048EA03430B4343F00073536038E7BB1973
:103B4000202005EB0313D3F8F4150143C3F8F41553
:103B500083F8F10583F8F225BB19002205EB031366
:103B600083F8F02539E6BB192020002105EB03136B
:103B7000D3F8F42583F8F0150243C3F8F42583F84D
:103B8000F10583F8F21528E6B2F8DA350E489BB253
:103B9000A2F8D835DBB24A6848EA0343024013432F
:103BA00043F000734B608CE6B0F8DA354A689BB29C
:103BB000A0F8D835DBB2064848EA03430240134375
:103BC000044A1A434A60EFE6009C00FC00E800FE4D
:103BD000009800FC002000822DE9F04F451C83B0C6
:103BE00014469DF8342000F08B800646DFF8C0A311
:103BF00000EB8000B7000AEB001C00019CF8AC95BC
:103C0000B9F1000F7CD05044FF2C9E464FEA41088A
:103C100000F5B6657AD1002A78D09CF8F125202AE3
:103C200065D19CF8F025012A61D00122DCF8B0159D
:103C3000DAF800408CF8F02505E0DAF80020121BD5
:103C4000192A00F21D818A6912F40042F5D1B819CF
:103C50004FF0220C0C9B0AEB001080F8F1C54FF0DE
:103C6000100CC0F8D43580F8F2C5C0F8F425A0F8DF
:103C7000DAE5B0F8DA35C0F8E4259BB2FF2B00F2A4
:103C80001581B0F8DA354A689BB2A0F8D835DBB2B6
:103C9000C14848EA034302401343C04A1A434A60FA
:103CA00007EB060B0AEB0B1BBBF8DA359BB2002BBC
:103CB00000F0CE81DBF8B0250CE0DBF8B02591698F
:103CC00011F0200140F04D81DAF800301B1B0A2B67
:103CD00000F270819369214628465B0700F1068156
:103CE0009369DB06EBD571F01FFE0028E5D0BAF82A
:103CF0009C36304601339BB2AAF89C36FFF780FB16
:103D00004FF00009484603B0BDE8F08FBA190AEB3E
:103D1000021292F8F1152029E9D10C99002900F03E
:103D2000C08092F8F0150129E1D00121DAF800B045
:103D300082F8F015D2F8B01506E0DAF80020A2EB10
:103D40000B02192A00F29C80886910F40040F4D11B
:103D5000BA194FF0220C0C9B0AEB021282F8F1C543
:103D60004FF0400CC2F8D43582F8F2C5C2F8E40531
:103D7000C2F8F4058848A2F8DAE54B6801920340DE
:103D800000F1044043EA080300F508401843486086
:103D90005946284671F030FE002840F0A080019A74
:103DA000D2F8B0158C6206E0DAF80030A3EB0B0312
:103DB0000A2B00F287808A6912F04002F4D0BA1907
:103DC0000AEB0212B2F8DA359BB2FF2B40F26481A3
:103DD0004B6871480340724843EA08031843FF23C5
:103DE000A2F8D8354860BC190AEB0414D4F8B01511
:103DF00006E0DAF80030A3EB0B030A2B00F2E980AF
:103E00008A6912F00402F4D04A6AD4F8D4351A70E0
:103E1000B4F8DA35B4F8D825013B013A9BB292B236
:103E2000A4F8DA35D4F8D435A4F8D8250133C4F889
:103E3000D435B4F8DA359BB213B1002A00F0EA8029
:103E4000B4F8DA359BB2002BD0D15946284671F030
:103E5000A9FD034600287FF44AAFD4F8B0252020FE
:103E6000504DD06151682940516084F8F10584F8C3
:103E7000F235374400230AEB071A8AF8F03541E798
:103E8000BB19202000210AEB0313D3F8F42583F893
:103E9000F0150243C3F8F42583F8F10583F8F21511
:103EA00025E74FF40073C2F8F43520E74B683A4A2F
:103EB00013403B4A43EA08031A43FF23A0F8D835CE
:103EC0004A60EDE6BB1920200AEB0313D3F8F41582
:103ED0000143C3F8F41583F8F10583F8F225BB1903
:103EE00000220AEB031383F8F02500E7526ADBF89F
:103EF000D4351A70BBF8DA35DBF8D425013B013232
:103F00009BB2CBF8D425ABF8DA35BBF8D835BBF883
:103F1000DA25013B92B29BB2ABF8D835002A3FF4C8
:103F2000C3AE002B7FF4C0AEDBF8B01504E0DAF8C6
:103F300000301B1B0A2B4CD88A6912F08002F6D085
:103F4000BBF8DA359BB2FF2B54D94B68164A1340A5
:103F5000164A43EA08031A43FF23ABF8D8354A60F0
:103F6000A2E69369590703D5BBF8D835002BBDD11C
:103F700020200C4CBB19D06151680AEB031321407F
:103F800051600022C3F8F42583F8F02583F8F10589
:103F900083F8F225ABE600BF009800FC0024008205
:103FA0000024FF8100E800FE009C00FC0000FF01EF
:103FB000002F002437440AEB0717D7F8F43587F8A9
:103FC000F01543F02003C7F8F435202387F8F135C6
:103FD0008DE6BB190AEB0313D3F8F41583F8F0252B
:103FE00041F02001C3F8F415202183F8F11583F87E
:103FF000F2257CE6BBF8DA352F489BB24A68ABF86D
:10400000D835DBB2024048EA0343134343F0007360
:104010004B6049E6D4F8B01505E0DAF80030A3EBC0
:104020000B030A2BD5D88A6912F08002F5D0B4F8B8
:10403000DA359BB2FF2B1FD94B681F4A13401F4A2A
:1040400043EA08031A43FF23A4F8D8354A60F7E689
:104050002146284671F0A6FC00287FF448AEDBF824
:10406000B0352021164CD9615A6822405A608BF82D
:10407000F1158BF8F205FCE6B4F8DA350E489BB280
:104080004A68A4F8D835DBB2024048EA0343134338
:1040900043F000734B60D3E6B2F8DA3509489BB2BF
:1040A000A2F8D835DBB24A6848EA0343024013431A
:1040B000054A1A434A6096E6009C00FC0000FF0196
:1040C00000E800FE009800FC002400820348D0F8BD
:1040D000603113B100F5AA70184770470000002442
:1040E0000348D0F8803113B100F5BA701847704713
:1040F000000000240348D0F8A03113B100F5CA70C5
:1041000018477047000000240348D0F8C03113B1AD
:1041100000F5DA7018477047000000240348D0F813
:10412000E03113B100F5EA70184770470000002431
:104130000348D0F8003213B100F5FA701847704701
:10414000000000240348D0F8203213B100F50570B8
:1041500018477047000000240348D0F8403213B1DC
:1041600000F50D7018477047000000240348D0F890
:10417000603213B100F51570184770470000002435
:104180000348D0F8803213B100F51D70184770470E
:10419000000000240348D0F8A03213B100F52570C8
:1041A00018477047000000240348D0F8C03213B10C
:1041B00000F52D7018477047000000240348D0F820
:1041C000E03213B100F53570184770470000002445
:1041D0000348D0F8003313B100F53D70184770471D
:1041E000000000240348D0F8203313B100F54570D7
:1041F00018477047000000240348D0F8403313B13B
:1042000000F54D70184770470000002410B41C469C
:10421000436884466FF30F0323434360036843F00E
:1042200001030360036843F400730360002C3AD079
:1042300040F2E930DCF814309B0748D5002A49D019
:1042400012F8013B40F2E9308CF82030DCF81430F1
:10425000DB0720D40138F9D1214B9C450CD0A3F5C4
:1042600078439C4538D003F580639C4536D003F5F0
:1042700078439C450BD103201A4A00EB400002EB27
:10428000C002B2F8683301339BB2A2F86833002051
:104290005DF8044B70479CF83000C0B209B101F8DA
:1042A000010B013CC4D1DCF814301B07FBD5DCF852
:1042B000183001205DF8044B43F01003CCF818309F
:1042C000DCF8003023F00103CCF8003070470138EF
:1042D000B0D1C1E7FF23B5E70120CDE70220CBE74E
:1042E00000300140000000242DE9F84300242C4E4A
:1042F0008046036856F83450AB4209D001340E2C86
:10430000F8D1284A0021052006F0CAFE002019E055
:10431000254B03EB8409D9F8A076AFB198F80510C6
:1043200000204B1C01EB410203EB430307EBC202ED
:10433000DB00C2F80C80C2E90400F854182303FB28
:1043400001700830BDE8F8830721682006F02EFFD1
:104350000146C9F8A006E8B1394668227EF0B6FEEB
:10436000D9F8A01606EBC4043B4689600C600962CC
:104370008963096556F83320954205D001330E2B29
:10438000F8D14F600F46C9E7084F07EB83174F601E
:104390000F46C3E7064A052006F082FEB6E700BFD7
:1043A000E0450C08B0EC0C08002F0024D8350024A0
:1043B000D8EC0C0830B40C4C0022234603E0013248
:1043C00014330E2A0CD093F804C08445F7D1DD686D
:1043D000294201D10029F2D1142303FB024000E05D
:1043E000002030BC704700BFB4030024F0B4446820
:1043F000A37913F0020266D002224FF0080C036882
:1044000064795B689D48204493F83C40012C90F807
:10441000380156D0012483F83C40022483F83D4003
:10442000142848D8DFE810F086004700470047000E
:10443000C1004700470047003601470047004700DA
:10444000F6004700470047001500470047004700B7
:10445000510018688A4E046AB04224F48034046221
:10446000046A456824F4003444EA0242446D24F0AE
:10447000700444F060040ED006F58066B0420AD0A5
:10448000804F06F58046B04218BFB84203D006F50B
:104490008066B04201D145F4803545604465816550
:1044A0000262426D42F008024265426D22F004024F
:1044B0004265426D42650121002283F83D1083F878
:1044C0003C20F0BC7047944699E718686C4E046A2B
:1044D000B04224F480140462046A456824F4001491
:1044E00044EA0252446D24F4E04444F4C0440ED043
:1044F00006F58066B0420AD0624F06F58046B042AB
:1045000018BFB84203D006F58066B04203D125F447
:10451000003545F4802545604465C1650262426D01
:1045200042F400624265426D22F480624265426D4F
:104530004265C0E71868544D046A514E24F00104E6
:10454000B0420462046A24F0020442EA04024468AD
:10455000876905EA070545F060050FD006F5806616
:10456000B0420BD006F57056B04207D006F5806613
:10457000B04203D006F58066B04207D122F00802AF
:1045800044F440744CEA020222F004024460856163
:1045900041630262826942F008028261826922F00C
:1045A000040282618269826185E71868374D046A76
:1045B000334E24F01004B0420462046A24F0200454
:1045C00044EA02124468876905EA070545F4C045D4
:1045D00000F0998006F58066B04200F09480294F83
:1045E0002B4EB04218BFB84203D006F58066B042E9
:1045F00001D144F440644460856181630262826950
:1046000042F400628261826922F48062826182697E
:10461000826150E718681A4E046AB04224F480544C
:104620000462046A456824F4005444EA0232C4690E
:1046300024F4E64444F4C0440ED006F58066B0424B
:104640000AD0104F06F58046B04218BFB84203D0DA
:1046500006F58066B04201D145F480454560C461ED
:1046600001640262C26942F40062C261C26922F45A
:104670008062C261C269C2611DE700BF18450C08B3
:1046800000000140004001408CFFFEFFFF8CFFFE58
:104690000044014018681F4D046AA84224F4807445
:1046A0000462046A466824F4007444EA0222C4697D
:1046B00024F0730444F060041ED005F58065A84220
:1046C0001AD0154F154DA84218BFB84203D005F5B2
:1046D0008065A84201D146F440564660C461C1637A
:1046E0000262C26942F00802C261C26922F0040299
:1046F000C261C269C261DEE622F4006242EA0C22B3
:1047000022F48062E7E722F0800242EA0C1222F0F3
:1047100040026EE7000001400040014000440140BB
:1047200042685379032B0FD8DFE803F00B0805022A
:1047300010684030704710683C307047106838305F
:10474000704710683430704700207047D0E900028D
:10475000064B517992790B44406893F8381153070E
:1047600001D575F075B975F095B900BF18450C08FD
:10477000F0B54468374A2469C368C4F303245B680E
:1047800052F82460EFF31184102585F312884568F0
:10479000314F95F805E0D0F80CC002EB4E02D5F889
:1047A00000E0158CDEF80C2005F4F05522EA050235
:1047B000CEF80C2017F806E0DCF8102053F80E5065
:1047C0001F2A25F0010543F80E5039D9203A20253B
:1047D000DCF804C005FA02F2CCF80C20E2B282F355
:1047E0001188BA5DDFF874C003EB020E46684569B4
:1047F000DEF8044004EA0C0C4CEA0101CEF8041087
:104800007179032924D8DFE801F018151202316804
:104810004031CEF80C500124CEF80810995841F0E0
:10482000100199509958214399500474F0BD316892
:104830003C31EEE731683831EBE731683431E8E795
:104840002025DCF804C005FA02F2CCF80820C5E700
:104850000021DEE718450C08F8460C080000FFFFB1
:1048600003681A7E012A2ED0002293F83010012905
:1048700009D093F8481001290ED093F8601001294F
:104880001BD02ABB7047022142F4806283F83010AB
:1048900093F84810012904D1022142F4006283F800
:1048A000481093F86010012907D01B6800211B688D
:1048B0005962D9680A43DA607047022142F4805293
:1048C00083F86010F1E702214FF400721976CCE70B
:1048D0004FF40072E9E700BF08B5204B98420ED0B4
:1048E00003F5806398420AD01D4A03F5804398423D
:1048F00018BF904203D003F5806398421BD1FDF7A7
:104900007FFC1849184BCA69C969C2F30222C1F376
:1049100002211A4492F8302002F01F02D040114ABE
:104920001269C2F3C03241EAC202134493F83C3127
:1049300003FB00F008BDFDF763FC0A490A4BCA6996
:10494000C969C2F3021CC1F3021103EB0C0292F815
:10495000302002F01F02D040E1E700BF000001401C
:10496000004001400044025818450C0870B50E463E
:1049700005EE102AD0E90031013E1A680868B6B287
:104980005C681568FFF7A8FF07EE900AB8EE455A75
:104990009FED527AF8EE677A87EE850A30EE070AC5
:1049A00079F080FE23680138AB4280B252D0C4E96E
:1049B000005000238022E660A360A261C4E90433B2
:1049C00094F83D3003F0FF02002B62D00223211D3A
:1049D000284684F83D30FCF78FF9414B0122B5F1B0
:1049E000804FA5EB030384F83D20B3FA83F34FEA2D
:1049F000531334D09BBB3B4A95420CD002F58062E6
:104A0000954208D002F58062954245D002F5784281
:104A1000954241D070BD94F83C30012BFAD002226F
:104A2000314B012184F83D20A8680340AB6084F835
:104A30003D1084F83D206A68A96822F0700221F0D8
:104A40008001012000236A60A96084F83D0084F899
:104A50003C3070BD636883423AD06060A9E794F847
:104A60003C20012AD6D002211F4A002084F83D10A4
:104A7000A9680A400121AA6084F83D10022284F846
:104A80003D206A68A9680BB90028D6D022F47002CC
:104A9000D3E784F83C2099E794F83C20012AB9D068
:104AA0000221114A114884F83D10A968281A0A40C9
:104AB000B0FA80F00121AA600022400984F83D107C
:104AC00084F83C200A4A9542D8D00028D6D170BD3F
:104AD000E368B3427FF46DAF70BD00BF0AD7233CDB
:104AE00000000140000400408800CEFF00040140A7
:104AF000000C0040024B0348D3F8A016FCF794BF0B
:104B0000002F002400000140034B4FF08040D3F8F9
:104B1000A416FCF789BF00BF002F0024024B0348F6
:104B2000D3F8A816FCF780BF002F00240004004033
:104B3000024B0348D3F8AC16FCF776BF002F0024D5
:104B400000080040024B0348D3F8B016FCF76CBFD6
:104B5000002F0024000C0040024B0348D3F8BC1681
:104B6000FCF762BF002F002400040140024B034801
:104B7000D3F8CC16FCF758BF002F002400180040D3
:104B8000024B0348D3F8D816FCF74EBF002F002481
:104B900000400140024B0348D3F8DC16FCF744BF49
:104BA000002F002400440140024B0348D3F8E016D4
:104BB000FCF73ABF002F00240048014010B5064C16
:104BC0000648D4F8BC16FCF72FFFD4F8D0160448DA
:104BD000BDE81040FCF728BF002F0024000401406E
:104BE000001C004010B5064C0648D4F8BC16FCF773
:104BF0001BFFD4F8D4160448BDE81040FCF714BFDE
:104C0000002F00240004014000200040BFF34F8F1C
:104C10000549064BCA6802F4E0621343CB60BFF358
:104C20004F8F00BFFDE700BF00ED00E00400FA0574
:104C30000021012008B50CF0CBF972B6FFF7E6FFB2
:104C40002DE9F043BFB0BFF35F8F8A4C0021626A49
:104C50000B460D4622F4803262620A46C4F8941074
:104C6000C4F898300133C4F89C20112BC4F8A0205C
:104C7000F6D10523C4F89430636A43F48033636249
:104C8000BFF34F8FBFF36F8F7B487C4A7C49121A6A
:104C90007CF09EF9D4F888207A4B012142F470020E
:104CA000C4F8882019601D611A6842F080021A60F9
:104CB0001A680A431A601A6842F480321A601A6845
:104CC00042F480521A609D61DD611D629D62DD6269
:104CD0001D635D639D63DD631D645D641A6822F47A
:104CE00080221A601D664FF00063674AC2F80811FF
:104CF000A36075F017FE654AD36813F0040FD368FC
:104D000040F0A380624B0021604A0591D96A21F0EE
:104D10000101D962DB6A03F001030593936943F44F
:104D200040439361936903F440430593059B936962
:104D30009E04FCD54C2200210EA8564C7EF0C6F9EC
:104D4000554A42F20303A4F110011268B3EB124F6B
:104D50004FF000024FF0040308BF0C460892E268CF
:104D6000A370002A4CD1494A494B916941F4404112
:104D70009161926902F440420892DA6A42F00102BB
:104D8000DA62DB6A03F001030893089B3F4A9369E8
:104D90009D04FCD53B4B4FF4403540480321D3F8EC
:104DA000E02042F08002C3F8E0200122D3F8E03096
:104DB00003F080030793079B85610D9BCDE90013EA
:104DC000002375F06BFC022301204FF48031A28890
:104DD000CDE9173304231993A379CDE90E01E079C6
:104DE000217A1C900EA81D91CDE91A2308220023D8
:104DF000CDE91E23FBF78AFC032838D0A0B1FEE7DB
:104E0000234BD96A21F00101D962DB6A1F4903F003
:104E1000010308938B6923F4404313438B618B692F
:104E200003F440430893B0E71D4B1A6812F00E0FCD
:104E30003AD11A6822F00F0242F002021A601B688F
:104E400003F00F03022B2FD0FEE723F00703154CCE
:104E500043F00203D360216805E023685B1AB3F5D1
:104E60007A7F3FF64FAF53689F04F6D54AE7FFF7C6
:104E7000DFFE00BF00ED00E000000000C8350000CC
:104E8000B06A0D08004402580080005100480258E2
:104E900000040058DC0400240010005C001C0258D0
:104EA00000200052002F00246C4A936903F0700325
:104EB0003F2B05D8936923F0700343F040039361BF
:104EC000664AD36903F070033F2B05D8D36923F0FA
:104ED000700343F04003D361604AD36903F4E06395
:104EE000B3F5806F05D2D36923F4E06343F48063A4
:104EF000D3615A4A136A03F070033F2B05D8136A33
:104F000023F0700343F040031362544B9A69100777
:104F100005D49A6922F00F0242F008029A614F4AC2
:104F2000936923F470639361136899018CD51369B5
:104F300041F288314A4C23F0070343F00303136125
:104F4000206804E023681B1A8B4200F299811369E0
:104F500003F03803182BF5D1936903F00F03082BE6
:104F600005D9936923F00F0343F0080393613D4A89
:104F7000136803F00F03022B0BD9136823F00F0300
:104F800043F002031360136803F00F03022B00D0F9
:104F90005AE7324A936903F07003402B05D99369AD
:104FA00023F0700343F0400393612C4AD36903F06C
:104FB0007003402B05D9D36923F0700343F04003FD
:104FC000D361264AD36903F4E063B3F5806F05D952
:104FD000D36923F4E06343F48063D3611F4A136A07
:104FE00003F07003402B00F243811C4EFDF7E6F8FE
:104FF0001D4BB2691D4DC2F30322134493F83030A8
:1050000003F01F0320FA03F3D5F82C012B60FDF702
:105010001DF8002840F035811023159017900EA838
:105020000E93FBF773FB002840F021813368104A90
:1050300043F080033360D6F8F43043F00203C6F83F
:10504000F430D6F8F43003F002030493049B136A9F
:1050500043F001031362074B216810E0004402583B
:10506000002F00240020005218450C0800000024E6
:105070000004005880380100013B3FF4F8AE22687C
:105080009142F9D0226823689B1A0A2BFBD9A04CC5
:105090004FF480224FF440130EA80E924FF00008F8
:1050A0002F9374F03BFDD4F8EC3041F203029949A0
:1050B000032643F002030EA80227C4F8EC30D4F80C
:1050C000EC3003F002030393039BD4F8943043F0D5
:1050D0000203C4F89430D4F8943023F00203C4F8E7
:1050E00094300B688C49B2EB134F8C4B8C4A28BF21
:1050F0000A465A601A6822F47C5242F400521A603E
:105100001A6842F060021A600E96CDE92B8874F09E
:1051100005FD4FF4E0430EA8CDF8E4800E93CDE9F1
:10512000258874F0FBFC18230EA8CDF8B8800E93E8
:10513000CDF8CC8074F0F2FC4FF4803305220EA839
:1051400012960E9321934FF4FA73CDF8588011976D
:10515000CDE90F230423CDE91488139374F0DEFC0A
:10516000D4F8E0303A464FF480716E4843F00103C2
:10517000C4F8E030D4F8E03003F001030993099B50
:105180004346CDE9006875F089FA23693A466648D6
:1051900023F0FE7343F088732361D4F8E03043F0CA
:1051A0000403C4F8E030D4F8E03003F004030693BD
:1051B000434606994FF40071CDE9006875F06EFA28
:1051C000236923F07E4343F0FC432361FCF7F6FFA1
:1051D0002860BFF35F8F554D4646554C01276B6ADB
:1051E00023F480336B62C5F8948023E0002946D015
:1051F000D4F80090637A103414F8060C1B0643EAC6
:10520000007343EA410314F8051C43EA814314F890
:10521000041C43EA414314F8031CC5F898600136A6
:1052200043EA0143C5F89C90032E43F00103C5F8FF
:10523000A03027D06368217A002BD7D0D4F8009013
:105240000029D7D129F01F01A3EB0108B8F1200FE5
:1052500038BF4FF0200840467CF09CF8411E0346C2
:1052600007FA01F0804508BF1946C9B2C2E7FEE758
:10527000136A23F0700343F040031362B5E6FEE7C0
:10528000E2E5E1E50523C5F894306B6A43F4803329
:105290006B62BFF34F8FBFF36F8FBFF34F8FBFF3BF
:1052A0006F8F0022C5F85022BFF34F8FBFF36F8F6F
:1052B0006B6943F400336B61BFF34F8FBFF36F8FA4
:1052C000C5F88420BFF34F8FD5F8805043F6E076C1
:1052D0001649C5F34E34C5F3C905640104EA060056
:1052E0002B4640EA8372013BC1F86022F9D2203C90
:1052F00014F1200FF2D1BFF34F8F4B6943F4803389
:105300004B61BFF34F8FBFF36F8F3FB0BDE8F083AA
:10531000004402580010005C7FBB22000084004063
:105320007FBB2230000002580008025800ED00E068
:10533000EC0400243F4B586D012830B585B06ED089
:105340003D494FF6FF003D4ACC683D4B04403D4D82
:105350003D482243CA605A6FC5F8582AD3F8F42052
:1053600042F00202C3F8F420D3F8F42002F0020263
:105370000392039AD3F8DC2042F00052C3F8DC20F9
:10538000D3F8DC2002F000520292029AD3F8DC201B
:1053900042F08042C3F8DC20D3F8DC2002F08042E7
:1053A0000192019AD3F8DC2042F00042C3F8DC20DD
:1053B000D3F8DC20036802F0004224480092009AEF
:1053C000D1F8FC40224A44F08074C1F8FC40A2FBB2
:1053D00003420024920CC5F85C2A1E4AC0F8B02F84
:1053E0001D4A4460A2FB032302689B0942F00102AC
:1053F000013B0260B3F1807F07D34FF0E0221369D5
:1054000043F00403136105B030BD4FF0E022F020FB
:105410005361072381F8230094611361EDE70021B4
:105420000BF0D6FD0D4B1A6882F308885B6898472D
:10543000FEE700BF0040005800ED00E00003FA0561
:1054400000440258002F002400000024001000E057
:1054500083DE1B4355CEACC5D34D62100098F01FC0
:105460002DE9F843384E984606EB8003D3F84C41BB
:10547000002C66D004F1CA0306F5B6760546B4F8EA
:10548000CA02A36104F5E57366601746E3614FF451
:105490008073261DE160C4E904332368C4F8C43076
:1054A000A36300284AD194F8C90009F03DFC18F024
:1054B000080F94F8C89034D1BA0723D4FB0711D44D
:1054C000052194F8CE0270F01DFB94F8CE32012233
:1054D0001E4903F01F005B09824041F8232030463B
:1054E000BDE8F8830135484609F01EFCEDB218B15D
:1054F00040F206630572C38094F8CC22022109F0C1
:10550000F1FBDDE76B1CDBB218B1037240F206530E
:10551000C38094F8CD22022109F0E4FBFB07CFD52C
:10552000E0E70135EDB218B140F206730572C380B1
:1055300094F8CD22022109F0D5FBC1E76FF026FED9
:10554000B1E72646CBE700BF18450C0800E100E0B4
:105550000148FBF71FBD00BF200500240148FBF7F1
:1055600019BD00BFF00700240148FBF713BD00BFC1
:10557000C00A00240148FBF70DBD00BF900D0024B8
:105580000148FBF707BD00BF601000240148FBF78E
:1055900001BD00BF301300240148FBF7FBBC00BF76
:1055A0000016002470B52422456B00238168C0F8E2
:1055B000B42004462A6800F1340622F001022A6071
:1055C0002B606B60AB608279C0F8BC3080F8B03083
:1055D000C0F8B430C364C0F8B83043659302816347
:1055E00003F480534179C363130303F4005303644A
:1055F000130203F48063436401F00203C90745D436
:10560000002B7BD1836412F00802D4F8B43059D057
:10561000002B7FD024233046C4F8B4302B6823F00D
:1056200001032B60FCF760FF012815D0E36D002B10
:1056300077D16B68304623F490436B60AB6823F0FE
:105640002203AB60AB6843F00803AB602B6843F008
:1056500001032B6074F0D0F96279D5070DD5D4F829
:10566000C030196841F480711960996841F00101F6
:105670009960196841F020011960900705D5D4F8A8
:10568000C020136843F08003136070BD042181645F
:1056900053B10C23D1078364B5D5E36D4FF480314A
:1056A00043F0020361662EE0D307ACD5C36D12F060
:1056B000080243F00203C3654FF480334366D4F815
:1056C000B430A5D10BB194F8B020242384F8B020D5
:1056D0003046C4F8B4302B6823F001032B60FCF78C
:1056E00003FF0128B8D0E36DBBB96B68304623F4E3
:1056F00090436B60AB6823F02A03A6E7082383641A
:10570000D30780D5E36D43F00103E3654FF4003325
:10571000236678E784F8B0307CE73046FBF760FB1F
:10572000E3E73046FBF75CFB83E700BF816039E7C6
:10573000417137E7817135E72DE9F843434D3C204E
:10574000434C05F5D072B5F8A631C4F8602AA4F828
:105750006C3AB5F8AA21B5F8AE31A4F86E2AA4F8CF
:10576000643A09F0E1FA0746422009F0DDFA0646FC
:10577000382009F0D9FA81461FB10D23FB800023A0
:105780003B721EB10D23F38000233372B9F1000F79
:1057900005D00D23A9F80630002389F80830B5F8A4
:1057A000B2313920A4F8663AB5F8B631A4F8683AAF
:1057B000B5F8BA31A4F86A3A09F0B6FA80463A2048
:1057C00009F0B2FA05463B2009F0AEFA0446B8F1FA
:1057D000000F05D00D23A8F80630002388F8083004
:1057E0001DB10D23EB8000232B721CB10D23E38030
:1057F00000232372484607F077FF0121484609F04D
:105800004FFA404607F070FF284607F06DFF20462C
:1058100007F06AFF4046012109F042FA28460121BB
:1058200009F03EFA0121204609F03AFA384607F01D
:105830005BFF304607F058FF3846012109F030FA87
:1058400030460121BDE8F84309F02ABA18450C0892
:10585000002F00242DE9F04F9A4D7C2299B00021B1
:1058600005F214507DF032FC4FF48032D5F8606AB6
:1058700095F844353468C5F818254FF40032C5F85A
:105880001445C5F824250222C5F82825002B00F070
:10589000A08003218C4B8D4A85F8441561680B402C
:1058A00043F0FA036360236843F003032360D36C7F
:1058B000DE0340F11F8108A8FCF7E2FC0A9B4FF4CD
:1058C000FA70B3F5FA7FB3FBF0F0C0F06881804A5C
:1058D0002968B2FBF0F202322B685B1A9A42FBD8BD
:1058E00000227C4B7C490292A260E2680E68134061
:1058F0007A4AA2FB062641F2883243F48053760AA4
:10590000E36002FB06F63346002B00F0A381626BD6
:10591000013B1106F8D5724A4FF4D573A263A36018
:105920006C4AE3681A4041F208131343E3604EB136
:105930003346626B12F0450F02D0920440F10883A7
:10594000013BF6D10023634AC5F85035A360E368F4
:105950001A40334642F48052E260002B00F07A8114
:10596000626B013B1106F8D55D4BA363029A4FF6BB
:10597000FE739A4200F2A281DFF85891594FDFF886
:105980006081002337212046A36041F23713E2688B
:1059900002EA0902134341F28832E360FDF7CCFAD0
:1059A000002840F05981A76041F22913E26802EA19
:1059B00009021343E3604EB13346626B12F0450FA8
:1059C00002D0920440F1F180013BF6D14FF08050BB
:1059D00042E1454B9C4259D0444B9C4200F04881E7
:1059E00095F86C0A09F0A0F9834695F86E0A09F05B
:1059F0009BF9824695F8640A09F096F9814695F874
:105A0000660A09F091F9804695F8680A09F08CF960
:105A1000074695F86A0A09F087F995F86D2A044651
:105A20000E21584609F05EF9504695F86F2A0E216E
:105A300009F058F9484695F8652A0E2109F052F9FF
:105A4000404695F8672A0E2109F04CF995F8692A25
:105A500038460E2109F046F90E2195F86B2A2046AA
:105A600009F040F90221B6F9040070F04BF8B6F9DC
:105A70000430002B07DB03F01F0001225B091C49E7
:105A8000824041F82320D5F8144502E70F4BD3F8A4
:105A9000D42022F48032C3F8D420D3F8D42042F4A6
:105AA0008032C3F8D420D3F8D42002F4803201929B
:105AB000019ADA6F42F48032DA67DA6F22F48032C8
:105AC000DA678DE7002F0024002CC0FF0044025845
:105AD00010210100C0E0FEFF00000024D34D621041
:105AE000C5002000000010C10070005200240248D0
:105AF00000E100E0906A916AD76A11F47C7F536BF1
:105B0000C1F305164BD0C3F3CC0307F0010700F037
:105B1000030007EE906A07FB03F30128F8EEE76A3B
:105B200007EE103ABAEEE97A00F0F282022800F0AD
:105B30006983002840F0EC821368980640F16B837B
:105B40001168B7EE006A136BC1F3C102C3F3080317
:105B500007EE903A564BF8EEE77AD34037EE877A65
:105B600007EE903A37EE067AB8EEE76AC6EE267A86
:105B700067EE877A4F4AF7EE006A136B136B126B6E
:105B8000C3F3064307EE103AB8EEC77A37EE267A2B
:105B9000C7EE876AFCEEE67A17EE903A8FE62A683F
:105BA0002B689B1A022BFBD99AE6636B5B0700F10B
:105BB000CC81C4F838806269029B002A03F101039A
:105BC0000293029B04DB4FF6FE718B427FF6D9AE47
:105BD00002994FF6FE73994200F2D182570071D5B7
:105BE000236801279807C5F84C7500F0D78100237A
:105BF000DFF8C4802046A36041F20233E26802EA83
:105C000008021343E360FBF74BF928BB636904F117
:105C1000180A04F11C09C5F88035A369C5F8843554
:105C2000E369C5F88835236AC5F88C3541F203135A
:105C3000A060E26802EA080204F120081343E3606E
:105C400046B1636B13F0450F02D09A0440F19A827B
:105C5000013EF6D14FF00040012385F84435D5F8D8
:105C600048350343C5F84835012019B0BDE8F08F29
:105C7000104BD3F8DC2022F40072C3F8DC20D3F8F8
:105C8000DC2042F40072C3F8DC20D3F8DC2002F4FC
:105C900000720092009AD3F8842042F40072C3F894
:105CA0008420D3F8842022F40072C3F8842097E67D
:105CB0000090D00300440258C0E0FEFF029A9A42CE
:105CC00000F25D822368990700F06881D5F84C7571
:105CD000032F8CD1D5F87025D5F87435A169090D3D
:105CE000C5F85415910F8DF82010C2F383618DF81B
:105CF0002110C2F301618DF82210C2F307418DF823
:105D00002310C2F30721D2B28DF824108DF825207C
:105D10001A0DADF82620C3F303428DF82820C3F3F3
:105D2000C0328DF82920C3F380328DF82A20C3F3C6
:105D300040328DF82B20C3F300328DF82C20002246
:105D40008DF82D20002F40F0F78140F6FC71D5F83A
:105D5000782501EA830343EA92730C93C2F3C2638A
:105D60008DF83430C2F302638DF83530C2F34253FC
:105D70008DF83630C2F382438DF83730C2F3C23328
:105D80008DF838300C999DF8383001319DF8280095
:105D900003F0070300F00F00023399400123834012
:105DA000C5F85C15C5F860355B0A01FB03F3C5F85F
:105DB00064354FF40073DFF8709407212046C5F86E
:105DC0006835C2F380338DF83930C2F3C61302F060
:105DD0007F028DF83A308DF83B20D5F87C35D5F828
:105DE00058254FEA024ADA0F8DF83C20C3F341727E
:105DF0008DF83D20C3F382628DF83E20C3F38352B9
:105E00008DF83F20C3F340528DF8402000228DF8DA
:105E10004120C3F300428DF84220C3F3C0328DF815
:105E20004320C3F380328DF84420C3F340328DF811
:105E30004520C3F300328DF84620C3F381228DF84C
:105E40004720C3F30122C3F346038DF848208DF8A1
:105E5000493001238DF84A3041F20713C4F808A0F5
:105E6000E26802EA0902134341F28832E360FDF777
:105E700063F800287FF4F0AE2E686369990161D45D
:105E80004FF0400841F2101310212046C4F808805A
:105E9000E26802EA0902134341F28832E360FDF747
:105EA0004BF800283FD1C4F808A041F23713E2684C
:105EB0003721204602EA0902134341F28832E360A7
:105EC000FDF73AF878BB4FF0FF330D216362C4F859
:105ED0002880E36A23F0FF0343F06303E36241F2A7
:105EE0000D13A0602046E26802EA0902134341F262
:105EF0008832E360FDF720F8A8B908AB03E02A6810
:105F0000921B013247D0626B12F4957F626B48D1CD
:105F10001204F4D503F12001D4F8802043F8042BB7
:105F20009942F9D1EBE7D5F84835C5F84835BD4B6E
:105F30000122A363D5F848350343C5F8483585F8F1
:105F4000442591E64FF40060F1E70423A3633DE5A7
:105F5000636B5B0700F15981636BDF0700F14E81D2
:105F6000636B580601D54023A36301220023372128
:105F70002046C5F85025A360AB4AE3681A4041F2B9
:105F80003713134341F28832E360FCF7D5FF002852
:105F90003FF4ECAC1AE54FF00040C8E74FF08060EA
:105FA0005AE6100700F13581626B910700F13681E6
:105FB000626B920608D533E1D4F8802043F8042BB5
:105FC0002A68921B0132E6D0616B11F48051F3D143
:105FD000964B012FA363089BC3F381128DF80C200D
:105FE000C3F340128DF80D204FEA132222F0FF0276
:105FF00042EA1362DDE9090392B200BAADF80E205D
:10600000DAB204908DF81420C3F307229DF8330010
:106010008DF81520C3F303524FEA13438DF8162071
:106020000B9A23F0FF03D4B243EA0403ADF818300F
:10603000C2F385238DF81A30C2F301238DF81B308B
:10604000C2F3031302F00F028DF81C308DF81D20EF
:106050008DF81E009DF81C309DF81D20DBB2D2B2D9
:1060600005D1134314BF4FF400714FF48071D5F87C
:106070002005C5F86C156FF0ADFB00287FF4F4AD7A
:106080002C6803E02B681B1B013330D06FF080FBC2
:106090000428F7D100230121D5F85C25C5F848353F
:1060A000C5F8403585F84415002A3FF4DDAD4FF4BE
:1060B00080406FF08FFB00287FF4D6ADD5F84C35CB
:1060C000EBB1012B7FF4D0AD0220594C85F888004C
:1060D00004F26C530FCB84E80F0004F27C531034AD
:1060E0000FCB84E80F00002019B0BDE8F08F4FF00F
:1060F00000420123C5F8482585F84435B4E5D5F8B4
:106100005035002BE1D0012B7FF4AEAD1846DCE713
:10611000DFED487A87EEA66A136BC3F3080307EE38
:10612000903AF7EE005AF8EEE77A77EE877A77EE54
:10613000A57A67EE867A1DE5012F13D11B04D5F8E9
:10614000782503F47C1343EA12430C930C9B013330
:106150009B02C5F85C35C5F864354FF40073C5F88B
:10616000603526E62F4B4FF080500122A363D5F80F
:1061700048350343C5F8483585F844256CE54FF0AC
:10618000807069E5636B5B0760D4636BDE0759D48D
:106190002369DBB2032B57D1274BA363636913F445
:1061A000604F09D05C0455D413F4004F14BF4FF472
:1061B00080504FF480304FE51B0C1B4A2046C5F839
:1061C00058351B04A360E3681A4041F209331343B6
:1061D000E360FAF765FE00287FF43EAD6269C5F81A
:1061E0007025DAF80030C5F87435D9F80010C5F814
:1061F0007815D8F80010C5F87C156FE50123A36366
:10620000FFF7A0BBDFED0D7A84E70423A363FFF75C
:1062100099BB08208BE6DFED0A7A7BE7022086E651
:10622000202084E6FF0FE01FC0E0FEFF3A0F0018B9
:10623000042F00240024744AC50020000024F44ADE
:106240000024744C0123A363012005E504231846B0
:10625000A36301E54FF40050FEE400BF10B5104CFD
:10626000D4F8C43323B119689A880B691A420AD04A
:10627000FFF7F0FA38B994F88C330133DBB2072B0F
:1062800084F88C3303D9002384F8983310BDD4F8F4
:106290000C240123C4F8882384F8983310BD00BF70
:1062A000002F002470B58B4C94F898536B1E082B6C
:1062B0001DD8DFE803F0786A7C1C4E05351C2600EB
:1062C000A36A002B6DD10722D4F80C34D4F8805384
:1062D00084F89823C4F88833002D62D0D4F884332E
:1062E0000120D4E9DD21A84794F898536B1EDBB256
:1062F000022B4ED9042D18BF082D0CBF0120002001
:1063000070BDFCF7BBFE002840F0D880D4F888337D
:10631000D4F80C24FA339342ECD2FFF79FFFC3E783
:10632000FCF7ACFE0028F1D0D4F894330022012B06
:1063300084F88C2340F2C680D4F89023013B0821D6
:106340000132C4F8943384F89813C4F890230120E0
:1063500070BD666A002E71D1FCF790FE002875D0E2
:106360000423D4F8805384F88C6384F89833002D88
:10637000EDD0D4F884333046D4F87423D4F87813AD
:10638000A84794F898536B1EB1E76FF001FA042800
:106390006BD0D4F80C34D4F888239B1AC82B00F2A5
:1063A0008280002070BD022384F898337CE7FAF7DE
:1063B00077FF0028EDD194F85C500422B4F85E1009
:1063C000236EC4F894031B0E206EA4F8A01384F867
:1063D0009823000C216E84F8A333226E090A94F8E6
:1063E000643084F8A62384F8A73394F8653084F8E1
:1063F000A4031B0994F8652084F8A513A06E02F08D
:106400000F02B4F86E1084F8AC33B4F86E3084F830
:10641000AD23C3F30B13B4F86E2084F8A25343EA00
:10642000112302F00F02C4F8A80303F00F0384F84D
:10643000B02303F5FA63A4F8AE3335E7D4F8883314
:10644000D4F80C2464339342BFF454AFFFF706FF33
:10645000D4F88053002D3FF427AF0022D4F88433C2
:10646000D4F878131046A8471EE7FAF719FF00285A
:106470008FD194F88830002BA3F10203B3FA83F391
:1064800008BF01255B0984F88D5384F88E33FAF731
:1064900007FF00287FF441AFA26F0323C4F89C23B9
:1064A00084F8983300E7FFF7D9FE94F8980304289E
:1064B00018BF08280CBF0120002070BD042384F8F9
:1064C000983344E7FAD1FCF705FE94F898536B1E15
:1064D0000DE700BF002F00242DE9F04706460D46CA
:1064E00090461F465F4C94F8981304290BD0082956
:1064F00007D1D4F89033B34205D0FCF7EBFD022866
:10650000F1D001209FE00123C4F88083C4F8847394
:1065100084F87C33A362062384F89833EB06C4E93D
:10652000DD564CD1BFF34F8F4F4A05F500712B4616
:10653000C2F8683220338B42FAD1BFF34F8FBFF3DA
:106540006F8F002D50D094F84435012B37D1731C38
:10655000D4F8641500228B42C4F848253DD80323A3
:10656000D4F814754FF4007AC4F8305584F84435E3
:106570004FF40073FA621021C4F834353846D4F869
:106580004C35C7F808A0FA68012BDFF8E49041F217
:10659000101318BF760202EA0902134341F288324F
:1065A000FB60FCF7C9FC804628B3304B0122BB637B
:1065B000D4F848350343C4F8483584F84425FFF738
:1065C0004DFED4F8805335B1D4F884330022D4F88A
:1065D00078130120A847032035E0D4F8483543F06C
:1065E0000073C4F84835EAE7D4F8483543F000634F
:1065F000C4F84835E3E74FF0FF33182138467B6293
:10660000C7F828A0FB6A23F0FF0343F09003FB6266
:10661000FB6843F04003FB609023BD6501253D65A9
:10662000C4F8403541F21813BE60FA6802EA090264
:10663000134341F28832FB60FCF77EFC28B9FB6B08
:1066400043F48D73FB63BDE8F087084BBB63D4F85C
:1066500048350343C4F8483584F84455C4F84085A8
:10666000ADE700BF002F002400ED00E0FF0FE01FAA
:10667000C0E0FEFF2DE9F04F674C1F4683B0064691
:1066800094F898330D469046042B09D0082B03D07C
:10669000002003B0BDE8F08FFCF71CFD0228F7D105
:1066A00015F01F0147D101225C4BC4F8705A626299
:1066B0009A604FF400725A60002D4AD094F8443525
:1066C000012B38D1701CD4F86435C4F848159842B1
:1066D00048D80323D4F814A5C4F83C2584F84435DD
:1066E000D4F84C35C4F83855012BCAF82C1037D0E3
:1066F000730201934FF40079494B41F21012504656
:10670000CAF80890DAF80C1019400A431021CAF8A8
:106710000C2041F28832FCF70FFC414B834640B31A
:10672000404B0122CAF83830D4F848350343C4F846
:10673000483584F84425FFF791FDD4F88053002DA7
:10674000A6D00022D4F88433D4F878131046A84792
:106750009EE7D4F8483543F00063C4F84835EAE7CB
:106760000196C7E7D4F8483543F00073C4F84835BC
:10677000E1E74FF0FF3211215046CAF82420CAF851
:1067800028904FF00109DAF82C2022F0FF0242F0A5
:106790009202CAF82C20DAF80C2042F04002CAF823
:1067A0000C208122CAF85850CAF85090C4F84025ED
:1067B000019ACAF80820DAF80C201A4041F21113A5
:1067C000134341F28832CAF80C30FCF7B5FB60B1D4
:1067D000144BCAF83830D4F848350343C4F8483568
:1067E00084F84495C4F840B5A5E705234846C4F8A5
:1067F000808384F89833DAF83C30C4F8847343F427
:106800009573CAF83C30D4F80C34C4E9DD56C4F8AA
:10681000883303B0BDE8F08F002F002470390024C6
:10682000C0E0FEFFFF0FE01F6EF00EBE6EF00CBE6C
:1068300010B51C2008F078FA0446112108F030FA4F
:106840001CB1A38822681B049361C8200CF01EF8B9
:106850002046BDE8104006F047BF00BF2DE9F04FCD
:10686000DFF8109587B0D9F87C4A636913F0010B03
:1068700002D007B0BDE8F08F6269A3691A42F8D070
:106880006369A26913409D0703D5636903F002039E
:1068900063616369A26900941340D80614D5A369A3
:1068A00023F01003A361236A03F4F01203F00F0531
:1068B000B2F5802F00F09C84B2F5402F00F08E825C
:1068C000A36943F01003A3616369A269134019032C
:1068D0007CD46369A26913405F0300F1B5806269EB
:1068E000A3691A4256D46369A26913401E0509D5EB
:1068F000009BD3F80838DD0700F1B184636903F425
:10690000006363616369A2691340180110D563696C
:1069100003F00063636199F8703E002B40F03C8205
:10692000012389F8703E636DC3F38303C9F8743E95
:106930006369A2691340D90400F1B2816369A26955
:1069400013409B0400F14B816369A26913401E0749
:1069500000F117826369A2691340DD0200F10C8225
:106960006369A2691340980200F1F9816369A26921
:106970001340590000F1EE816369A26913405A0780
:106980007FF577AF65686B0700F15B8463681D4333
:1069900065606EE7009B03F50062D3F8043823F0CE
:1069A0000103536099F8703E012B00F00A82D9F878
:1069B000803E93F89C22042A03D193F89D2283F809
:1069C0009C22636903F0004363618CE7D4F8185894
:1069D000D4F81C381D402D0C3FF47BAF04F5306714
:1069E000DFF884834FF0000A2046CDF804B008E0B9
:1069F0006D080AF1010A07F1200708F11C0800F0F0
:106A0000038215F0010BF3D000F530614FEA4A1410
:106A100001EB4A139E68D0F814281640F20700F1E3
:106A2000B483310700F1F481F10601D51023BB6076
:106A3000B20601D52023BB60B30402D54FF4005346
:106A4000BB60D9F87C0AD3E7D4F81878D4F81C389E
:106A50001F40BFB2002F3FF442AF009B4FF0000831
:106A6000CDF808B0A346C04D03F5106A444609E0CE
:106A700004F1010C7F08644605F11C050AF1200AA7
:106A800000F0A183FE07F3D5DBF8103804F00F0205
:106A9000DBF83468E1B2D640F601F6B21E430BF5DE
:106AA000106303EB44139B681E406301F0070193DE
:106AB00027D50120009BD9F8808E00FA02F2D3F886
:106AC000343823EA0203009AC2F83438CAF80800BE
:106AD000D9F88C0AAB6C012800F0CC83002C40F074
:106AE0007783D8F89422022A00F0DE8432F004037F
:106AF00000F02F8598F8A032012B02D1002388F8EE
:106B0000A032330702D50823CAF80830F00602D5B0
:106B10001023CAF80830710602D54023CAF808309D
:106B2000B20702D50223CAF808303306A0D5D5E94A
:106B300014E070459CD86301AEEB000204F1010C37
:106B400003F510686B6CD844934228BF1346D8F8FD
:106B50001820033392B2B2EB930F32D373460BEB90
:106B60000C36A646CDF804B01C46844240F2EC83B5
:106B7000221A6B6C99F88C1A9A4228BF1A46AB6C91
:106B800002F1030B4FEA9B0B69B991B203318908FB
:106B900009D003EB810153F8040B8B423060FAD12A
:106BA000AB6CD5E9144013441044AB64D8F81830EA
:106BB00068659BB29B45D8D92346DDF804B074467E
:106BC0009E4686453FF656AF04F00F040122DBF8DF
:106BD0003438A24023EA0203CBF834384AE7D4F829
:106BE00000296FF30A02C4F80029D4F8042842F4FB
:106BF0008072C4F80428D4F808389F0700F1028195
:106C000013F0060318BF0F23C9F8883AFBF7F8FA08
:106C1000D9F8886AF3B2022B00F040834FF4105386
:106C2000E268003ED9F8805E4FF0400722F47052CF
:106C300018BF0126D5F8D002E260E26813430022B3
:106C4000E36001241146402372F0B4FB3B4600226E
:106C50008021D5F8D002C5F86471C5F8584172F0AA
:106C6000A9FB0023AC61C5F894326B60C5F8A4326F
:106C7000D5F8C8326F6285F89C42002B00F059832A
:106C8000D5F8B432002128465B689847D9F8803E91
:106C9000D9F87C4A1E74636903F40053636153E6B8
:106CA000009B03F50060436823F0010343604FF449
:106CB000846323612D4B013B02D022699206FAD4F2
:106CC000D9F8805A1DB3009B4FF67F3103F510634E
:106CD00099600BF1010B1A682033AB4522F40012C6
:106CE00043F8202C53F8202C42F0006243F8202C6B
:106CF000C3F8E811D3F8E02122F40012C3F8E02130
:106D0000D3F8E02142F00062C3F8E021E0D1C3698A
:106D100043F00113C361D9F8AC3A002B46D1426964
:106D200042F22B0313434361036943F00B030361F6
:106D3000009920460E4AD1F8003823F4FE63C1F8CA
:106D4000003899F88C1A72F0B5FB636903F480532C
:106D50006361F3E5636903F0804363610CE6636993
:106D600003F40013636101E67C390024410D030044
:106D7000403D0024002F0024636903F48013636105
:106D8000EEE5D9F8800E90F89C32032B1DD0636994
:106D900003F008036361DDE5D9F8803E042193F830
:106DA0009C2283F89C1283F89D22C1E5D0F88430A0
:106DB00043F00B03C0F88430436C43F00B0343648F
:106DC000B6E7002389F8703EFBE5D0F8B432DB6902
:106DD000002BDCD09847D9F87C4AD8E7C5EBC50230
:106DE00004F58051C3F30A1309EB8202D2F8900C28
:106DF00003440868C9F8400E0968C2F8903CC9F815
:106E0000441E5DE50223FFE60446DDF804B060E5BC
:106E1000D9F87C2A0823BB6002F53063126C234446
:106E200010460292B84A9968904204D90A0402D5E1
:106E30004FF400429A60D9F8804E99F8403E04F52C
:106E40002A7184F8A83299F841EE84F8A9E2B9F8D9
:106E5000422EA4F8AA2203920122B9F844CEA4F843
:106E6000ACC2B9F8460EC4F8942203F01F02A4F88D
:106E7000AE02012AC4F8980200F06A82022A00F0E9
:106E80009182002A40F0878203F06003202B00F0FB
:106E90005A83402B00F05783002B40F08A83BEF1C9
:106EA000090F14D8DFE80EF0CD9F13C3138C7213B3
:106EB0004C2DBBF1000F00F02F850323012184F836
:106EC0009C32D4F8B4326160002B40F00F858021F1
:106ED000D4F8D00272F014FBD4F8D002002172F082
:106EE0000FFB894B029A9A427FF69EADD9F88C1A15
:106EF00001297FF499AD854AD9F87C0A72F0DAFA53
:106F000092E59DF80CB0BBF1010F89F884BEDED884
:106F100094F89C32022BCCD0032B00F0D284D4F80E
:106F2000D002802172F0ECFAD4F8D002002172F085
:106F3000E7FAD4F8B432594620465B689847D0E760
:106F40000128D4F8D03244D194F89C22022A00F2CD
:106F50007884002A3DD0002122464FF0020C42F8EE
:106F6000081FC4F894C2C4E90700C3E914019A6475
:106F700018694FF480710128998703F13C0108BF1B
:106F8000DA64C2B2186872F025FCAAE7039B0022FB
:106F90001B0AADF81620013B062B98D801A252F827
:106FA00023F000BFDD700408C1700408EF7004080E
:106FB000CF6E0408CF6E0408A97004087970040825
:106FC0005CEA000CD4F8D03203D1039A7F2A40F255
:106FD0009F801846802172F093FAD4F8D0020021E5
:106FE00072F08EFA7DE794F89C32013B022B3FF65B
:106FF0006EAF039B012B7FF474AF0020D4F8D03226
:10700000C4F8A402E061042203F13C01C4F8942214
:107010004FF4807298649A871A69012AC3E91400B0
:1070200008BFD864D2B2186872F0D4FB59E7039B4A
:10703000012B7FF456AFC4F8A432D4F8D03200202C
:10704000E0E794F89C22D4F8D032013A022AC0D862
:107050000228BED1D4F8A4220021002A224618BF5B
:107060004FF0030B42F80CBFC4F89402C4E90700C8
:1070700018659A6459657BE7237C002B7FF427AF62
:10708000D4F8B4320DF116001B6B98470722034663
:107090004270BDF81620B4F8AE12002A40F0C38347
:1070A00000297FF41EAFC8E7237C002B7FF40FAFCD
:1070B000D4F8B4320DF116005B6B98470346E8E74D
:1070C000227CD4F8B432002A40F05C849B6A0DF133
:1070D00016009847022203464270DAE7D4F8B0322D
:1070E0000DF11601207C1B6898470346D1E79DF8F7
:1070F0000C30052B3FF6EBAEDFE813F065045D04C2
:1071000055044D04D20226040A30544F403D002459
:1071100094F89C22032A3FF45CAF03995FFA81FB49
:1071200084F89EB293F8BC23012A11D01A6800207B
:1071300083F838B0D2F800C82CF4FE6CC2F800C84E
:10714000D2F800C84CEA0111C2F8001883F8BC0359
:107150000422002003F13C01C4F894224FF4807211
:10716000E0619A871A699864012AD2B208BFD8648C
:10717000C3E91400186872F02DFBBBF1000F00F09A
:10718000F283022384F89C32ABE60122BA60D9F87C
:107190008C2AD0F840E0012AD3F808C000F0B8806B
:1071A000AC4A964500F0B981D9F88C3C5AEA030301
:1071B00000F03B82D8F808225FFA8AF1D9F8800EF5
:1071C00072F084FB2DE45C46DDF808B0FFF787BB66
:1071D000D8F8B4325B69002B3FF493AC98F89C224A
:1071E000032A7FF48EAC40469847D9F87CBA88E4ED
:1071F00047F6F07213423FF463ABC3F30A13C5EBD7
:10720000C502EF00D91C09EB82028908D2F884CCB0
:1072100009D00CEB810004F580566246316842F8D3
:10722000041B8242FAD17A1B0CEB030109EB8202A8
:10723000C2F8841CD2F8901C1944C2F8901CFFF7C5
:107240003FBBD9F8800E0122D0F8B43280F89C22DE
:1072500001795B689847D9F87C4AFFF797BBD9F862
:10726000803E042193F89C2283F89C1283F89D228F
:10727000FFF744BB6A6C1344AB64002CA8D1D9F867
:10728000CC2AD9F8C43A002A7FF42BAC0146724AC2
:107290005846019372F00EF9019B22E46F4B704A3D
:1072A0000344934240F244816E4B6F4A034493423D
:1072B00040F258816D4B6E4A0344934240F2CC81B8
:1072C0006C4B6D4A03449342C0F0FD816B4B6C4A9A
:1072D0000344934240F26D826A4B6B4A03449342EB
:1072E000C0F08582694B6A4A03449342FFF496AC2E
:1072F000684B694A03449342C0F0DF82674B684A97
:10730000034493422CBF4FF4C0534FF4E05387E43F
:107310001CF0080F00F01081624A96457FF681ABA1
:107320001CF4004F3FF47DAB4FF400429A60FFF72E
:1073300078BBD5F8B832002B7FF4A2ACD5F8C032B8
:10734000002B7FF49DACA1E4DDF804B074463BE46F
:1073500003F060025B0602D5402A7FF4B8AD94F8D2
:107360009C32013B022B3FF6B2AD5FFA8CFCBCF1C4
:10737000030F3FF6ACADD4F8B43220469B68984773
:10738000B4F8AE32002B7FF4ACAD00287FF4A9AD89
:10739000D4F8D03236E603F08001D4F8D00272F08F
:1073A000AFF89EE503F0600BBBF1200F00F0CB803F
:1073B000BBF1400F00F0C780BBF1000F7FF487AD39
:1073C0005FFA8CF3BEF1010F194600F09681BEF111
:1073D000030F00F07C81BEF1000F40F0698194F84A
:1073E0009C32D4F8D002022B00F00582032B7FF4EC
:1073F000F1AD1CF0800F01F00F024FF0140340F0CC
:10740000418203FB0242D2F858B1BBF1000F00F0F9
:10741000C68103FB014303F5AA73002940F0B5823E
:1074200000221A600222C4F89422C4E907220265ED
:107430000022836442654FF4807200F13C01828730
:107440000269012AD2B208BFC364006872F0C2F9AF
:1074500047E500BF0A31544F403D0024405327FF09
:10746000FF340C00401E1BFF3F420F0000DC0BFFEF
:107470007F4F1200808CF9FE20D6130060B6E5FE27
:107480005FE3160000D3CEFE40771B00C05BB3FE67
:10749000C091210000CA91FE20753800E05459FEC9
:1074A000E09C41000A30544FD8E90812914200F2A2
:1074B0008D80D8F81C10B1FBF2F302FB131313B943
:1074C0008A4240F2CD80D8F8B432DB682BB198F80C
:1074D0009C22032A01D1404698478021D8F8D00247
:1074E00072F00EF8D8F8D0320522002003F5FE71B4
:1074F000C8F894221A69C3F80802012AA3F8FC010B
:10750000D2B208BFC3F80C02C3E98400186872F055
:1075100061F9D9F87CBAFFF7EDBA1CF4004F7FF49B
:1075200003AF1CF0200F3FF445AE20229A6041E6E5
:107530004FF47053FFF774BB1CF0200F16D02022BD
:107540009A60FFF76EBAD4F8B43220469B68984729
:10755000C7E48021D8F8D00271F0D2FFD9F87CBA04
:10756000FFF7C8BA4FF46053FFF75ABBC34A9645BA
:1075700003D91CF4004F7FF4D7AE1B69D8F804225E
:10758000C3F31203D31AC8F81432D8F808321344DC
:10759000D9F88C2C5AEA0202C8F8083200F00D81A2
:1075A0001A465FFA8AF1D9F8800E72F08FF9FFF768
:1075B00038BAD4F8D0028021039271F0A1FF039A67
:1075C000D4F8D002114671F09BFF8AE48A1AD8F8E9
:1075D000D002C8F8202092B200F13C01C8F81C206B
:1075E00002650022836442654FF4807282870269DB
:1075F000012AD2B208BFC364006872F0EBF8D8F871
:10760000D03200211A69C3F80812012AA3F8FC112C
:10761000D2B2186808BFC3F80C12C3E9841103F58D
:10762000FE7172F0D7F8FFF765BA026C934B9A427D
:1076300003D90B68002BFFF6BDAD00230B610B696E
:1076400043F400230B610B6943F018030B610B69D2
:1076500043F0C0430B61ADE54FF45053FFF7E0BA80
:10766000D8F898329942BFF42EAFD8F8D032002023
:107670004FF48072C8F81C0003F13C019A871A6924
:107680009864012AD2B2C3E9140008BFD86418680C
:1076900072F0A0F80021D8F8D032C8F89812B1E7FB
:1076A000D4F8B032D3F814B0BBF1000F40F05481DD
:1076B000D4F8D002802171F023FF5946D4F8D002CB
:1076C00071F01EFF0DE44FF44053FFF7A9BA94F890
:1076D0009C22D4F8D032022A00F08480032A5DD1A3
:1076E000039A10437FF4ABAC48063FF4A8AC1846AD
:1076F000039371F005FF039BA1E494F89C32022BE5
:1077000062D0032BD4D1039B002B7FF4EAAB0A4653
:10771000D4F8D03251063FF492AC02F00F015A680F
:1077200091423FF68CACC1EBC1021CF0800F4FEAD6
:10773000820240F01D8102F5FE721C204FF0000C09
:1077400000FB01301A4480F8FDC1117000219170D6
:1077500093F8BC1301293FF472AC012183F8BC13E8
:1077600092F801C01078D178BCF1010F1A68A1F12C
:1077700002010CBF02F5106202F53062012902EB32
:107780004012106820F40010106003D8116841F016
:1077900080511160002283F8BC2350E418468021F8
:1077A00071F0AEFE5946D4F8D00271F0A9FEFFF791
:1077B00098BB4FF43053FFF733BA314A012102939B
:1077C00071F078FE029BEBE611F07F0BD4F8D0024B
:1077D000E5D071F095FED4F8D002802171F090FED2
:1077E000FFF77FBB11F07F0B1846D8D0F1E74FF4BD
:1077F0002053FFF715BA0B465B067FF4EBAB1CF08A
:10780000800F4FF002024FF0000114BF04F1140387
:1078100004F5AA731960C4F89422C4E90722C0E9E8
:107820001421836407E600293FF407AC8A42D4F8A8
:10783000D00228BF0A460221C4E90722C4F89412E4
:10784000F5E5032A7FF4C5AB0222211DC4F894227A
:107850000022C4E907005A654FF48072186503F1ED
:107860003C009A871A699964012AD2B208BFD96488
:107870000146186871F0AEFFFFF733BB0A30544F72
:10788000403D002403FB0243D3F818B0BBF1000FC6
:1078900085D001F07F02531C03EB830304EB8303C9
:1078A000002A3FF4BDAD1C2101FB020292F83E20EC
:1078B000003A18BF01221A60B4E54FF40053FFF7F5
:1078C000AFB9BBF1000F1CD0616801293FF4B5AB23
:1078D000D4F8B432C9B220465B68984799F8841E40
:1078E000D4F8B4326160002B3FF4F1AA1B68204643
:1078F000984700287FF4EBAAD4F8D032E061FFF774
:1079000082BB022359462046C4F804B084F89C3256
:10791000D4F8B4325B6898470422D4F8D032C4F863
:107920001CB0C4F894224FF4807203F13C01C3F8F8
:1079300048B09A871A69012AC3E914BB7FF472AB75
:10794000C3F84CB0FFF76EBBD4F8B032D3F818B020
:10795000BBF1000F3FF4ACAE0DF11601207CD8470F
:107960000346FFF796BB012384F89C32FFF7B9BAB0
:107970001C203C324FF0010C00FB01301A4480F80F
:107980003DC0E2E6DB6AFFF7A2BB1C2202FB01015D
:1079900091F8FE218CE7D4F8B032D3F810B0BBF1E7
:1079A000000FD9D184E6D4F8B032D3F80CB0BBF1D3
:1079B000000FD1D17CE6D4F8B032D3F808B0BBF1D7
:1079C000000FC9D174E6D4F8B032D3F804B0BBF1DB
:1079D000000FC1D16CE600BFF8B5594DD5F8CC43C6
:1079E00023699E0702D5E368980748D4236959079D
:1079F00002D5E3685A073AD423691B0702D5E36826
:107A00001F072CD42369DE0602D5E368D8061ED4EE
:107A10002369D90702D5E368DA0738D423691B063E
:107A200002D5E3681F066ED42369DE0502D5E3683C
:107A30001D066FD42369580602D5E368590670D431
:107A400023699A0602D5E3689B0671D4F8BD6FF0EE
:107A5000100200232261E26985F8E833D8E76FF06D
:107A6000080200232261E26985F8E833CAE76FF073
:107A7000040200232261A26985F8E833BCE76FF0B5
:107A8000020200232261A26985F8E833AEE72D4B9C
:107A90006FF001029C422261C0D1D5E9D967BE4294
:107AA000BCD0D5F848238CBFC6F58057BF1B264BEA
:107AB000D2F814C23344B9B2C2F80832C2F8101274
:107AC000BCF1000FAAD14FF0010ED5F860033E447F
:107AD000C5F8C010C2F814E240F201124366A0F8E3
:107AE000582002697245D2B2C0E91B1C08BF8366E8
:107AF00000F15801006871F05DFDB6F5805F1BD0A4
:107B0000C5F864638AE76FF0800323612369DE05AB
:107B100090D58CE76FF480732361236958068FD565
:107B20008BE76FF04003236123699A068ED58AE7BD
:107B30006FF020032361F8BD0023C5F864336DE7BF
:107B4000002F002400140040884D0024034B93F8BC
:107B50002400032894BF00200120704774320024C1
:107B6000004870479C32002470B4154D00202B460D
:107B700093F82A4014B1DE698E4205D001301033EB
:107B80000828F5D170BC7047AAB1AB6903EB40235C
:107B90009A4201D1022C07D095F8B83113B90123CC
:107BA00085F8B83101236B7005EB0015012385F8CA
:107BB0002A3070BC704705EB001585F82A20E1E7F4
:107BC000A05D002430B40023184C204684F8A43073
:107BD00003E001331030082B1AD0C5698D42F8D16B
:107BE00090F82AC0BCF1030FF3D19AB1A16901EB5F
:107BF00043218A4207D094F8B82112B9012284F8AF
:107C0000B8210122627004EB0314012384F82A30A6
:107C100030BC7047D4F8A02004EB031304210132D8
:107C200083F82A10C4F8A020F2E700BFA05D00246A
:107C3000A0B183681BB10C4B07229A7070470A4AA7
:107C400004211078137503289170C2E9033314BF1F
:107C50004FF480738023C2E901337047024B012245
:107C600083F8B8215A707047A05D00240346202293
:107C700001481A80704700BFD01800240346202214
:107C800001481A80704700BFF018002403462022E4
:107C900001481A80704700BF1019002403460A22C9
:107CA00001481A80704700BF3019002410B50E4BF0
:107CB0000E4C03F16C02DB6ED4F83415B4F83805C1
:107CC000C4F8D02588619847D4F8D035002BFBD074
:107CD0001B6998470028F7D0B4F838350020D4F84D
:107CE00034251B04936110BDD0180024A05D00242E
:107CF00038B5084BD3F8D03553B1DB6914460D467F
:107D000098474FF40073026800202A60238038BD32
:107D10001B68FFDEA05D002408B5064BD3F8D03504
:107D200023B11B699847013840B208BD4FF0FF30BE
:107D300008BD00BFA05D0024002070472DE9F04180
:107D4000194C1546B4F84425D4F84005160486614C
:107D500023B30E4603EB050804E0D4F8D0350BB38B
:107D60001B699847D4F8D015E1B100234F68284625
:107D700031461A46B8470028EFD0D4F8D035002B4A
:107D8000FBD01B6998470028F7D0013506F500762F
:107D9000A845E7D1D4F84005B4F844258261002015
:107DA000BDE8F081FEE700BFA05D00242DE9F041B1
:107DB000184C1546B4F84425D4F8400516048661DD
:107DC00023B30E4603EB050801E01B699847D4F87E
:107DD000D01551B10023CF68284631461A46B8471E
:107DE000D4F8D03510B1002BEFD1002313B11B69AB
:107DF000984710B9D4F8D035F8E7013506F5007684
:107E00004545E4D1D4F84005B4F84425826100200A
:107E1000BDE8F081A05D002400207047704700BFDE
:107E2000007970470079C0F340107047007940092D
:107E3000704700BF704700BF03685A1C026019708A
:107E4000704700BF03685A1C02601970704700BF7A
:107E5000024BD3F8D40503681B681847A05D0024C3
:107E60002DE9F0413A4E33787E2B03D00027384677
:107E7000BDE8F08108214FF4FC4341F221041AB21D
:107E80005B00002A84EA42009BB2B8BF83B201398A
:107E9000F5D1B6F80140002C37D02E4A2E4DAA421B
:107EA000E4D2052CA2F106028CBF0027012714445E
:107EB000AC4228BF47F00107002F47D141F2210E05
:107EC000A24214D0501E04F1FF3810F8011F0822FE
:107ED00083EA012319B25B0000298EEA410C9BB2B0
:107EE000B8BF1FFA8CF3013AF4D14045EDD1218897
:107EF00061B1A21DAA42BAD2052904EB01002246B3
:107F0000B5D9A842B3D20446DAE7144C671E41F251
:107F10002105BC4617F8012F83EA0223082219B273
:107F20005B00002985EA41009BB2B8BF83B2013AE9
:107F3000F5D16445EDD16788094AFF1A231DB7FAC8
:107F400087F79B1B7F09A2F8D83590E70F468EE78D
:107F500000000208070002080000040801000208EF
:107F6000A05D002410B50B4C236D23B119689A88CD
:107F70000B691A420AD0FDF76DFC38B9064B012295
:107F800020761B6884F82420636110BD002384F8E8
:107F9000243010BD743200240C33002438B5037C27
:107FA0000446D0F8D002002B52D14FF400730222C5
:107FB000012171F0FFF901204FF40073C4F86C0146
:107FC0000222D4F8D002812171F0F4F9244B002070
:107FD000D4F8CC22012103F5BC65E162C4F8C85293
:107FE000A3F8E807A3F83C0813689847D4F8D042F0
:107FF00094F8BC332068012B12D01022194B026177
:10800000013B02D00269D106FAD46022154B02610D
:10801000013B02D002699206FAD4002384F8BC33F3
:108020000022114B1F2504F50671C4F830220122ED
:10803000C4F82C52A4F818222269C4F82432012A68
:10804000D2B208BFC4F8283271F0B4FA002038BDAB
:1080500040230222012171F0ADF901204023ADE758
:10806000A05D0024410D03008C65002470B5002242
:10807000D0F8C84205461C4B84F838120D2684F807
:10808000082204F50B70C4F82C3204F50374D5F8FB
:10809000D0322E631A6740F2011203F15801DE66F6
:1080A000A3F858201A695866012AD2B208BF986608
:1080B000186871F07FFAD5F8D0321F200022012114
:1080C000C3F82442C3E98B021A69A3F818128A4242
:1080D0001868D2B203F5067108BFC3F82842BDE89C
:1080E000704071F067BA00BF555342532DE9F04319
:1080F000177883B0164605468846D0F8C8425A2FEE
:108100005CD8DFE817F0C5005B005B0076005B0021
:108110005B005B005B005B005B005B005B005B0087
:108120005B005B005B005B005B00A7005B005B002B
:108130005B005B005B005B005B00600171005B004B
:108140005B0071005B005B005B005B0010025B008A
:1081500073015B005B0097015B0007015B005B0044
:108160005B005B00D5005B005B005B005B005B00BD
:108170005B005B005B005B005B005B005B005B0027
:108180005B005B005B005B005B005B005B005B0017
:108190005B005B005B005B005B005B005B005B0007
:1081A0005B005B005B005B005B005B005B005B00F7
:1081B0005B005B005B005B005B00F30094F85D22FA
:1081C000002105254FF0FF30531C04EBC202DBB247
:1081D00082F83C5282F84012042B08BF0B4684F808
:1081E0005D3203B0BDE8F0830023A4F80A3200201A
:1081F000F7E77021002294F85C3221700C21C4F85A
:108200000520E17194F85D12C4F801209942C4F888
:108210000920C4F80D20627413D004EBC3010133AC
:1082200091F83C02DBB2A070042B91F8410220735C
:1082300091F8401218BF84F85C32617308BF84F86B
:108240005C221223A4F80A323379122BCFD8A4F877
:108250000A32CCE75378DB0700F18981D0F8CC32C1
:1082600001EBC1011279D86900EB81000379053374
:10827000934228BF1346A4F80A32002BB7D0C21885
:10828000234412F8011D824203F8011DF9D1AEE723
:10829000D4F81462002E40F01382D5F8CC32084690
:1082A0009B689847002840F05982A4F80A029EE78C
:1082B000537813F0020340F0DE81D4F86012D4E961
:1082C000992002448A42C2D994F85D2205201146C1
:1082D0000132D2B204EBC101042A81F83C0281F8D8
:1082E000403200F0FC8184F85D2280E7C84B082210
:1082F00003CBA4F80A22206040466160D5F8CC3256
:10830000DB68984700283FF472AFE37863F07F039F
:10831000E3706CE794F80892B9F1000F40F04781E0
:1083200094F91832002BC0F26A82D0F8CC32084699
:108330009B6898470746002840F04D82D5F8CC321C
:108340004046DB6898470146002840F01B81D6F87C
:108350000220D5F8C80212BAC4F86422B6F8073071
:10836000D0F860625BBA9BB21A44C4F86832B24279
:1083700000F22082B4F85E2202FB03F3D4F8142248
:10838000934240F06881B3F5007F4FF0010028BFB1
:108390004FF4007384F808021A46D5F8D032C3F8B7
:1083A0002C221A69C3F8301203F506718242A3F831
:1083B0001802D2B21868C3F8244208BFC3F8284292
:1083C00071F0F8F813E70023082208462360636081
:1083D000D5F8CC32A4F80A22DB68984700283FF48D
:1083E00006AFA37863F07F03A37000E7D0F8CC3228
:1083F00004F25E22084604F518715B68984700286D
:1084000040F07081D4F860320822A080013BA4F8CB
:108410000A22190E1A0C61F30700190A62F30F20E1
:10842000B4F85E2261F3174052BA63F31F60E28032
:108430002060DCE694F80872002F40F0B68094F9D2
:108440001832002B80F2A581D0F8CC3208469B6808
:108450009847002840F09680D6F8022012BAC4F857
:108460006422B6F80730D5F8C8625BBAD6F8601255
:108470009BB21A44C4F868328A4200F24781B4F8C9
:108480005E2202FB03F3022284F80822D4F81422AD
:108490009A4240F03B814FF40073D5F8CC2240461D
:1084A0003146A4F80A32B6F85E32D6F86842176947
:1084B00003FB04F4D6F86422B4F5007F28BF4FF420
:1084C0000074B4FBF3F39BB2B8470028C0F23481C8
:1084D000D5F8D03200222C6303F1580118685E668B
:1084E000C3E91B4240F20112A3F858201A69012A7D
:1084F000D2B208BF9E6671F05DF8B6F85E22B4FB9A
:10850000F2F2D6E9991311449B1AD6F83422121BC1
:10851000C6E99913C6F83422002B7FF468AE032312
:1085200086F8083263E6002608460DF1020201A92A
:1085300026606660A660D5F8CC325B689847002854
:1085400040F0AB8008200223BDF802200C21E0702F
:10855000238152BA019BA4F80A12013B6281180ED2
:10856000E371190C1A0A20716171A2713FE6294B5F
:108570000722186899889B79A180A4F80A222060B4
:10858000A37134E6D5F8C822022092F85D3202EBDE
:10859000C3010133DBB281F83C0281F84072042B45
:1085A00000F0F48082F85D3221E6264673E7B4F8E5
:1085B0005E320846D4F868622146D5F8CC2203FB27
:1085C00006F65769B6F5007FD4F8642228BF4FF449
:1085D0000076B6FBF3F39BB2B8470028C0F22181C6
:1085E000B4F85E32D4F86422D4F86812B6FBF3F023
:1085F0000244091AC4F86422D4F83422C4F8681278
:10860000921BC4F8342239B92846FFF72FFDEEE556
:1086100038470C0830470C08D5F8D00201FB03F3AB
:1086200001220021B3F5007FC0F82442A0F81822EF
:10863000026928BF4FF40073C0F8301200F50671CC
:10864000012AC0F82C32D2B208BFC0F82842006814
:1086500070F0B0FFCBE590F85D3205245A1C00EBBA
:10866000C303D2B283F83C4283F84012042A60D09C
:1086700080F85D22BBE594F85D32052000215A1C8C
:1086800004EBC303D2B283F83C0283F84012042AFD
:108690007FF429AE84F85D12A9E5D5F8C82202203E
:1086A00092F85D3202EBC3010133DBB281F83C0288
:1086B00081F84062042B7FF475AF82F85D6296E525
:1086C00094F85D32052000211A460133DBB204EB39
:1086D000C202042B82F83C0282F84012DAD084F8FD
:1086E0005D3284E5D5F8C8220224002192F85D327B
:1086F00002EBC3000133DBB280F83C4280F8401249
:10870000042B7FF44FAF82F85D1270E596F85D326E
:1087100005211A460133DBB206EBC202042B82F8B4
:108720003C1282F8400214BF86F85D3286F85D0282
:108730005DE580F85D125AE5D5F8C82204240021D1
:1087400092F85D3202EBC3000133DBB280F83C42A9
:1087500080F84012A3427FF425AFD4E7D5F8C822B1
:108760000520022592F85D3292F85D12013302EB8A
:10877000C101DBB281F84062042B08BF3B4681F89F
:108780003C5282F85D3284F8080230E582F85D726E
:108790002DE594F85D3205211A460133DBB204EB76
:1087A000C202042B82F83C1282F8407297D184F8FE
:1087B0005D721CE590F85D3205241A460133DBB288
:1087C00000EBC202042B82F83C4282F84012B0D087
:1087D00080F85D320BE5D5F8C822022092F85D32B0
:1087E00019460133DBB202EBC101042B81F83C02D4
:1087F00081F840927FF4D6AE82F85D92F7E494F867
:108800005D3205211A460133DBB204EBC202042BB0
:1088100082F83C1282F840927FF461AF84F85D9256
:10882000E5E4D5F8C8220424002092F85D32194608
:108830000133DBB202EBC101A34281F83C4281F873
:1088400040027FF4AFAE82F85D02D0E4D0F8C812E7
:1088500010B591F80832022B07D0033B012B02D848
:108860000021FFF703FC002010BD01F21B2291F84C
:1088700019120446FFF73AFC0028F4DA01212046D9
:10888000FFF7F4FBEFE700BF70B5D0F8D05201213D
:10889000044695F8BC33A5F818128B4208D0002284
:1088A000286885F8BC1371F071F8002385F8BC3393
:1088B000D4F8D052002640F20112C4F86C6195F849
:1088C000BC33A5F85820012B08D001222868114696
:1088D00085F8BC2371F05AF885F8BC630025D4F8FC
:1088E000C802E5627BF01AF82846C4F8C85270BD89
:1088F00038B5D0F8C8520446D0F8D00295F81832EE
:1089000013B9D5F814323BB9812170F0F9FD95F80F
:108910000932022B0ED038BD95F80932002BF3D165
:10892000012170F0EDFDD4F8D0028121BDE838407E
:1089300070F0E6BDD4F8D0321F20002205F5037593
:108940000121C3F82452A3F8181203F50671C3E9F4
:108950008B021A691868012AD2B208BFC3F82852DC
:10896000BDE8384070F026BE70B5D0F8C842054664
:1089700094F8086286B1012E01D0002070BD04F287
:108980001B2294F81912FFF7B1FB0028F5DA012138
:108990002846FFF76BFBF0E7D4F81432D4F8102226
:1089A000C4F83432D0F8D032C4F83022D3F83032A0
:1089B0001F2B08D1324BD4F80C229A4203D194F8E1
:1089C0001912012918D994F85D320021052628468C
:1089D00004EBC3020133DBB282F83C6282F840123E
:1089E0000222042B84F8092208BF0B4684F85D326A
:1089F000FFF77EFF002070BD94F81A32013B0F2B69
:108A0000E1D804F21B22FFF771FB002894F808322A
:108A10002BDB013B022BB0D9B4F80A1259B3D5F8BD
:108A2000C832042283F80822D3F8342283F838624B
:108A3000521AC3F83422D3F81432994228BF194687
:108A4000D5F8D0321A692963012AD96640F201119A
:108A5000D2B21868A3F8581003F158015C661E677B
:108A600008BF9C6670F0A6FD87E7052B8FD02846CF
:108A7000FFF73EFF81E72846FFF7F8FA7DE700BFE2
:108A8000555342432DE9F041002382B00446D0F80B
:108A9000C852ADF806300B7813F0600239D0202AA6
:108AA0000DD08021D4F8D00270F02AFD0021D4F836
:108AB000D00270F025FD022002B0BDE8F0814A78B6
:108AC000FE2A00F0DD80FF2AEBD14A88002AE8D197
:108AD000CA88002AE5D11B06E3D44FF4807305F55C
:108AE00003700121A5F80832D4F8D0321F24C3E95D
:108AF0008B421A69C3F82402012AA3F81812D2B2D1
:108B000003F5067108BFC3F82802186870F052FD1B
:108B100025E04B780B2BC4D801A252F823F000BFFC
:108B2000438C0408838B0408A38A0408A38A0408DE
:108B3000A38A0408A38A0408A38A0408A38A040851
:108B4000A38A0408A38A0408638B0408518B0408D1
:108B500090F89C32032BA4D18B78C5F80432002006
:108B6000AAE790F89C32D0F8D002032B00F0B28034
:108B7000802170F0C5FC0021D4F8D00270F0C0FC58
:108B800099E7D0F8D0628F8896F8BC3391F9042029
:108B900007F00F07012B00F006810123002A31683E
:108BA00086F8BC33C0F2AC801023884A0B61013ACE
:108BB00000F000810B6913F01003F8D186F8BC3384
:108BC000C7EBC7039B00C7EBC7024FF0000803F5D4
:108BD000FE7306EB8202F11882F8FC7182F8FD81C7
:108BE00096F8BC23012A09D00122306886F8BC23FC
:108BF0004A78F15C70F0CAFE86F8BC8307EB870701
:108C00000023D4F8D00204EB8707C7F85831237C3F
:108C1000002B40F0BC804FF400730222012170F061
:108C2000C9FB0123C4F86C3195F80932022B96D1A7
:108C30008121D4F8D00270F063FC002385F809325A
:108C40008DE790F89C32D0F8D002032B90D102230C
:108C5000002200F13C01C4F89432C4E907334265B4
:108C60000DF10604026903654FF48073012A8464E0
:108C7000838700D1C464D2B2006870F0ABFD6EE7A8
:108C80004E88002E7FF40DAFCF88012F7FF409AFFF
:108C90001A067FF506AFD0F8CC3205F500759B6952
:108CA000984702222860D4F8D032C4F894224FF4B6
:108CB000807203F13C011868C4E907779A871A6942
:108CC0009D64012A1F65D2B25E6508BFDD6470F045
:108CD00081FD44E70222012305F501754FF48071FF
:108CE000C4F894220022C4E90733C0E914320269AF
:108CF000818700F13C019A42856408BFC564BAE7E8
:108D0000BB01324A43F020030B61013A58D00B6992
:108D100013F02003F9D186F8BC33C7EBC7039B00DF
:108D2000C7EBC70201213C3306EB8202F01882F840
:108D30003C7082F83D1096F8BC238A4209D086F830
:108D4000BC134278F15C306870F020FE002386F896
:108D5000BC3307EB87070023D4F8D00204EB870766
:108D6000BB61237CCBB94FF400730222812170F0E8
:108D700021FB0121E16295F80932022B3FF458AF43
:108D8000012B3FF4ECAE2046FFF770F9E7E64023F5
:108D90000222012170F00EFB43E7402302228121D1
:108DA00070F008FBE5E7C7EBC703002A4FEA83032F
:108DB000B6DB08E7C7EBC70386F8BC239B0002E7D6
:108DC000C7EBC70386F8BC239B00A9E7410D03004E
:108DD0002DE9F8430D46D0E9003113448B4220D8E9
:108DE0000446AE18476BCAB14FF0000900F11008F5
:108DF00001E0AE4212D0236B5A1C23442263202A86
:108E000015F8011B1974F4D14146204617B9FAF739
:108E1000CDF90746AE42C4E90C97ECD13846BDE81F
:108E2000F8834FF0FF37F9E700680379012B0AD088
:108E3000022B01D0002070478368F022DB0718D591
:108E4000FF2104F0ADBC826890F910C002F001026D
:108E5000417C60464FF0F00C10B584B00DF10F046A
:108E60000192FF228DF80FC00094FAF785FC04B040
:108E700010BD7F2104F094BC70B5056884B0044631
:108E80000E462B79012B16D0022B02D0002004B005
:108E900070BDAB68E122DB071DD52846114604F002
:108EA0007FFC0028F2D03246FF21206804B0BDE8E4
:108EB000704005F01DB8AA68697C02F0010295F9BE
:108EC00010000DF10F050192E12200958DF80F20A1
:108ED000FAF752FCE5E76121284604F061FCE0E77F
:108EE00070B5056884B004460E462B79012B17D067
:108EF000022B02D0002004B070BDAB68C32228460C
:108F0000DB074CBFE121612104F04AFC0028F1D0CD
:108F10003246FF21206804B0BDE8704004F0E8BF8D
:108F2000AA6895F9100002F00102697C01920DF126
:108F30000F020092C3228DF80F20E122FAF71CFCE9
:108F4000E4E700BF0068CA43037941EA0211012B3C
:108F5000CAB209D0022B01D0002070478368DB071A
:108F600016D5D22104F01CBC10B584B0846890F9E9
:108F700010C08DF80F200DF10F0204F00104417CA8
:108F80000092D22260460194FAF7F6FB04B010BDBD
:108F9000522104F005BC00BF70B5056884B00446DA
:108FA0000E462B79012B1BD0022B02D0002004B0DF
:108FB00070BDAB68F0222846DB074CBFE121612180
:108FC00004F0EEFB0028F1D02246FF2152F8040BFA
:108FD00004F08EFF0028E9D02379337004B070BD0F
:108FE000AA6895F9100002F00102697C01920DF166
:108FF0000F020092F0228DF80F20E122FAF7BCFB5D
:10900000E0E700BF00680379012B0AD0022B01D0F2
:10901000002070478368B422DB0718D5FF2104F0D5
:10902000BFBB826890F910C002F00102417C60462B
:109030004FF0B40C10B584B00DF10F040192FF2273
:109040008DF80FC00094FAF797FB04B010BD7F2194
:1090500004F0A6BB00680379012B0AD0022B01D0D3
:109060000020704783680A46DB0716D5A52104F067
:1090700097BB10B584B0846890F910C00DF10F0251
:1090800004F001048DF80F10417C60460092A52287
:109090000194FAF771FB04B010BD252104F080BBE8
:1090A00000680379012B0AD0022B01D00020704701
:1090B00083689622DB0718D5FF2104F071BB826814
:1090C00090F910C002F00102417C60464FF0960C0E
:1090D00010B584B00DF10F040192FF228DF80FC07E
:1090E0000094FAF749FB04B010BD7F2104F058BB8F
:1090F00000680379012B0AD0022B01D000207047B1
:1091000083680A46DB0716D5872104F049BB10B5F2
:1091100084B0846890F910C00DF10F0204F00104CE
:109120008DF80F10417C6046009287220194FAF777
:1091300023FB04B010BD072104F032BB0068C90155
:109140000379CAB2012B06D0022B01D00020704750
:10915000782104F025BB10B584B0846890F910C064
:109160008DF80F200DF10F0204F00104417C0092F4
:10917000782260460194FAF7FFFA04B010BD00BFF0
:1091800000680379012B0AD0022B01D00020704720
:1091900083685522DB0718D5A52104F001BB82683E
:1091A00090F910C002F00102417C60464FF0550C6E
:1091B00010B584B00DF10F040192A5228DF80FC0F7
:1091C0000094FAF7D9FA04B010BD252104F0E8BAEA
:1091D000F0B5044683B00D461746061D2068037996
:1091E000012B19D0022B02D0002003B0F0BD836800
:1091F0003246FF21DB075CBF3246FF2104F01EFE32
:109200000028F1D015B12379DB07E7D4002FECD08B
:1092100023793B7003B0F0BD8268417C02F0010C01
:1092200090F91000FF22CDE9006CFAF7D5FCE7E7D2
:1092300070B50446051D82B020680379012B16D055
:10924000022B02D0002002B070BD83682A46FF21A5
:10925000DE075CBF2A46FF2104F0F0FD0028F1D0B4
:109260002379DB07EFD520680379012BE8D18668E5
:10927000FF22417C06F0010690F91000CDE900566E
:10928000FAF7AAFCEAE700BF024630B5044652F8F6
:10929000040B83B00379012B0ED0022B01D00020E8
:1092A00008E0FF2104F0CAFD0028F8D02079C0436F
:1092B00000F0010003B030BD8568417C05F0010578
:1092C00090F910000092FF220195FAF785FCEBE778
:1092D00070B5B42282B00446FF21006804F0BEFAE3
:1092E00010B9002002B070BD2068251D0379012B44
:1092F00013D0022BF5D183682A46FF21DE075CBF1D
:109300002A46FF2104F09AFD0028EAD02379DB07E2
:10931000E8D520680379012BEBD18668FF22417CD8
:1093200006F0010690F91000CDE90056FAF754FC5A
:10933000EAE700BF70B50A4682B00446A52100687E
:1093400004F08CFA10B9002002B070BD2068251D11
:109350000379012B13D0022BF5D183682A46FF2114
:10936000DE075CBF2A46FF2104F068FD0028EAD032
:109370002379DB07E8D520680379012BEBD18668D8
:10938000FF22417C06F0010690F91000CDE900565D
:10939000FAF722FCEAE700BF70B582B00446CDE9D7
:1093A0000023FFF795FF10B9002002B070BD5522D1
:1093B000A521206804F052FA0028F5D0251D2A4680
:1093C000FF21206804F094FD0028EDD02379DB070D
:1093D000F5D40DF1FF350DF1070615F8011F2046F4
:1093E000FFF7A8FF0028DFD0B542F6D1DDE700BFC8
:1093F000002A34D0F0B5044683B00E46051D8F1800
:1094000016F8012BA521206804F028FA90B9002055
:1094100003B0F0BD8268417C02F0010C90F91000AD
:10942000FF22CDE9005CFAF7D7FB0028EFD02379C3
:10943000DB070FD520680379012BEBD0022BE6D197
:1094400083682A46FF21DB075CBF2A46FF2104F020
:10945000F5FCEAE7B742D3D1012003B0F0BD01200B
:10946000704700BFF0B5962283B00E460446FF2138
:10947000006804F0F3F910B9002003B0F0BD251D19
:1094800020680379012B1ED0022BF5D183682A4670
:10949000FF21DF075CBF2A46FF2104F0CFFC002834
:1094A000EAD02379DB07EBD4E1222068114604F0EF
:1094B000D5F90028E0D03246FF21206803B0BDE88E
:1094C000F04004F015BD8768FF22417C07F00107DA
:1094D00090F91000CDE90057FAF77EFBDFE700BFF7
:1094E000002A42D0F0B5044683B00E46051D8F1801
:1094F0009622FF21206804F0B1F990B9002003B052
:10950000F0BD8268417C02F0010C90F91000FF224E
:10951000CDE9005CFAF760FB0028EFD02379DB0788
:109520000FD520680379012BEBD0022BE6D183689D
:109530002A46FF21DB075CBF2A46FF2104F07EFCA0
:10954000EAE7E1222068114604F088F90028D5D026
:109550003246FF21206804F0CBFC0028CED0013633
:10956000B742C5D1012003B0F0BD0120704700BF54
:10957000F0B50B4605461646044683B087211A46C9
:1095800055F8040B04F06AF920680379012B19D00F
:10959000022B02D0002003B0F0BD83682A46FF21D1
:1095A000DF075CBF2A46FF2104F048FC0028F1D009
:1095B0002379DA07E8D4002EEDD0C3F340133370DB
:1095C00003B0F0BD8768FF22417C07F0010790F9E6
:1095D0001000CDE90057FAF7FFFAE7E7F0B5782178
:1095E00083B0164604460022006804F037F910B92B
:1095F000002003B0F0BD251D20680379012B13D096
:10960000022BF5D183682A46FF21DF075CBF2A467B
:10961000FF2104F013FC0028EAD02379DA07EBD409
:109620005B09337003B0F0BD8768FF22417C07F00F
:10963000010790F91000CDE90057FAF7CDFAEAE7F3
:1096400070B5CC2282B00446A521006804F006F96A
:1096500010B9002002B070BD2068251D0379012BD0
:1096600013D0022BF5D183682A46FF21DE075CBFA9
:109670002A46FF2104F0E2FB0028EAD02379DB0729
:10968000E8D520680379012BEBD18668FF22417C65
:1096900006F0010690F91000CDE90056FAF79CFAA1
:1096A000EAE700BF70B5B42282B00446FF2100682B
:1096B00004F0D4F810B9002002B070BD251D206858
:1096C0000379012B21D0022BF5D183682A46FF2193
:1096D000DE075CBF2A46FF2104F0B0FB0028EAD079
:1096E0002379DA07EBD4CC212046FFF723FE0028AC
:1096F000E1D002E02379DB07DED52A46FF2120688E
:1097000004F0F6FB0028F5D1D5E78668FF22417CFE
:1097100006F0010690F91000CDE90056FAF75CFA60
:10972000DCE700BF02784368022A0FD00B490269C8
:10973000D1F81C02023A184010B4400AD1E984144E
:1097400004FB02005DF8044B08447047034AD2E969
:10975000812102EB410202EB53207047A05D0024FF
:109760002DE9F04F83B002F002077D4D019308B957
:10977000002F65D1D5F80C42002C4FD14FF0FF3EA1
:10978000774C4FF0000CF146F046F246E36994F84E
:109790002A60984200F09580C6B3012E05EB0C1BA1
:1097A0000AD19BF82B60F30706D416F07E0F03D185
:1097B000F60900F08980E0460CF1010C1034BCF190
:1097C000080FE3D1BEF1000F04DAB8F1000FC0F2C8
:1097D0008D80C646D5F89C4005EB0E1C0EF10206A6
:1097E0000134CCE9070405EB061CC5F89C40CCF815
:1097F00004400024CCF8084005EB0614A47A042C9D
:109800001ED8DFE804F0274119414300E6460CF179
:10981000010C1034BCF1080FB8D1D3E7D5E9843678
:1098200006FB0434A042A9D395F8B83113B901233B
:1098300085F8B83101236B70002003B0BDE8F08FCC
:1098400095F8B831002B4DD0012302206B7003B086
:10985000BDE8F08F12F00104D5F818C06CD105EB0B
:109860000610019B4FEAE20C90F80B80032B6CF37F
:10987000C71880F80B805DD94FF6FF70834228BF70
:10988000034605EB06100381002F41D1500705D593
:1098900005EB0610C37A43F00103C372D30608D563
:1098A00005EB0616F37AC3F34502013262F3460371
:1098B000F372AB69012003EB4E230B6003B0BDE8EC
:1098C000F08FC6B9E64685E7666A1034B24588BFB0
:1098D000E1460CF1010C88BFB246BCF1080F7FF4E1
:1098E00055AF6FE7012385F8B831ADE7B9F1000F47
:1098F000A2DBCE466EE7D5F89C400CF10206E646A8
:10990000013405EB061CC5F89C40CCF8044073E715
:10991000D5F8A000D5F89C3001300133C5F8A0007F
:1099200005EB0E10C5F89C30036205EB061304200E
:109930009872ABE72346A4E7D5F8D035002B3FF467
:109940007BAF5C680CEB4E210023064AA047002841
:109950003FF472AF05EB06160223B3726CE700BF4B
:10996000A05D0024697B040870B5104D82B00E46DE
:109970002B78022B15D1020AC4B2D5F804020023B9
:1099800001A910440322FFF7EBFE012807D12B7831
:10999000019A022B0CBF22F8146042F8246002B036
:1099A00070BDC0F3D41200F07F04E6E7A05D002490
:1099B0002DE9F04F434E0D4683B0174631782B68A2
:1099C00003293DD002295FD14FEA13294FF4807A51
:1099D0005FFA83F8421E012A23D84FF0010B9F4201
:1099E0001AD901288CBF00240124D6F87C211AB191
:1099F000D6F8981199424AD0D6F8040200230922D9
:109A000001A94844FFF7ACFE012822D0022813D058
:109A100020B12B689F42E8D803202F6003B0BDE837
:109A2000F08FB8F1000F12D096F8B83113B90123B6
:109A300086F8B83101237370022003B0BDE8F08FBF
:109A40004FF0800AC3F3D41903F07F08C2E7D3466E
:109A5000C5E73178022913D00329EDD1019B53F8D2
:109A6000282022F07042B2FA82F22B685209A242F8
:109A70001FD0D8445B44D0452B601DD20229EDD1C4
:109A8000019B33F81820EEE74FF4807ADAE7D6F836
:109A90001412013A02EB41224902B2FBF1F21344E3
:109AA000B3FBFBF20BFB12320AB15B449B1A2B6037
:109AB000B0E79F42B2D8AFE709F101094FF00008C3
:109AC000A8E700BFA05D00242DE9F04FDFF88491E6
:109AD0008B4685B0174699F800C00968BCF1020FA3
:109AE000D9F8045240F08280CEB24FF4807305EB77
:109AF0001125A6EB010890449844B94208F1FF38BB
:109B0000B8FBF3F84AD200F00103A8446FF0404AD2
:109B10000193BCF1030F07EB0604A8EB05032846ED
:109B200014BF4FF480728022641A03A9944228BFA4
:109B30001446944228BF002E14BF012200220A328C
:109B4000FFF70EFE01282AD199F800C0DBF800E0EB
:109B5000BCF1020F0EF1010324D0B44255D9039891
:109B600006EB0A02011F00EB820201EB840142F8BE
:109B7000043F8A4203F10103F9D1DBF80030A11B55
:109B800019448F42CBF8001002D1019B002B48D121
:109B90008F4205F101054FF00006BAD8012005B04B
:109BA000BDE8F08FB44246D903986FF00042811EA1
:109BB000324401EB440100EB420222F8023F9142A1
:109BC00003F10103F9D1A11B71448F42CBF80010BE
:109BD000DED1019B002BDBD086466FF000434FF6B1
:109BE000FF72012023442EF81320D8E701F07F06EE
:109BF000C1F3D413BCF1030FA6EB01081D4414BF3D
:109C00004FF480738023904476E7AEEB060E0EEBA4
:109C100004018F42CBF80010BAD1019B002BB7D0C2
:109C200003986FF040434FF0FF32234440F8232065
:109C3000DBF80010ACE7AEEB060E0EEB04018F4232
:109C4000CBF80010A4D1019B002BA1D0DDF80CE0D3
:109C5000C3E700BFA05D002430B50446C06983B0EF
:109C600010B9012003B030BD0D460023032201A925
:109C7000FFF776FD0128F5D1B4F92020002A19DB81
:109C8000019B012D4FEA421103EB421203D0022D3A
:109C90001AD1E5205854A368D3612378032B04D14B
:109CA0000023137753779377D377636A190C538321
:109CB0009182D6E7054A92F8B81109B982F8B8013D
:109CC000012302205370CDE7E368E5E7A05D00249F
:109CD0002DE9F041044682B00D4694F83C30042B47
:109CE0007DD8DFE803F02A03684839003D4E4FF67F
:109CF000F777DFF8F48016E0BA425AD86BF0F2F941
:109D000001284FF0000133D1206BFFF72DFE012811
:109D10002ED1019AD6F81812531E22638B4228BF07
:109D20000B46C6F81832327801A9236B032A18466D
:109D30009AB2E1D14345E1D93BE06900204601F008
:109D4000FE01FFF789FF01283FD1636B002B18BF8D
:109D5000022084F83C00C0E794F82830042B02D19C
:109D6000002384F82830A36B0BB1204698470120CC
:109D700002B0BDE8F0811B4E0021E26AD6F89831AE
:109D800006F5BA70C6F898219B1AD6F8142202FB81
:109D900003F3D6F87C2102EB4322C6F87C21D6F8E7
:109DA000802102EB4322C6F88021FFF755FF0128EE
:109DB0000BD10420CDE7626B04F130010020FFF7E6
:109DC00083FE012801D10320C3E70228D0D194F8F3
:109DD0002830042BCCD1002384F82830C8E7022097
:109DE000F5E700BFA05D0024F7FFFF0F38B504467C
:109DF00094F83430052B60D8DFE803F031251D13CB
:109E00000D0394F82830082B3FD02D4B012202205F
:109E100083F8B92138BD94F82830082B30D00120C0
:109E200038BD00212046FFF717FF012845D1042047
:109E300084F83400DCE7D4E90B01FFF795FD012835
:109E40003BD10320F4E74FF0FF31206BFFF78CFD8F
:109E5000012832D1E36A002BF3D00220E8E7184D45
:109E600004F130010120D5F80C220232FFF7A0FDE9
:109E7000012813D00238C0B201281ED80520D7E728
:109E80000023012084F82830CAE7002301220220A1
:109E900084F828300A4B83F8B921BBE7E368D5F88A
:109EA0001412226B03EB4123C5F81822C4E90332D4
:109EB000E36A002BBCD16262BAE7002038BD00BF64
:109EC000A05D0024F8B5044694F83830032B4BD835
:109ED000DFE803F021180B0200212046FFF7BCFE4B
:109EE000431EDBB2012B40D9F8BD0120626B04F1A7
:109EF0003001FFF7E9FD01284FF00303F0D184F8AA
:109F00003830E1E700211E48FFF7A6FE01284FF098
:109F10000203F4D0E4E71B4BE6681A78D3F8141276
:109F2000032AD3F87C51D3F8980114BF4FF4807200
:109F30008022206102FB01F1871A0244A5EB412532
:109F400006EB4126E660C3F87C51D3F88051C3F894
:109F50009821A5EB4121C3F88011E36AC4E90C0202
:109F60005BB960620123CAE7022094F82830062B0F
:109F7000BAD1002384F82830F8BD2763F2E700BF88
:109F8000145F0024A05D00244368C3F308020A4460
:109F9000B2F5007F2DE9F041054682B00C4605D2AE
:109FA00023446B60012002B0BDE8F08190F91A20D3
:109FB000501C09D04449023201EB0212D17A21F03F
:109FC0000101D172FF22AA7695F91B20511C13D0F2
:109FD0003D4E023206EB0211C97AC1F34501012957
:109FE00041D9013901F03F0106EB0212FF26D07A78
:109FF00061F34600D072EE762A78022AD0D0324E33
:10A00000D6F81422B4EB422F4FEA42282DDCD6F8C2
:10A010001C721F407A42A24227DCE219286942459D
:10A0200013D32A7E12072BD5D6F89821411C8A42D9
:10A030001DD300D100214344A4EB08086861084601
:10A04000DB1B08EB070429616B600028AAD032787B
:10A05000032A33D080B24FF6F7729042A2D81A4644
:10A0600014446C609EE70021BEE700209BE796F851
:10A07000B82102BB012386F8B83173706B68DAE748
:10A0800001A96BF02FF80128EFD16B68A4EB08044D
:10A0900028699844297868613C44A8EB0703019833
:10A0A00002291A466B602861CFD1D6F82412B3EB8F
:10A0B000412FD5D376E701227270BCE7034A904264
:10A0C0003FF670AFCBE700BFA05D0024F7FFFF0FA6
:10A0D0002DE9F0474FF0010882B0044694F838307B
:10A0E000032B00F2A580DFE803F055170C020020D7
:10A0F000236C84F8280003B19847022002B0BDE821
:10A10000F0870022236C84F828200BB12046984762
:10A11000012002B0BDE8F08723786768022B03D0E6
:10A12000444BD3F81C321F40C7F34F272046FFF79C
:10A13000F9FA404E3F1A0546BFB207EB050C022262
:10A1400001A9002328461FFA8CF9FFF709FB012813
:10A150004FF400724FF00001D0D1019878F0B6FFB3
:10A16000E3694FF4007120460BB16368EBB1D6F898
:10A1700014325A1E914547D20135FFF705FF0028DA
:10A18000DBD196F8B83113B9012386F8B83186F8D7
:10A190000180D2E72046FFF729FE012802D00228DD
:10A1A00046D1032084F8380098E7019B4FF0203215
:10A1B0004FF0100E4FF02E0C42F62E6AC3F801201D
:10A1C000C3F80520A3F8092083F800C0D4F824C000
:10A1D000A3F820A083F80BE0C3F82220C3F82620C0
:10A1E00083F82A20E26BA3F81AC02CFA0EFC5A87D7
:10A1F00022FA0EF2A3F814C09A8683F82BE0D6F860
:10A2000014325A1E9145B7D3C3EBC35320465902AB
:10A2100001F50071FFF7B8FE20B996F8B8311BB10F
:10A22000012373700220BDE7012386F8B831F7E7F8
:10A23000002063E7A05D0024B1F904300F2B2DE965
:10A24000F0410D4682B00446164631D02046FFF755
:10A2500069FA94F91B80B8F1FF3F3AD0584F07EBE9
:10A260000813DB69984211D097F8B831002B6BD0F6
:10A2700001237B702378022B5CD02269002A71D1E4
:10A2800000230120336002B0BDE8F081B96901EB21
:10A290004821002964D0AB88204601331BB201EB72
:10A2A0004311AB803160FFF73DFA28600120EAE7F7
:10A2B0004FF40071FFF768FE002841D04FF6FF739E
:10A2C0002046AB80FFF72EFA94F91B80B8F1FF3FD0
:10A2D000C4D12378022B3BD02269002AD0D0384F3A
:10A2E0003B78032B62D093B24FF6F7718B4294BF49
:10A2F00000230123002BC1D128B997F8B831002BD6
:10A3000047D001237B700023112201A9FFF728FA0F
:10A31000012825D10199BB69CB1A48BF03F2FF136D
:10A32000B3F5805F4FEA63222AD24FFA82F884F8AD
:10A330001B80AEE7D7F824226368B3EB422F9FD28D
:10A34000002002B0BDE8F081012387F8B8318FE723
:10A350001B4F6368D7F82422B3EB422FCCD38FE78F
:10A36000237888E73B78032B17D093B24FF6F77228
:10A37000934294BF00230123002B81D10020E0E70A
:10A3800097F8B83113B9012387F8B83101237B70EE
:10A39000CDE7012387F8B831B3E70A4B9A4294BF5F
:10A3A00000230123002B7FF46BAFE7E7054B9A42B4
:10A3B00094BF00230123002B7FF460AF9CE700BF14
:10A3C000A05D0024F7FFFF0F70B50378044690F8F6
:10A3D00018C0023B012B02D91CF0060F66D11CF0FD
:10A3E000200F3FD194F91A30591C09D0364A023354
:10A3F000FF2102EB0313DA7A22F00102DA72A1766E
:10A4000094F91B305A1C13D02F48023300EB03126F
:10A41000D27AC2F34502012A45D9013A02F03F023D
:10A4200000EB0313D97A62F34601FF22D972E27678
:10A430001CF0080F0DD0244890F89C31072B05D054
:10A4400090F8B831002B39D001234370002380F8F5
:10A450009C310023E26A237084F828302AB3BDE8D7
:10A460007040104718480023E5690246D169103250
:10A470008D4206D00133082BB4D0D16910328D4201
:10A48000F8D1023300EB0312D27AC2F34502012A5B
:10A4900018D9013A02F03F0200EB0313D97A62F3B4
:10A4A0004601D9729EE70022BAE770BD0121FFF78D
:10A4B000D3FB0128F9D194F818C090E7012380F864
:10A4C000B831C1E70022E7E7A05D002438B5194C98
:10A4D00094F8E4312BB970B190F828201AB11846DD
:10A4E00038BD002038BD0146442204F5DE7076F008
:10A4F0006FFD012038BD04F5DE7501464422284673
:10A5000078F0E4FD237803224FF6FF71022B2846F2
:10A51000A4F8D61118BF1346D4F8201284F8D42119
:10A52000102284F8BC31C4F8E01184F8D5216CF015
:10A5300063F8DEE7A05D0024F8B54FF0FF312C4C46
:10A54000002322460D4603E001331032082B14D0BD
:10A5500092F82A000428F7D104EB031090F82B009E
:10A56000C707F1D46E1C106A01D08142ECD91D4698
:10A57000013301461032082BEAD1002D01DA012007
:10A58000F8BDAE1CD4F8D02504EB06131989D1B957
:10A590002F012744A169D4F8D035F86901EB452192
:10A5A000CBB1DD680023134AA847A0B1022808D127
:10A5B000D4F8A03004EB06160122013BB272C4F8B5
:10A5C000A0300020F8BD04EB05132F01D86912B1AB
:10A5D00093689847DDE7D4F8A03004EB0616032112
:10A5E0000122013BB17284F8A420C4F8A030E8E74E
:10A5F000A05D0024C57B0408704700BF10B54FEA7A
:10A60000511E024400EB8E0C624529D901F01F0354
:10A610004FF0FF3450F82E1004FA03F30B4093FA76
:10A62000A3F3B3FA83F3DBB2202B16D10CF10401B0
:10A630008A4202D817E08A4212D98C460431DCF8EB
:10A64000003093FAA3F3B3FA83F3DBB2202BF2D0FA
:10A65000ACEB000C03EBCC0010BD03EB4E1010BDB7
:10A660004FF0FF3010BD204610BD00BF03694168A8
:10A6700053EA0102F0B43B4E5DD0C56A013390ED60
:10A68000067A6A1C876830EE077A0361012AC26283
:10A6900080ED067A42D090ED075A07EE902AD0ED71
:10A6A000096A70EE455A3468B8EEE76A611AC5EE79
:10A6B000867AB94277EE857A30EE670AC0ED087A7D
:10A6C000C0ED077AF0EE667AE5EE807AC0ED0A7AA0
:10A6D000C0ED097A01D8F0BC7047012A28DD06EEEA
:10A6E000905AF8EEE66A87EEA66AB5EEC06AF1EE19
:10A6F00010FA1DDBF1EEC67AF4EE677AF1EE10FA8D
:10A7000016D6D0ED056AF4EEE76AF1EE10FA15D52B
:10A71000037BFBB10323F0BC03707047326880ED0C
:10A72000080A521A002180ED070ABA424162D2D9C2
:10A73000DFED0D7AE5E7316841609EE707EE903A7C
:10A740000223F8EE677A0370F0BCC7EE276AC0ED0B
:10A75000066A7047316800220361C362416082610A
:10A76000B9E700BF0C3300240000000010B5DFED96
:10A770004F4A844600F1480E0346DA6AB1EC017A8A
:10A78000D3ED067A013277EE877A012ADA62C3EDD9
:10A79000067A71D093ED075A07EE902A93ED096A75
:10A7A00077EE455AF8EEE77AC5EEA76A76EE857A37
:10A7B000F0EE466A37EE677AC3ED087AE5EE876A0F
:10A7C000C3ED0A6AC3ED077A1833C3ED036A734514
:10A7D000D3D1374C416822680369521A816801332A
:10A7E0008A42036147D990ED056A0022DFED2F5AB6
:10A7F000DCF82C10F0EE657ADCED0A6A012901F133
:10A80000FF3E11DD07EE90EAF8EEE77A86EEA77AD2
:10A81000B5EEC07AF1EE10FA45DBF1EEC77AF4EE50
:10A82000677AF1EE10FA3ED6B4EEE76A01320CF127
:10A83000180CF1EE10FA26D4022AD9DDB4EEE76A3C
:10A84000F1EE10FA1FD407EE903AD0ED066A90EDC3
:10A850000C7A0223F8EE677AD0ED125A037086EE76
:10A86000A76AC7EE276A85EEA77A80ED066AC0ED73
:10A870000C6A80ED127A10BDF0EE477A83ED087A0B
:10A88000F0EE646A9EE7037B13B10323037010BDEF
:10A89000002221680361C3624160826102634364F4
:10A8A0008264C36510BDDFED017ABDE700000000E2
:10A8B0000C330024B0EEC06AF0EEE05AF0EE407ABD
:10A8C000F4EEC65AF1EE10FA0EDCB5EE400AF1EEE7
:10A8D00010FA4AD0F4EEC65AF0EE466AF1EE10FADB
:10A8E0004FD5B0EE655A03E0F0EE656AB0EE465A19
:10A8F00085EE267A9FED242A9FED243A9FED244A87
:10A90000DFED244ADFED242ADFED243AB7EE005ACA
:10A91000DFED236AF4EEC65AF1EE10FAA7EE023A22
:10A92000E7EE223AA7EE034AA7EE235AE7EE044ADF
:10A93000E7EE246AB1EE667A87EE050A10D4F5EEEA
:10A94000C00AF1EE10FA03D59FED167A37EE400AF1
:10A95000F5EEC07AF1EE10FA48BFB1EE400A70474A
:10A960009FED117A37EE400AE9E7F5EEC00ADFED18
:10A970000F7A9FED0F0AF1EE10FA58BFB0EE670A9A
:10A980007047B0EE465AB3E739094E3DE3B59EBE77
:10A9900088FA16BE45FE7FBF99FB243F69A2163E8A
:10A9A000A7DFA8B4DB0F4940DB0FC93FA7DFA834FE
:10A9B000DA0F4940D1ED007AF7EE002AD0ED043AE3
:10A9C00090ED054AE7EEA73AD0ED064A90ED075A1A
:10A9D000D0ED085A90ED096AD0ED0A6A90ED0B7A35
:10A9E000C0ED043A91ED003AD1ED013AD0ED0C7A88
:10A9F000A3EE234A80ED054AD1ED003A91ED024ADB
:10AA0000E3EE844AC0ED064AD1ED004A35EE245A01
:10AA100080ED075AD1ED014A91ED005AE4EE855AD6
:10AA2000C0ED085AD1ED015AA5EEA56A80ED096A7C
:10AA3000D1ED015A91ED026AE5EE866AC0ED0A6A2F
:10AA4000D1ED016A37EE267A80ED0B7AD1ED026AFC
:10AA500091ED007AE6EE877AC0ED0C7A91ED027AFC
:10AA6000D1ED017A90ED0D3AD0ED0E3AA7EE273AEE
:10AA700090ED0F4AD0ED104A90ED115AD0ED127AB8
:10AA8000D0ED135A90ED006A80ED0D3A75EEA25AA2
:10AA900091ED023AD0ED016AE3EE033A90ED027ACD
:10AAA000C0ED0E3AD1ED023A34EE234A80ED0F4A62
:10AAB00091ED004A74EE844AC0ED104AD1ED014A8E
:10AAC00035EE245A80ED115A91ED025AC0ED135A19
:10AAD00077EE857AC0ED127AD1ED017AD1ED005A88
:10AAE00067EEA77A91ED025AE5EEA57AE5EE057AD2
:10AAF000A5EEA76A80ED006A91ED016AE6EE276A8D
:10AB0000C0ED016AD1ED026AA6EEA77A80ED027A65
:10AB100090ED037A77EE277AC0ED037A704700BF95
:10AB20002DE9F04F4FF00009864600F1100506466A
:10AB3000034689B000F13008074648462C468B464C
:10AB40009C46B246CDF80CE000283CD10CF1040C38
:10AB5000A445FBD1032800F1010151D09C46AA462F
:10AB6000029398B1DCED047AAAEB0903B646019290
:10AB70007246F3EC016A0EF1100E92ED007A534525
:10AB8000E6EEC77ACCED047AF2D1019ADCED046AE4
:10AB90000CF1100C15ED047A0AF1100AC445C6EE4A
:10ABA000877ACCED007ADCD1029B0436084608F1A6
:10ABB0000408143314351034103709F104099C4685
:10ABC000B2460028C2D0DCED007AD6463946019262
:10ABD0007246F1EC016A0EF1100E92ED007A994284
:10ABE000E6EEC77ACCED007AF2D10CF1040C019AB2
:10ABF0000AF1040AA445E6D1032800F10101ADD110
:10AC0000DDF80CE00023594604AD76467746002077
:10AC10000493059306930793F2EC017AE5EC017A2D
:10AC2000B0B104AC3B46B4EC017AF3EC016AE6EE59
:10AC3000C77AB34245ED017AF5D1013004280BD033
:10AC4000F2EC017A10371436E5EC017A0028E8D1ED
:10AC5000103714360120DFE708AD10310EF1400E39
:10AC6000042875ED017AA1F10402744641ED017AE0
:10AC70001ED07346F3EC016AB1EC017AA342E6EE12
:10AC8000C77AC2ED007AF5D15EED016A013887EE30
:10AC9000A67A82ED007A17D0AEF1140E103C114660
:10ACA00075ED017A0428A1F1040241ED017AE0D1A9
:10ACB0005EED016A103CAEF1140E032087EEA67A19
:10ACC00001ED017A1146EBE709B0BDE8F08F00BF56
:10ACD00060EEA00AE0EE000AF5EEC00AF1EE10FA0E
:10ACE00007DBB1EEE00AB4EE400AF1EE10FA00D64E
:10ACF00070479FED010AFBE70000000060EEA00A2C
:10AD0000E0EE000AE1EE010AF5EEC00AF1EE10FAFB
:10AD100007DBB1EEE00AB4EE400AF1EE10FA00D61D
:10AD200070479FED010AFBE700000000DFED297A84
:10AD3000B4EEE70AF1EE10FA28DD9FED277A30EE47
:10AD4000470AB4EEE70AF1EE10FAF8DCDFED237AF9
:10AD5000B4EEE70AF1EE10FA2FDD30EE670A37EEB7
:10AD6000C00A60EE007ADFED1E5A9FED1E6ADFED2D
:10AD70001E6AA7EEA56A9FED1D7A60EE275AE7EEE0
:10AD8000866AA7EEA67AA5EE870A7047DFED187AE5
:10AD9000B4EEE70AF1EE10FAD8D59FED0F7A30EE57
:10ADA000070AB4EEE70AF1EE10FAF8D4DFED0B7AF9
:10ADB000B4EEE70AF1EE10FACFDC9FED0E7AB4EEB6
:10ADC000C70AF1EE10FACCD530EE270A37EE400A6A
:10ADD000C7E700BFDB0F4940DB0FC940DB0FC93FAE
:10ADE0009A7C2E36FAAF4FB93587083CA4AA2ABE02
:10ADF000DB0F49C0DB0FC9BF10B5404CB4FBF2F408
:10AE0000A14219D3DFED3E7AF7EE005AB0EE677A31
:10AE1000B0EE676AF0EE676A0023C0ED005AC0ED3D
:10AE2000017A80ED027A80ED036AC0ED046A8361E5
:10AE300043610362C36110BD07EE902ADFED315A12
:10AE4000B7EE006ADFED306AB8EE677A07EE901A67
:10AE5000B0EE405AF8EE677A27EE257A67EEA67ACA
:10AE6000C6EE076AC7EEA64AFDEEE47A17EE902A10
:10AE70002032402A3FD8B0EE640AFFF757FFB0EE09
:10AE8000404ADFED227A34EEA70AFDEEC07A17EED3
:10AE9000902A2032402A29D8FFF748FFF8EE006AAE
:10AEA00060EE266A012B1CD0B7EE006AF6EE004A6F
:10AEB00036EE406A66EE244A35EE055AF7EE007A21
:10AEC00084EE057A77EE275A37EEC75A84EEA57AD4
:10AED000C6EE257A86EEA56AC5EE256AF0EE475ADB
:10AEE0009AE7F7EE004AB0EE666AE5E7DFED086A3A
:10AEF0009FED030AD6E79FED024AC2E720A10700B3
:10AF000000000000BD378635DB0FC940DB0FC93FAD
:10AF100000000080DFED077A30EE270AFDEEC07AF0
:10AF200017EE903A2033402B00D8FFE69FED020A3F
:10AF3000704700BFDB0FC93F000000002DE9F84F4C
:10AF40009DF828408946DDF82CB00546002C1746B0
:10AF50001BF8011B0CBF4FF020084FF030081C1EDF
:10AF600008463ADB00295CD0002C53D04FF0000A91
:10AF70005B4600E064B313F8016B013C002EF9D18D
:10AF8000BAF1000F2FD1264644B14D45414628461F
:10AF900000D2B847013CF8D10B9B18780146A0B10C
:10AFA0004FF0FF344FF0000A00E09B464D45284625
:10AFB00000D2B8475B4613F8011B0029F5D10B9B63
:10AFC000F61A5E44BAF1000F10D13046BDE8F88F92
:10AFD000BAF1000F1BD15646E0E7634229B31C4685
:10AFE0004FF0010AC4E70028E0D10646002C04F126
:10AFF000FF3AEADD54464D454146284600D2B8475F
:10B00000013CF8D2013656443046BDE8F88F30B1E5
:10B010002646CBE726464FF0FF34B246C6E7064643
:10B02000D3E72646002CB0D1CFE76FEA040A0E46DC
:10B03000E0E700BF0FB430B583B00C4C06ABD4F8DA
:10B040005018D4F84C0853F8042B01936CF078FE98
:10B050000546D4F8D40503685B6998470028F8D002
:10B06000284603B0BDE8304004B07047A05D00241E
:10B070000EB410B583B00446084905AB01A853F8D7
:10B08000042BCDE900346CF05BFE0022019B1A70AA
:10B0900003B0BDE8104003B0704700BF457E040810
:10B0A0000CB4F0B53C4CADF5277DD4F85438002BEA
:10B0B0006DD094F85C3899420BD90123D4F86028FC
:10B0C0008340134205D10DF5277DBDE8F04002B065
:10B0D0007047324B4FF47A71314A1B68A2FB03026E
:10B0E00006A8920901FB12332E49FFF7C1FF06ABF8
:10B0F000AC9A064603442C4901A80193ADAB0093DA
:10B100006CF01EFE019B0A2100225D1C0195197046
:10B11000019BD4F85458591C01911A70ADB12B6899
:10B120005B6A1BB128469847D4F854589DF818100C
:10B130000029C8D00DF119042B6828461B689847D0
:10B1400014F8011B0029F7D1BDE7D4F85878002F77
:10B15000B9D0304426ABFD2206A9841C1846ADF8B0
:10B1600010202246CDF81250ADF8165075F030FF81
:10B1700002220346044402A93846CDE9023433F0E2
:10B180002DFF0DF5277DBDE8F04002B07047D4F8E3
:10B190005838002B8DD196E7A05D00240C33002495
:10B1A000D34D6210F4EC0C08397E0408194A0330C0
:10B1B00010B5D2F8644804EB9003B3F5007F19D8BA
:10B1C000C2F8643802F6680220F00300C3F5007389
:10B1D00002EB8404104A9B0002EB810151F8902C91
:10B1E00010440E4A41F8900C04210020FFF758FF4C
:10B1F000204610BD00210A4A00240846FFF750FFF0
:10B20000054A204652F8083C43F0007342F8083CD7
:10B2100010BD00BFA05D0024986E002400ED0C0856
:10B2200024ED0C0803685A1C02601878704700BFB0
:10B2300003681A46591C016012F8021B0260587814
:10B2400041EA0020704700BF02681346511C0160AC
:10B2500013F802CB0360D31C5178036093781B046E
:10B2600043EA0123111D43EA0C030160D07843EA4D
:10B270000060704712B370B50446864604E0981B20
:10B2800017D114EB0C0C15D01EF8013BA3F14100B3
:10B29000A2EB0E0C192811F8010BA0F1410598BF83
:10B2A000203300F12006192DE9D91B1A04D10028FA
:10B2B000E7D170BD604670BD184670BD104670473E
:10B2C00003880021194A30B503F0030E90F802C03C
:10B2D000174CA3F5FA630EEB4E0E0CF1FF3C40F257
:10B2E000B5550CEB8E0C04EB4C044FEA930C238AFF
:10B2F000847905FB0C3390F803C022444FF47A7430
:10B300000CF1FF3C634490F804C003EB43030CEBE7
:10B31000C30C43790089CCEB0C1C03EB8C03C3EB0F
:10B32000031302EB8302C2FB040130BD80436D387E
:10B3300030470C08F8B516461F463F4D04463946BF
:10B3400030464FF47A72002370F0ECF93B4B054421
:10B350003B4F3C4E83FB0510E9172844C1EB6011BD
:10B3600083FB0103C8170B44C0EB631087FB003C51
:10B37000C317C3EBAC0386FB03764FEAE37ECEEB49
:10B38000E61EC1EB0116A5EB860CC0EB00154FEADB
:10B390008E0684F806C0A1EB8501617103EB4301C1
:10B3A000A0EBC10040F2B55101FB1E332071B3F593
:10B3B000896F35DA40F2DA218B4237DCB3F5B77F9B
:10B3C0002149B4BF4FF0000E4FF0010E0EEB4E00BE
:10B3D00075464FEA4E0701EBC001C88C1B4907EBCD
:10B3E0000E0C01EBCC0C0B210CF1160C01E03CF81F
:10B3F000020D984211DD0139F9D17744124901EB70
:10B40000C701088A012106F5FA6E0133A17075445F
:10B410001B1A22812580E370F8BD0131C9B2F2E721
:10B42000032540F296500627AE46D7E7022540F2A4
:10B4300029400427AE46D1E780BC92C78988888816
:10B44000ABAAAA2A73B06D1630470C0840470C0807
:10B4500030B5304C8DB086460D46EC461EF0030FDD
:10B460000FCCACE80F000FCCACE80F0094E80F0055
:10B470008CE80F000FD1284B284A03FB0EF3B2EBE8
:10B48000B30F44D3264AB2EB331F34BF012200224C
:10B49000C2F11D0200E01C220EF1FF33019240F2C6
:10B4A0006D122048002B194602FB0EF21E4CB8BF4D
:10B4B0000EF10201EE4602EBA10280FB0310DB1746
:10B4C000ADF1040101EB8501A3EB6015C3EBE013C3
:10B4D0002A441A44253284FB0230D3171044C3EBAC
:10B4E000A003C3EBC303D31A5EF8040FC21871455F
:10B4F00084FB023C4FEAE2739444C3EBAC03C3EB1E
:10B50000C303A2EB0303EFD1C01A0DB030BD1D225F
:10B51000C2E700BFA0470C08295C8FC2285C8F02DD
:10B520000AD7A3001F85EB51932449920D4B10B508
:10B53000D3E9004354EA03020AD10146002340F252
:10B54000011218460B80C1F802208B710B8110BDCF
:10B55000054A1268121943F10003FFF7EBFE0120C0
:10B5600010BD00BF986E00240C33002430B5134D7D
:10B5700083B00446D5E9001351EA03020AD100233F
:10B5800040F2011218462380C4F80220A3712381DF
:10B5900003B030BD0A4A1268521843F10003FFF7A6
:10B5A000C9FE2B8920460DF106022146ADF8063072
:10B5B00069F0F8FC012003B030BD00BF986E002494
:10B5C0000C3300242DE9F047044688B094F830305D
:10B5D000042B11D8DFE803F04C135D035600237EE3
:10B5E0009A0640F1F0800023112204A9E069FEF7D9
:10B5F000B7F8012800F0E78008B0BDE8F087C94D32
:10B6000003AE04F11C0705F5DE793246394648469B
:10B61000FEF712FE012800F0F1800228ECD195F926
:10B62000D6315F1C09D00233FF2205EB031385F8E6
:10B63000D621DA7A22F00102DA7295F9D7315E1C4E
:10B6400014D0023305EB0312D27AC2F34502012A69
:10B6500040F25081013A02F03F0205EB0313D97A20
:10B6600062F34601FF22D97285F8D721042306E050
:10B67000AD486AF0C1FF4FF6FF720123228484F8BF
:10B680003030A3E70020E36A207008B0BDE8F0473F
:10B690001847A44D95F8E431002BADD104F11C07F7
:10B6A00003AE05F5DE78324639464046FEF7C4FD66
:10B6B000012840F00D81039B002B00F0E8801A78F0
:10B6C0000AB1E52AEFD1AA699A1A48BF02F2FF121D
:10B6D000B2F5805F4FEA622180F041810901934A0F
:10B6E0000A44917B04290CD0D5F89C100131C5F88F
:10B6F0009C10516004219173D5F8A0200132C5F847
:10B70000A02095F9D621501C09D0023205EB021277
:10B71000D17A21F00101D172FF2285F8D62195F965
:10B72000D721511C14D0023205EB0211C97AC1F3A2
:10B730004501012940F25681013901F03F0105EB35
:10B740000212FF2085F8D701D07A61F34600D0724B
:10B7500020220021184677F0B9FCD4F831100346B6
:10B76000D4F8352005A819605A6094F83B20B4F845
:10B7700039109A721981627E0193DA72FFF7F6FE30
:10B78000019B002800F0D4809DF816009DF817203A
:10B790009DF8191042EA4012BDF814004901A0F2C8
:10B7A000BC7042EA40229DF81A0041EA50019DF81F
:10B7B000180092B241EAC02188B2D9811A821A8354
:10B7C000D88203235BE720466AF016FF2369002B2B
:10B7D00000F08380237E03F0F70213F00403227647
:10B7E00040F08A80122A00F0A6800022E36A2046F8
:10B7F00084F8282008B0BDE8F0471847DDF80C8031
:10B80000B8F1000F00F0B68098F80030002B00F07F
:10B81000B18098F80BA01AF0080F7FF4F6AE0B2257
:10B8200004F13101404676F063FF00287FF4EDAE6D
:10B83000637E8AEA0303DF0640F1D88095F9D631AA
:10B840005E1C09D00233FF2105EB031385F8D611E6
:10B85000DA7A60F30002DA7295F9D721511C3FF4CD
:10B8600005AF023205EB0213DB7AC3F34503012B6C
:10B8700040F2FB80013B03F03F0305EB0212D17A5B
:10B8800063F34601FF23D17285F8D731EEE695F8D0
:10B89000BC310922022B3FF4E9AE95F8E431002BCC
:10B8A0007FF4E4AE85F8F43185F8F0311E4885F870
:10B8B000E421C5E97E33D5F8D031C5F8E831D5F8B3
:10B8C0001832C5F8EC31FEF703FC01283FF4EBAE6B
:10B8D00002287FF491AE0423D1E6237E1B0784D592
:10B8E000104B93F89C21002A7FF486AE072283F840
:10B8F0009C217AE70022B0E60023A5682046E66A8C
:10B90000294684F82830FEF73FFB002864D194F8DC
:10B910002830002B7FF470AE0223C4E90B6584F855
:10B92000283069E6A05D00245C5F0024BC5D002433
:10B9300044F2817242E7E06A0421626AA063204611
:10B9400084F83C3084F8281063636362C4E90B22F6
:10B95000C4E9023308B0BDE8F0476AF04DBE95F87F
:10B96000B82112B9012285F8B82101226FF00F0128
:10B970006A70B4E695F9D631591C09D00233FF221A
:10B9800005EB031385F8D621DA7A22F00102DA7288
:10B9900095F9D7315A1C13D0023305EB0312D27A32
:10B9A000C2F34502012A1FD9013A02F03F0205EB1A
:10B9B0000313D97A62F34601FF22D97285F8D721A1
:10B9C000237EDB067FF552AE2A486AF015FE4FF65D
:10B9D000FF720223228452E6002E3FF40DAE204671
:10B9E000334652E60021AAE60022E0E7B8F8142028
:10B9F000B8F81A3043EA0243D5F8142263625202BF
:10BA0000D8F81C30B3FBF2F102FB1131A36009B18D
:10BA100013445B1AE36084F819A095F9D6315A1CD7
:10BA200009D00233FF2205EB031385F8D621DA7A19
:10BA300022F00102DA7295F9D721531C3FF4C1AE0E
:10BA4000023205EB0213DB7AC3F34503012B0ED957
:10BA5000013B03F03F0305EB0212D17A63F3460189
:10BA6000FF23D17285F8D731ABE6002305E7002329
:10BA7000F1E700BF5C5F00242DE9F04390F8283027
:10BA800083B00446013B082B0BD8DFE803F0393DB7
:10BA90001F24052A0A2F34000121FEF719F9012875
:10BAA00002D003B0BDE8F08300222378216C84F833
:10BAB0002820002BF5D00322E162D4E9010384F8A9
:10BAC0002820834238BF03462046A36003B0BDE868
:10BAD000F043FEF779BC002103B0BDE8F043FEF768
:10BAE000F7B803B0BDE8F043FEF7ECB903B0BDE82A
:10BAF000F043FEF77BB903B0BDE8F043FEF7E8BAC8
:10BB000003B0BDE8F0435DE5DFF830914368D9F854
:10BB10001C62026B19461E40D9F8140294F800C04A
:10BB2000B5184702B5EB402F41D34FF6F778BCF17B
:10BB3000020F14D025692846002D5AD16168A368E8
:10BB40000020E26A8B4284F8280038BF0B46A360CD
:10BB5000002AA6D0204603B0BDE8F0431047616834
:10BB6000D9F82402B1EB402F5CD22069217E09076D
:10BB700032D5D9F89811451CA9422AD299F8B811A2
:10BB8000002943D1012389F8B83189F80130226BAB
:10BB9000636894F800C0D21B3B4432449B1B0026D0
:10BBA0009742194663602263C4E90450BFD9BCF1CF
:10BBB000020F37D02569002DC1D099F80030032B32
:10BBC00036D0ADB24FF6F7739D42B8D811446160DC
:10BBD000B5E7E0D10025DEE701A969F083FA012885
:10BBE0007FF45FAF2069019D94F800C06368226B09
:10BBF000D1E799F8001003290ED0A9B2414594BFAE
:10BC0000002101210029B1D06168D4E7012189F820
:10BC1000011094F800C0BEE707498D4294BF00218F
:10BC20000121EFE7D9F82432B1EB432FCED386E7D9
:10BC3000014B9D4283D8C9E7F7FFFF0FA05D0024A9
:10BC400088422DE9F04198464FF0010439D301FBB9
:10BC500004F4B0FBF4FC8C45F9D264B30025BCF1CC
:10BC6000000F04FB1C00B4FBF1F7D4BF0026012633
:10BC70006DB966B9A142354619D9C6460CF1300CEA
:10BC80000EF801CB00238EF80030BDE8F081BCF146
:10BC9000090F18DD002A0CBF57233723C64663441B
:10BCA000A14205F101050EF8013BF046EAD83C46F9
:10BCB000B0FBF7FCD3E7C64600238EF80030BDE8A2
:10BCC000F0818446CAE73023E8E700BF2DE9F04160
:10BCD0000446154608469442B4FBF2F607D205FB2B
:10BCE0001644134B1B5D00F8013BBDE8F081964202
:10BCF000B6FBF2F70CD20E4B05FB176705FB16449B
:10BD0000DA5D1B5D00F8012B00F8013BBDE8F08116
:10BD1000BA42B7FBF2F807D905FB1878044B13F8C1
:10BD2000082000F8012BE7E74046FFF7CFFFF3E7D5
:10BD300034ED0C08B5EEC00ADFED357A0023F1EEE4
:10BD400010FA30B5C8BF30EE270A87B0D8BF30EE42
:10BD5000670ADFED307A054603A9029320EE270A31
:10BD6000CDE90033FDEEC07A17EE904A84EAE47024
:10BD7000A0EBE4706AF0D2F9002C03A8B4BF2D2325
:10BD800020238DF800306EF0B3FE01282AD002285F
:10BD900034D003281ED003A9684678F011F968460C
:10BDA0006EF0A6FE044669462846033CE4B22246ED
:10BDB00075F00EF9002328462B556EF099FE2E22C1
:10BDC000431C0DEB04012A54E81878F0F1F82846DA
:10BDD00007B030BD302303A968468DF8013078F0F4
:10BDE000EFF8DCE743F23002302303A96846ADF8F0
:10BDF00001208DF8033078F0E3F8D0E743F2300308
:10BE000003A96846ADF8013078F0DAF8C7E700BF5B
:10BE10006F12033A00007A440378202B03D110F804
:10BE2000013F202BFBD0092BF9D02D2B63D02B2BDE
:10BE3000B7EE000A08BF01300278A2F13003D9B290
:10BE4000092961D8F2EE046ADFED4D7A07EE103A67
:10BE500010F8012FB8EEC77AA2F13003D9B2A7EEDD
:10BE6000A67A0929F0EE477AF0D92E2A50D0037825
:10BE700003F0DF03452B3BD110B442782D2A73D059
:10BE80002B2A62D0A2F130030130092B63D80024A1
:10BE9000002303EB830302EB430310F8012FA2F10D
:10BEA0003001303B0929F4D9B3F59A7F1A46B7EE31
:10BEB000007A28BF4FF49A72072B09D91346DFED99
:10BEC000316A083B27EE267A072BFAD802F00702E0
:10BED0002AB1F2EE046A013A27EE267AFBD1002C51
:10BEE0003BD0C7EE877A5DF8044B20EE270A7047F7
:10BEF00020EE270A704742780130BFEE000AA2F117
:10BF00003003D9B209299DD92E2ADFED1D7AAED191
:10BF100043780130A3F13002D1B20929A8D8B2EE9A
:10BF2000047AF0EE475A06EE902A10F8013FB8EE78
:10BF3000E66AA3F13002D1B2C6EE076A092927EEFC
:10BF4000257A77EEA67AEED992E782780230A2F1CE
:10BF50003003092B9BD9B7EE007A67EE877A5DF83C
:10BF6000044B20EE270A704782780230A2F130039A
:10BF7000092B01D801248BE7B7EE007AB1E700BFA7
:10BF80000000000020BCBE4C0378092B01D0202B00
:10BF900005D110F8013F202BFBD0092BF9D02D2B18
:10BFA00009D001784FF0010CA1F13002D3B2092B76
:10BFB0000AD900207047417801304FF0FF3CA1F1D1
:10BFC0003002D3B2092BF4D8002310F8011F03EB81
:10BFD000830302EB4303A1F13002D1B20929F4D962
:10BFE0000CFB03F0704700BFAA4BAB4A2DE9F04FA2
:10BFF0004FF0000A99B09E1A41F221051F463422E3
:10C0000000210BA877F062F8A34AA44B0892CDE96F
:10C010000976DA68D10707D5A14A5A6002F1883259
:10C020005A60DB68DC070DD49C4BD3F80C21D20797
:10C0300008D59B4AC3F8042102F18832C3F80421D1
:10C04000D3F80C31002101227E2308A8159105A9FF
:10C050008DF858208DF81430FCF7BAFE0028C0F295
:10C06000288108214FF4FC4303E05B0001399BB2B7
:10C0700007D01AB2002AF8DA85EA4202013993B2EF
:10C08000F7D1884AADF81630874B934280F0508143
:10C0900098460DF11809CDE902A7B8F802204FF033
:10C0A000000CB8F80030C2F30B0B10048DF81DC063
:10C0B0000BF10601ADF81810C3F30B014FEA13336F
:10C0C000ADF81A108DF81C3000F191800622494617
:10C0D00008A8FCF77DFE0028C0F2FC80BDF81640E1
:10C0E00049460DF11E0011F8013B082284EA0324A1
:10C0F00003E06400013AA4B207D023B2002BF8DABF
:10C1000085EA4303013A9CB2F7D18842EBD15A4603
:10C11000D8F8041008A8FCF75BFE0028C0F2DA800B
:10C12000D8F8041001EB0B00814215D00139013819
:10C1300011F8013F082284EA032403E06400013A75
:10C14000A4B207D023B2002BF8DA85EA4303013A00
:10C150009CB2F7D18142EBD1ADF8164008F114083A
:10C16000504B984599D3DDE902A7002302224946A6
:10C1700008A8ADF81830FCF72BFE0028C0F2998013
:10C18000BDF816300DF11A0041F2210119F8012B0A
:10C19000082483EA022303E05B00013C9BB207D042
:10C1A0001AB2002AF8DA81EA4202013C93B2F7D1CE
:10C1B0004845EBD102220DF1160108A8ADF8163062
:10C1C000FCF706FE002874DB1498002840F08880F5
:10C1D000159800286DDB9DF85820002A40F09680C5
:10C1E00000280DBF012200220123002363E0E24664
:10C1F0006746019601370622494608A8FFB28DF826
:10C200001D70FCF7E5FD002850DBBDF816404946DF
:10C210000DF11E0011F8013B082284EA032403E01B
:10C220006400013AA4B207D023B2002BF8DA85EA01
:10C230004303013A9CB2F7D18842EBD1D8F80410FD
:10C240005A4608A801EB0A063146FCF7C1FD002852
:10C250002CDB06EB0B00864215D0711E013811F85D
:10C26000013F082284EA032403E06400013AA4B2F7
:10C2700007D023B2002BF8DA85EA4303013A9CB2D7
:10C28000F7D18142EBD1032FDA44ADF81640B1D19A
:10C29000019E63E70000040800000208002000522D
:10C2A000230167452CA60D0878A00D08DDE9016A79
:10C2B000039F012300220AF1010ABAF1020F02DCF6
:10C2C000002B7FF49CAE12B1FBF7CAFD28B9052004
:10C2D00006F020FFDDE902A7EBE719B0BDE8F08F1B
:10C2E000089B099A03449342E3D80CABC0F12002A7
:10C2F0002146184476F0EAFE159818B90CA908A84A
:10C30000F6F754FF00221590149262E70A4AD168AA
:10C3100041F00101D160D168C9077FF561AFD2F862
:10C320000C1141F00101C2F80C11D2F80C2157E7B1
:10C330000DF1180919E700BF0020005270B54588BB
:10C340000B4604460021C5F30B0518462A4676F035
:10C35000BDFE0A4A21690346914206D3084A91422A
:10C3600006D31846BDE8704008470029F9D170BDD2
:10C370002A46BDE8704074F02BBE00BF2CA60D0805
:10C380004BAB0D0890F83C20034602F0FF0012B1C1
:10C39000002283F83C2070474FF40063838170478C
:10C3A000012070470E4B10B40E4C1B6820681B1AFE
:10C3B000FA2B09D809B1A3680B600AB1E3681360CE
:10C3C00001205DF8044B7047074A002113680846B6
:10C3D000217123F004035DF8044B1360704700BF24
:10C3E0000C330024C0EA002494B8002401207047D4
:10C3F000044B0022002101201A615A619A61D9611F
:10C40000704700BFC0EA0024104B11491A68034668
:10C41000C869121AFA2A16D8D1ED046A012091EDE2
:10C42000057AFDEEE66AD1ED067ABDEEC77AFDEE3D
:10C43000E77A16EE902ADA8617EE102A1A8717EE98
:10C44000902A5A8770470020704700BF0C330024A1
:10C45000C0EA00240F4B70B593F8203082B00191F0
:10C46000ABB90D4B1D6895B12B681A687AB19B6802
:10C470006BB104462846984748B1019922462E6878
:10C4800028460B46316802B0BDE87040084702B04C
:10C4900070BD00BFC0EA002400BD00240B4B70B586
:10C4A0001E688EB133681A6872B19B6863B1054625
:10C4B00030460C46984738B131682A462346304604
:10C4C0000968BDE87040084770BD00BF18BD002472
:10C4D000014B5B6A5B681847C0EA0024024B0830D6
:10C4E0005B6A9B68184700BFC0EA002401207047C0
:10C4F00001207047012070470120704701207047DC
:10C5000031B10B4BD3ED0A7AF8EEE77AC1ED007A40
:10C510006AB10749074BC96ADFED076A0B4407EEAA
:10C52000903AF8EEE77A87EEA67A82ED007A7047C5
:10C53000C0EA00244D95FFFF0000C842012070476B
:10C54000012070477B4A014600239446104610B4F0
:10C5500090F904400C30012C4DD00133082BF7D159
:10C56000744C002394F904000C34022858D0013391
:10C57000082BF7D16F4C002394F904000C340328E6
:10C580006BD00133082BF7D16A4C002394F90400D7
:10C590000C34052877D00133082BF7D1654C0023E4
:10C5A00094F904000C34062800F083800133082B32
:10C5B000F6D1002392F904000C32072800F0938092
:10C5C0000133082BF6D15C4B1B68D80340F1A180E6
:10C5D0005A4B086803F58C7403E01433A34200F04F
:10C5E00098801A689042F8D1DA68D201F5D5012016
:10C5F0005DF8044B704703EB43035CF8233023B32F
:10C600004F480B7990F8C94090F8C800984218BF7D
:10C610009C420CBF01200020A2D15DF8044B704762
:10C6200003EB43035CF823308BB146480B7990F859
:10C63000C84090F8C900984218BF9C420CBF012026
:10C64000002097D15DF8044B70473A4C8AE7394C8B
:10C6500094F904000C34032893D103EB43035CF8F2
:10C660002330002B3BD038480B7990F8C84090F825
:10C67000C900984218BF9C420CBF0120002083D102
:10C680005DF8044B704703EB43035CF8233043B37E
:10C690002E480B7990F8C84090F8C900984218BF0E
:10C6A0009C420CBF012000207FF478AF5DF8044B62
:10C6B000704703EB43035CF82330002B3FF47AAF61
:10C6C00023480B7990F8C84090F8C900984218BFE9
:10C6D0009C420CBF012000208AD003466AE7154C1B
:10C6E00054E7144C5CE703EB43035CF82330002B66
:10C6F0003FF469AF174A0B7992F8C90092F8C82045
:10C700009A4218BF98420CBF012000207FF45BAF13
:10C710006EE70B79142B3FF46AAF173BDAB21E2A8F
:10C7200006D80D4B5DF8044BD34003F00100704771
:10C7300000205DE7649D0024686F0024B40300249A
:10C74000EC070024BC0A00248C0D00245C1000249B
:10C750002C130024FC150024010000660B4B8446BA
:10C76000002010B503F58C7E02E014339E450BD0FB
:10C770001A686245F9D1DA68441C8A42F5D0D9605A
:10C780001433E0B29E45F3D110BD00BFB4030024C2
:10C79000704700BF40F2FF72034B914203EBC003AE
:10C7A000A8BF114699867047C0EA0024112807D80F
:10C7B000044B03EB8003D3F890300BB19B681960F6
:10C7C0002CF044BDC0EA0024112807D8044B03EB29
:10C7D0008003D3F890300BB19B681960704700BF9D
:10C7E000C0EA00240C4A13787BB10C4B93F8D810A4
:10C7F00059B193F8D91059B150680022FA2883F83A
:10C80000D920A8BF4FF0FF3070476FF0010070478C
:10C810006FF00200704700BF941B0024C0EA0024A0
:10C820000B4B93F8DA2082B193F8DB2052B109491F
:10C830000022886883F8DB20B0F5967FA8BF4FF010
:10C84000FF3070476FF0020070476FF001007047D3
:10C85000C0EA0024941B0024024BD3F8DC305B6850
:10C86000184700BFC0EA0024024BD3F8DC309B68B5
:10C87000184700BFC0EA0024024BD3F8DC30DB6865
:10C88000184700BFC0EA0024014BD868704700BFBA
:10C89000941B0024044B93F8E03013B1034B186948
:10C8A00070476FF001007047C0EA0024941B002419
:10C8B000014BD3F8E4007047C0EA00244B1EDBB202
:10C8C000062B70B586B03AD81E4A32F813501E4B6C
:10C8D000A3F15804002808BF1C46A44620893CF850
:10C8E000082B4FFA82FE90B1A5EB0E022B1A002AFC
:10C8F000B8BF5242002BB8BF5B429A4202DD644689
:10C900004FFA80FE3CF8080F0028EDD122880F4B2B
:10C910001878A3790593A38804930D4BA67800910A
:10C920000C490396002818BF0B4603210120CDE9CE
:10C930000152094AFEF7B4FB204606B070BD4FF421
:10C940008075C4E784500C08001C00248477002400
:10C950004CF10C08A4070D0850F10C082DE9F0412A
:10C960004FF0B046D6F88050D6F888301D4010D031
:10C97000DFF824800127B5FA85F4C4F11F0458F8C4
:10C98000240007FA04F403689847A543C6F88840D2
:10C99000F1D1BDE8F08100BF706F002438B51446B6
:10C9A000002944D0344B0D469FED344A93ED3A7A3A
:10C9B000D3ED3D6AB8EEC76AB3F90421B8EEE60AD2
:10C9C000D3ED3B7A04EE902AB3F90021C6EE046A57
:10C9D00093ED3E7A05EE902AB3F9022105EE102A76
:10C9E000B3F9FE20B3F9FC30F8EEE44A06EE102A63
:10C9F000F8EEE55AF8EEE77AB8EEC55AB8EEC77A1F
:10CA0000C7EE843A07EE903AB8EEC66AE6EEA45A4C
:10CA1000F8EEE77AA6EE856AA6EEA57AE6EE867AC5
:10CA2000A6EE870AA3EEA70A71F03CFE28600CB3BD
:10CA3000114BF6EE005A9FED115AD3ED3B6AB3F954
:10CA4000F220F8EEE66AB3F9F03007EE102A9FED17
:10CA50000C6A07EE903A86EE850AB8EEC77AF8EED1
:10CA6000E77A20EE070AA7EEA50A20EE060A71F083
:10CA700019FE2060012038BDC0EA00240000F04A01
:10CA80000000C8420B4B03EBC00310B51C6B82B017
:10CA900001916CB107EE901A94ED047A94ED030ABB
:10CAA000F8EEE77AA7EE870A71F0FCFDA36818603C
:10CAB00002B010BDC0EA002470B506680D461446E9
:10CAC000F069A0B3D0F80130CDB1D0F80520B7EEB1
:10CAD000006A9FED1A7A07EE902ADFED195ADFED12
:10CAE000196AF8EE677A77EEC77A77EEA77A87EE5B
:10CAF000A57A77EE467A67EEE67AC5ED007AACB1B4
:10CB000007EE903A9FED107ADFED105AF8EEE77AD3
:10CB10009FED0F6ADFED0F6A67EE877A87EEA57AE1
:10CB200077EE467A77EEA67AC4ED007A70BD0921D9
:10CB30001420FEF73BFBF061C4E700BF9AC9CC4468
:10CB40009AC94C460E76D7450000484300E0FF44A2
:10CB5000000048423393884370B5066882B00D46A2
:10CB60001446F06900284AD0D0F80530F3EE096A7F
:10CB7000DFED265AB2EE047A07EE903A9FED246A72
:10CB8000D0F80130F8EE677A77EEE57A67EE867ACC
:10CB900067EEA67AF4EEC77AF1EE10FA20DCBAEE70
:10CBA000047AF4EEC77AF1EE10FA19D42DB19FEDA4
:10CBB000197A67EE877AC5ED007A7CB107EE903A74
:10CBC0009FED156ADFED156AB8EE677ADFED147A2E
:10CBD000E7EE067A77EEA67AC4ED007A02B070BD71
:10CBE00017EE900A6EF0F0F804460D460D4A042147
:10CBF0000320CDE90045FEF753FA02B070BD0921CC
:10CC00001420FEF7D3FAF061AEE700BF0000004643
:10CC1000000080380AD778430319C83D339388430E
:10CC2000000048C29CF10C082DE9F04105461F4662
:10CC30002848164695F9103082B003EB430350F8AC
:10CC40003380AB689A0716D501230DF106028DF8E3
:10CC5000061040460DF10701F7F7D8FA3B460022CF
:10CC600031464046F7F7D2FAAB689B0718D501204A
:10CC700002B0BDE8F0816B691BB19A881868120494
:10CC80008261154B1868154BC000A3FB0030144B94
:10CC900080095A685C68A4EB020C6045FAD2D3E7BD
:10CCA0000D4A4FF4FA700D4B12680D4900FB02F269
:10CCB0004868A3FB023292094B681B1A9A42FBD2C6
:10CCC0006B69002BD3D01A6801209B88936102B056
:10CCD000BDE8F081540300245C390024D34D621078
:10CCE000001000E010B50446006884B00379012B01
:10CCF0002DD0022B01D0002027E0836802AA13F078
:10CD0000010F4FF0060314BF1F219F21FFF78CFF77
:10CD10000028F0D0BDF80810BDF80A20C9BABDF847
:10CD20000C30D2BA07EE901ADBBAF8EEE76A07EEDB
:10CD3000902AB8EEE77A07EE903AC4ED046AF8EE6E
:10CD4000E77A84ED057AC4ED067A04B010BD8368F5
:10CD500002AA417C03F0010390F9100000921F2207
:10CD600001930623F6F738FFD2E700BF10B504465B
:10CD7000006884B00379012B2DD0022B01D0002054
:10CD800027E0836802AA13F0010F4FF0060314BFD7
:10CD90002521A521FFF748FF0028F0D0BDF8081095
:10CDA000BDF80A20C9BABDF80C30D2BA07EE901A05
:10CDB000DBBAF8EEE76A07EE902AB8EEE77A07EEFC
:10CDC000903AC4ED076AF8EEE77A84ED087AC4ED8C
:10CDD000097A04B010BD836802AA417C03F0010304
:10CDE00090F910000092252201930623F6F7F4FE35
:10CDF000D2E700BF006810B5037984B00C46012B60
:10CE000024D0022B01D000201EE0826812F0010F16
:10CE100003AA14BF1D219D21FFF706FF0028F2D0B1
:10CE2000BDF80C309FED106ADBBADFED106A07EE3B
:10CE3000903AB8EEE77AC7EE067A77EEA67AFDEE7C
:10CE4000E77A17EE903A238004B010BD836803AAF6
:10CE5000417C03F0010390F9100000921D22019320
:10CE60000223F6F7B9FED9E7CFF7534100007A4322
:10CE7000006810B5037984B0012B28D0022B01D0B3
:10CE8000002022E0836803AA13F0010F4FF0030390
:10CE90000CBF83211946FFF7C7FE0028F0D09DF88C
:10CEA0000C309DF90C109DF80D201B0400299DF8F5
:10CEB0000EC043EA02230D4AACBF00214FF07F4170
:10CEC00043EA0C030B43C2F8EC3004B010BD826897
:10CED00003AC0323417C02F0010290F91000CDE97C
:10CEE00000421A46F6F778FED7E700BFC0EA0024F2
:10CEF000006810B5037984B0012B28D0022B01D033
:10CF0000002022E0836803AA13F0010F4FF003030F
:10CF100014BF00218021FFF787FE0028F0D09DF884
:10CF20000C309DF90C109DF80D201B0400299DF874
:10CF30000EC043EA02230D4AACBF00214FF07F41EF
:10CF400043EA0C030B43C2F8E83004B010BD82681A
:10CF500003AC417C032302F0010290F91000CDE9FB
:10CF600000420022F6F738FED7E700BFC0EA0024EF
:10CF700010B50446006884B00379012B43D0022B1E
:10CF800007D0002213461046C4F83620638704B049
:10CF900010BD836802AA13F0010F4FF0060314BFFF
:10CFA00011219121FFF740FE0028EAD0BDF90C20A5
:10CFB000B7EE086ABDF90A3007EE902ABDF90820DD
:10CFC0005B4206EE902AF8EEE77A07EE103AF8EEAA
:10CFD000E66AB8EEC77A67EE867A66EE866A27EE6C
:10CFE000067AFDEEE77AFDEEE66ABDEEC77A17EE49
:10CFF000903A16EE902A1BB2E28617EE102A63874B
:10D00000228704B010BD836802AA417C03F00103AB
:10D0100090F910000092112201930623F6F7DCFD2F
:10D02000C2E700BF10B500230446006884B0C4F80E
:10D03000363063870379012B22D0022B01D00020E8
:10D040001CE0836802AA13F0010F4FF0060314BF1F
:10D0500003218321FFF7E8FD0028F0D0BDF90A3055
:10D06000BDF80810BDF80C205B4201EB410102EB5A
:10D07000420203EB4303E1866287238704B010BDBD
:10D08000836802AA417C03F0010390F9100000922A
:10D09000032201930623F6F79FFDDDE710B54FF05D
:10D0A000000C0446006884B0C4F836C0A4F83AC046
:10D0B0000379012B18D0022B01D0002012E08368E5
:10D0C00002AA13F0010F4FF0060314BF614680213E
:10D0D000FFF7AAFD0028F0D0029ABDF80C30C4F882
:10D0E0003620638704B010BD83686246417C03F03C
:10D0F000010390F910E0019302AB70460093062300
:10D10000F6F76AFDE6E700BF10B5002384B00446D9
:10D1100000680293CDF80B300279012A1ED0022A52
:10D1200019D1836802AA13F0010F4FF0070314BF4F
:10D130004E21CE21FFF778FDBDF80910BDF80B2078
:10D14000BDF80D30C9BAD2BADBBA0120E186228718
:10D15000638704B010BD1A461946F6E7826802AB31
:10D1600090F910C002F00102417C009360460192E8
:10D1700007234E22F6F730FDDEE700BF006810B54A
:10D18000037984B0012B0BD0022B06D1012303AA13
:10D19000FF21FFF749FD04B010BD002004B010BD11
:10D1A000826803AC417C02F0010290F91000009407
:10D1B0000192FF22F6F710FD04B010BD006810B513
:10D1C000037984B0012B2AD0022B22D1826812F07D
:10D1D000010F03AA14BF00218021FFF725FD1A4B80
:10D1E00083F8E00098B1BDF80C305BBA9BB2B3F5A0
:10D1F000FA6F22D2154A1649A2FB0323DB0807EE79
:10D20000903AF8EEE77AFDEEE77AC1ED047A04B0E1
:10D2100010BD0D4B002283F8E02004B010BD8268E1
:10D2200003AC417C022302F0010290F91000CDE929
:10D2300000420022F6F7D0FCD1E7054B4FF0FF3259
:10D240001A6104B010BD00BFC0EA0024CDCCCCCC24
:10D25000941B0024006810B5037984B00C46012BA0
:10D260001ED0022B02D0002004B010BD826812F044
:10D27000010F03AA14BF00218021FFF7D5FC00286D
:10D28000F1D05CB19DF80D309DF90C20DB0902EB6B
:10D29000820203EB830303EB4203238004B010BD3F
:10D2A000836803AA417C03F0010390F91000009207
:10D2B000002201930223F6F78FFCE0E7F8B5544B08
:10D2C0000D4614462DED048B1B7F022B18D09FEDCD
:10D2D000510A7DB120EE000ADFED4F7ADFED4F6A93
:10D2E0009FED4F7A20EE270AC0EE267A77EE877AF6
:10D2F000C5ED007A0CB14B4B2360BDEC048BF8BD3F
:10D30000494B4A4E1B6896F8081103F00202C1B956
:10D310005B0516D4B2B1464BB3F9182001EE102AC2
:10D32000B3F91620B3F9143000EE902AB8EEC11A02
:10D3300000EE103AF8EEE00AB8EEC00AFDF7DEFCA7
:10D34000C7E722B9D6F8183193ED330AC1E7D6ED15
:10D35000438A96ED449AF0EE680AB0EE490AFDF76A
:10D36000A9FAB5EEC00AB0EE408AF1EE10FA47D441
:10D37000B0EE680A2F4FF0EE490AFDF7A9FCDFED89
:10D380002E7ADFED2E6AF0EE408A28EE278AD7F853
:10D39000EC239FED2B6A9FED2B7AC8EE267AFCEEEC
:10D3A000E77A17EE903A9BB29B1A07EE903AF8EEA6
:10D3B000E77A67EE867AA7EEA67AFDEEC77AB0EE38
:10D3C000470A17EE903A2033402B1ED8FDF7AEFCEB
:10D3D000F0EE407A1C4BB97CA3F12C021846443B7A
:10D3E000D6ED450A90ED000A002918BF1346A8EEB5
:10D3F000E70AD3ED057A70EEA70AFDF769FC68E746
:10D40000DFED127A30EE278AB2E7DFED027AE1E74C
:10D4100018B9002400000000CDCC9C3F00409C4681
:10D4200082E6C5473313904368740024C0EA0024A1
:10D43000089E0024389E00240000C84235FA8E3C25
:10D440000AD7233CDB0FC93F38A20024DB0FC940B9
:10D4500030B5057983B084468E46012D0ED0022D5D
:10D4600002D0002003B030BD8468E40758BF41F00B
:10D47000800103B0BDE83040FFF7D6BB806814469A
:10D480000A46009400F001049CF811109CF9100069
:10D490000194F6F7A1FB03B030BD00BF10B5044600
:10D4A000006882B003796A46022B4FF006030CBF76
:10D4B00043210321FFF7CCFF68B1BDF80010BDF890
:10D4C0000220BDF8043049BA52BA5BBAE1866287DD
:10D4D000238702B010BDC4F83600608702B010BDCB
:10D4E00070B5066882B00446F569002D5CD0002254
:10D4F00004233046FF212A700DEB0302FFF7A8FF3B
:10D5000010B9002002B070BD04236A46FF212068D4
:10D51000FFF79EFF0028F4D09DF804309B09023BE2
:10D52000012BEED9BDF8043043F6FF7CBDF8062090
:10D530005BBABDF80010BDF80240C3F30D066645A6
:10D54000DFD0002EDDD053BA40F2FF7EC3F34A1283
:10D5500072451346D5D0002AD3D049BAC1F30D0283
:10D5600062451146CDD0002ACBD064BAC4F34A122A
:10D5700072451446C5D0002AC3D0721A002AB8BF1B
:10D580005242FF2ABDDC1A1B002AB8BF5242FF2AB2
:10D59000B7DC23440E445B107610C5F8013001233C
:10D5A000C5F805602B70ADE709211420FDF7FEFDDD
:10D5B000F061054626689AE770B5066882B0F4699E
:10D5C000F4B100210423304621700DEB0302FF214A
:10D5D000FFF73EFF10B39DF804309B0919D1BDF849
:10D5E00004200121BDF8063052BA21705BBA92B214
:10D5F000C3F34A13C4F80520C4F8013002B070BD6B
:10D60000054609211420FDF7D1FDF06104462E687E
:10D61000D7E7044A04210320FDF742FD002002B0B1
:10D6200070BD00BFC0F10C08184B03EB8000D0F8B0
:10D630001C0138B300EB400003EB800292F92DC1CE
:10D64000BCF1FF3F1FD092F83501D8B103EB0C00BD
:10D65000002310B590F880E18C2092F83411142248
:10D6600000FB0CFC0A4C0CEB0100013A714434F84D
:10D67000100013FA80F3F6D1064AA2FB0320C0F390
:10D680000F1010BD70470020704700BFC0EA002493
:10D69000C0300030CDCCCCCC30B50D4683B00320AB
:10D6A0001446FFF7C1FF01909DB107EE900ADFED30
:10D6B0000B5AB0EE006ADFED0A6AF8EE677AB8EE50
:10D6C000047A67EEA57AA7EE867A67EE267AC5ED2C
:10D6D000007A0CB1034B236003B030BD6740533A6E
:10D6E00000007A443313904310B1036882889A6132
:10D6F000704700BF0379022B00D0704790F91020CB
:10D7000008311C4802EB420210B41B4C83B050F8A5
:10D71000322000946944194C11F808CCA24224D05C
:10D7200017498A4223D001F580618A4205D0154B02
:10D730009A420CBF03234FF0FF33116803EB4303FE
:10D7400021F0010100EBC30011600169936851F8F9
:10D750002C1023F0E0430B439360136843F0010364
:10D76000136003B05DF8044B70470023E5E7012325
:10D77000E3E700BF5403002400010203003001402E
:10D78000003800400034014010B50446C06900B1C3
:10D7900010BD09211420FDF709FDE06110BD00BF97
:10D7A00090F91030F0B503EB4303284E154683B0D3
:10D7B00056F83360044683689A0719D501230DF1A2
:10D7C00006028DF8061030460DF10701F6F71EFD32
:10D7D00001230DF106020DF1070130468DF80650C8
:10D7E000F6F714FDA3689B0716D5012003B0F0BD22
:10D7F00043691BB19A88186812048261144B154A58
:10D800001868154BC0005768A3FB003080095368A7
:10D81000DB1B9842FBD2D1E70D4A4FF4FA700E4B56
:10D8200012680C4900FB02F24868A3FB023292091D
:10D830004B681B1A9A42FBD26369002BD5D01A6839
:10D8400001209B88936103B0F0BD00BF5403002406
:10D850005C390024001000E0D34D621010B503794C
:10D8600084B084468E46012B0DD0022B02D00020BE
:10D8700004B010BD8368DB0758BF01F07F0104B01E
:10D88000BDE810408CE781680DF10F001446724628
:10D8900001F001018DF80F40CDE900019CF8111055
:10D8A0009CF91000F5F768FF04B010BD10B50446F0
:10D8B000002221210068FFF7D1FFFC2220212068EF
:10D8C000FFF7CCFF402224212068FFF7C7FF0C227E
:10D8D00023212068FFF7C2FF002222212068FFF7E2
:10D8E000BDFF012010BD00BF10B5044694220B21DE
:10D8F0000068FFF7B3FF712201212068FFF7AEFF38
:10D90000002204212068FFF7A9FFC8220521206812
:10D91000FFF7A4FF002206212068FFF79FFFC8221F
:10D9200007212068FFF79AFF002208212068FFF7EF
:10D9300095FFC82209212068FFF790FF012010BD44
:10D9400000680379012B06D0022B01D0002070471C
:10D950001A46082124E7826890F910C002F00102FB
:10D96000417C60464FF0020C10B584B00DF10F04FD
:10D97000019208228DF80FC00094F5F7FDFE04B067
:10D9800010BD00BF00680379012B06D0022B01D027
:10D99000002070470122082102E78268417C02F0E2
:10D9A000010210B590F9104084B020460DF10F042B
:10D9B0000192082200948DF80F30F5F7DDFE04B0D7
:10D9C00010BD00BF10B50446006884B00379012B78
:10D9D00011D0022B02D0002004B010BD01220B2177
:10D9E000FFF7DEFE0028F6D01D220921206804B0D2
:10D9F000BDE8104032E7826890F910C002F00102E1
:10DA0000417C60468DF80F3001920DF10F020092BB
:10DA10000B22F5F7B1FEE5E72DE9F04105461F467B
:10DA20002848164695F9103082B003EB430350F8AE
:10DA30003380AB689A0716D501230DF106028DF8E5
:10DA4000061040460DF10701F6F7E0FB3B46324673
:10DA500000214046F6F7DAFBAB689B0718D501209A
:10DA600002B0BDE8F0816B691BB19A881868120496
:10DA70008261154B1868154BC000A3FB0030144B96
:10DA800080095A685C68A4EB020C6045FAD2D3E7BF
:10DA90000D4A4FF4FA700D4B12680D4900FB02F26B
:10DAA0004868A3FB023292094B681B1A9A42FBD2C8
:10DAB0006B69002BD3D01A6801209B88936102B058
:10DAC000BDE8F081540300245C390024D34D62107A
:10DAD000001000E030B5057983B084468E46012DF4
:10DAE0000DD0022D02D0002003B030BD8468E407C1
:10DAF00058BF41F0800103B0BDE830408CE780683A
:10DB000014460A46009400F001049CF811109CF998
:10DB100010000194F5F730FE03B030BD2DE9F0415F
:10DB2000104C00251746022304F5C27884F88511AD
:10DB3000FF210646424684F88451FFF7CBFF68B1C7
:10DB4000424630460223FF21FFF782FC30B1B4F891
:10DB5000843128465BBA3B80BDE8F0816FF00C0051
:10DB6000FAE700BFC0EA002430B5184D83B095F83D
:10DB7000DA300BB903B030BD04460DF10501006881
:10DB80006AF0BEFE9DF8053073B94FF406410122DC
:10DB900020680323A5F88411FF2185F886210C4A0B
:10DBA00003B0BDE8304095E70DF1060296212068EC
:10DBB000FFF7B4FF074ABDF806300749A2FB03236D
:10DBC0000122DB0885F8DB208B60DEE7C0EA002459
:10DBD00044EC0024CDCCCCCC941B002430B50446BE
:10DBE000006885B00379012B28D0022B0DD0204B83
:10DBF0006FF00102DA601F491F4AD1F884321568BC
:10DC00003233AB4228D305B030BD826812F0010F29
:10DC100003AA14BF5121D121FFF706F80028E6D04E
:10DC2000BDF80C30124A5BBA9BB2D360D368B3F52F
:10DC3000C87FE0DD4FF0FF33D360DCE7836803AAE1
:10DC4000417C03F0010390F91000009251220193EE
:10DC50000223F5F7C1FFE1E701F52272C1F8845212
:10DC6000002351212068FFF735FF05B030BD00BF0C
:10DC7000941B0024C0EA00240C33002470B52F4C00
:10DC800005460323002104F522720068FFF7E0FB3C
:10DC900058B96FF00103C4F8E430294AD4F88C3243
:10DCA000116832338B423FD370BDB4F88822F2EE54
:10DCB000046A94F88AC2082152BA94F8883292B25F
:10DCC00007EE902AF8EEE77A87EEA67ABDEEC77ADD
:10DCD00084ED397A58B25B0042000028DBB282F052
:10DCE0000702B8BFD3B20139F4D194F889220821D0
:10DCF000534058B25B0042000028DBB282F00702BA
:10DD0000B8BFD3B20139F4D19C45C6D1D4F8E430C0
:10DD10002BB1D4F8E4204FF6FF739A42BDD14FF0F7
:10DD2000FF33C4F8E430B8E7C4F88C120123286844
:10DD30003121044ABDE87040CCE600BFC0EA0024AF
:10DD40000C33002450ED002410B5164C82B003793A
:10DD500084F886210022012B84F8851184F884211F
:10DD600010D0022B03D06FF00C0002B010BD0323C3
:10DD700004F5C272FF21FFF74FFE0028F3D0002008
:10DD800002B010BD816804F5C2740323FF2201F0C4
:10DD90000101CDE90041417C90F91000F5F7ECFC60
:10DDA000EBE700BFC0EA002400680379012B0AD02A
:10DDB000022B00D07047836813F0010314D00023B6
:10DDC0000B4A512128E682680023417C02F00102BF
:10DDD00090F9100010B5064C82B0CDE900425122F6
:10DDE000F5F7CAFC02B010BD014AD12114E600BF0C
:10DDF00048ED002400680379012B0BD0022B00D0E2
:10DE0000704783680C4A13F0010F4FF0010311D0E3
:10DE1000002101E68268417C02F0010290F91000C5
:10DE200010B582B0044C019200220094F5F7A4FCD6
:10DE300002B010BD8021EFE550ED002490F91030C4
:10DE4000F0B503EB4303264E154683B056F8336016
:10DE5000044683689A0715D501230DF106028DF853
:10DE6000061030460DF10701F6F7D0F90123002224
:10DE700029463046F6F7CAF9A3689B0716D5012054
:10DE800003B0F0BD43691BB19A881868120482611F
:10DE9000144B154A1868154BC0005768A3FB003097
:10DEA00080095368DB1B9842FBD2D5E70D4A4FF43B
:10DEB000FA700E4B12680C4900FB02F24868A3FB93
:10DEC000023292094B681B1A9A42FBD26369002BFB
:10DED000D5D01A6801209B88936103B0F0BD00BFC4
:10DEE000540300245C390024001000E0D34D62107C
:10DEF00010B5037982B08E46012B0DD0022B02D0D3
:10DF0000002002B010BD8368DB0758BF41F08001DC
:10DF100002B0BDE8104091E7816814467246009453
:10DF200001F00104417C90F910000194F5F754FED2
:10DF300002B010BD30B5002385B004460221C0F800
:10DF400036300DF1070243870068FFF7D1FF18B1A3
:10DF50009DF80730DB0703D40025284605B030BD07
:10DF6000062302AA03212068FFF772FA0DF10702C7
:10DF700009212068FFF7BCFF05460028ECD09DF87A
:10DF8000073013F00C0FE7D1BDF80820BDF80C30B6
:10DF9000BDF80A10C2EB8232C3EB833320688900DC
:10DFA0009B009200218763870A21E2860122FFF706
:10DFB00055FC284605B030BDF0B5484D83B095F806
:10DFC000D8303BB195F890620446012E38D0022E2D
:10DFD00054D00EB103B0F0BD012280210068FFF7DC
:10DFE0003DFC0122FF212068FFF738FC3246314614
:10DFF0002068FFF733FC95F8912291212068FFF704
:10E000002DFC314601222068FFF728FC3246FF2113
:10E010002068FFF723FC324680212068FFF71EFCB2
:10E02000314601222068FFF719FC2D4B2D490122B2
:10E030001B68087085F89022C5F8943203B0F0BDD3
:10E0400001AA00210068FFF753FF9DF80430254F17
:10E05000DA07387039D5D5F89832002BBAD0204A73
:10E06000D5F89412126892B2521A9342B2D24FF07B
:10E07000FF3200237A6085F89032ABE701AA1321C2
:10E080000068FFF735FF9DF80430164F5B073870C6
:10E09000E1D0334601AA1E212068FFF7D9F9BDF867
:10E0A0000430206801225CBA0B21FFF7D7FB0E4B2E
:10E0B000A4B201223870A3FB0434002385F8D920D0
:10E0C000E40885F890327C6084E7054B02221B68E7
:10E0D00085F89022C5F894327CE700BFC0EA00249E
:10E0E0000C330024941B0024CDCCCCCC2DE9F04F74
:10E0F00082468DB0002090460AF1040708910690F0
:10E100000A930790069B5046DC0008EBC303059377
:10E11000FBF7DEF828B941E09AF8043013F0010269
:10E1200008D03A46FF21DAF80000FFF7E1FE0028A8
:10E13000F2D133E003929A070B9040F1CC80F021AA
:10E140005046FBF7F7F848B3083CDDF80C9008EBB5
:10E150000403012409932546089B003B18BF0123B3
:10E160000493049B082D8CBF002303F001039B46FE
:10E17000002B5DD06E1E089B43FA06F606F00106E2
:10E18000F2017821DAF80000FFF768FB30B1DAF825
:10E1900000000379012B3FD0022B07D000220A9BFD
:10E1A0001046069919700DB0BDE8F08F83683A46A5
:10E1B000FF21DB075CBF3A46FF21FFF73FFE002847
:10E1C000ECD09AF8043013F00102E0D199094FEA3B
:10E1D000531E4FEAD31C01EA5313DB074BD46645A9
:10E1E00002D0BBF1000F73D1BCF1000F2DD0059907
:10E1F00011F80930234301F809306400013514F0A7
:10E20000FF04EDB2ADD109F101095FFA89F9B9F165
:10E21000080F30D00124A4E78268417C02F0010C91
:10E2200090F91000FF22CDE9007CF5F7D5FCC6E798
:10E23000069BD3B1079BAB4217D9099B13F8093052
:10E240001C4214BF012600269AE74EEA0101039BF7
:10E2500011F0010F059908BF2B46039311F80930FF
:10E2600023EA040301F80930C7E7079B5E1BB6FAEF
:10E2700086F6760984E7402D07D80A9B069A1B7814
:10E2800093423FF63FAF024689E7059BDD795C1E6E
:10E290009E1D14F801CF082182EA0C0301394FEAD0
:10E2A0005C0C43F3000311F0FF0123F0730383EAD6
:10E2B0005202D2B2F0D1A642EBD19542DDD1069BFB
:10E2C0000133DBB20693039B002BDCD00793D4E72A
:10E2D0000B9E324663E70646324660E7026830B579
:10E2E000137985B00446012B61D0022B03D00025A1
:10E2F000284605B030BD916802AD1046C9072A46D0
:10E300004CBF19468221FFF799FD0028EFD09DF8F8
:10E310000830DA07EBD52A46072303212068FFF7E8
:10E3200097F805460028E2D011220A212068FFF75D
:10E3300095FA9DF80E301B07D9D42A49BDF808304C
:10E34000B1F89C2213FB02F3274A93423EDBB3F55C
:10E35000000F39DA002BB8BFFF331B125B421BB230
:10E36000BDF80A20E386B1F89E3212FB03F31E4A81
:10E3700093422FDBB3F5000F30DA002BB8BFFF3329
:10E3800043F30F22BDF80C30B1F8A012228713FB23
:10E3900001F3154A93421BDBB3F5000F1CDA002B87
:10E3A000B8BFFF331B125B421BB26387A0E7517CEF
:10E3B00002AD92F910009268009502F001020192FC
:10E3C0000222F5F709FCA0E7084BC9E7084BC7E7AD
:10E3D000074BEAE7064AD5E7044BE6E747F6FF7244
:10E3E000D0E700BFC0EA002401FF7FFF0180FFFFEC
:10E3F0000080FFFF10B5002386B0044600688DF84A
:10E400000F300379012B31D0022B02D0002006B04F
:10E4100010BD83680DF10F02D9074CBF2721A7213A
:10E42000FFF70CFD0028F1D09DF80F301B07EDD54C
:10E43000062304AA28212068FFF70AF828B3BDF9AB
:10E440001030002BB8BF03339A10BDF91230002BE7
:10E45000E286B8BF03339A10BDF91430002B22872F
:10E46000B8BF03339B10638706B010BD8268417C40
:10E4700002F0010290F910C001920DF10F02604606
:10E4800000922722F5F7A8FBCCE7C4F83600608796
:10E490000020BCE730B54FF0000C0446006887B0A0
:10E4A000C4F836C0A4F83AC00379012B2AD0022B55
:10E4B00002D0002007B030BD83680DF10F02D907EC
:10E4C0004CBF61468021FFF7B9FC0028F1D09DF8D0
:10E4D0000F301B07EDD5062304AA01212068FEF7A3
:10E4E000B7FF0028E5D0BDF81430BDF81010BDF816
:10E4F00012205BBA49BA52BA5B42E186228763872F
:10E5000007B030BD85686246417C05F0010590F991
:10E51000100001950DF10F050095F5F75DFBD4E7AF
:10E5200010B500230446006886B0C4F8363063870F
:10E530000379012B23D0022B02D0002006B010BD9E
:10E5400083680DF10F02D9074CBF06218621FFF722
:10E5500075FC0028F1D09DF80F305B07EDD5062340
:10E5600004AA00212068FEF773FF0028E5D0049A72
:10E57000BDF81430C4F83620638706B010BD826839
:10E58000417C02F0010290F910C001920DF10F02DE
:10E59000604600920622F5F71FFBDAE710B500236C
:10E5A0000446006886B0C4F8363063870379012BCF
:10E5B00012D0022B0DD183680DF10B02DB074CBF8B
:10E5C0003421B421FFF73AFC18B19DF90B30002B30
:10E5D00011DB002006B010BD8268417C02F0010210
:10E5E00090F910C001920DF10B02604600923422A6
:10E5F000F5F7F2FAE8E7092303AA24212068FEF7D9
:10E6000027FF0028E5D09DF810209DF80F109DF8F9
:10E61000133012041B0442EA01629DF8121043EA0F
:10E6200001639DF80C10C2F30F42C3F30F4322871E
:10E6300063879DF80D301B0443EA0163C3F30F4366
:10E64000E38606B010BD00BF0A4600212DE9F04167
:10E65000DFF8B08084B042F001020446274EFFF795
:10E66000FDF8D8F80070264DC6F8947218E0022B19
:10E670004FF000000BD1A3680DF10F0213212046CB
:10E68000DB0702D40DF10F029321FFF7D7FB9DF8B2
:10E690000F30287013F0070318D1D6F898222ABB40
:10E6A0002379012BE3D1A2680DF10F0102F00102E1
:10E6B000009101921322617C94F91000F5F78CFA15
:10E6C0009DF80F30287013F00703E6D001220B21CC
:10E6D0002046FFF7C3F8002220461146FFF7BEF898
:10E6E00001232870184604B0BDE8F081D8F8001066
:10E6F00089B2C91B8A42D3D2F4E700BFC0EA002422
:10E70000941B00240C3300240368DA6B10B5044614
:10E7100082B012B1904740B123685B6B1BB12146B8
:10E7200001A8984718B9FF23E38202B010BDBDF8D5
:10E730000630013B9BB2F7E7F0B50D4683B00446C7
:10E74000184616461F466CF0D3F92844E67329464E
:10E75000A0732046256800243B46324600946C692D
:10E76000A04703B0F0BD00BF38B58B680446016018
:10E770000D46984700230B4A237522612B6B13B17A
:10E78000204698472075084B93F8A4321BB1237D8F
:10E7900023F00103237500232046E382BDE83840BF
:10E7A000B2E700BF0001FF00C0EA0024144B30B5FF
:10E7B0001C6885B084B12379012B10D0022B0BD1BA
:10E7C000A1680246204611F0010118BF802105B062
:10E7D000BDE83040FEF7E4BF002005B030BDA268C0
:10E7E0000DF10F05617C8DF80F0094F9100002F017
:10E7F0000104802200950194F4F7BEFF05B030BDFE
:10E800000C760024F0B5274D85B02868002846D046
:10E81000B0228021FFF722F8286800283FD040224C
:10E820008021FFF71BF82868002838D000228021BB
:10E83000FFF714F8286890B310228021FFF70EF834
:10E8400028684FF4806400270DF10F0670B103793A
:10E85000012B10D0022B09D183680022402113F034
:10E86000010304BF1A464021FEF79AFF013CA4B2FF
:10E870009CB12868EAE78268013C90F910E002F058
:10E88000010CA4B2417C402270468DF80F70CDE996
:10E89000006CF4F771FF002CEBD105B0F0BD002047
:10E8A000CFE700BF0C76002410B50C4C2368A3B151
:10E8B000A0F1500280211846D2B2FEF7CFFF2068A7
:10E8C00058B100228021FEF7C9FF206828B110222C
:10E8D0008021BDE81040FEF7C1BF10BD0C760024BA
:10E8E000A0F12003F0B503EB83031C4D1C4E85B053
:10E8F000EC18053530681D4498B10379012B227856
:10E9000016D0022B09D00134AC42F7D100224021AD
:10E9100005B0BDE8F040FEF7A1BF4021FEF740FF83
:10E9200030680134AC42E7D10028EFD105B0F0BD2A
:10E930008168013490F910C001F00107417C8DF825
:10E940000F20604601970DF10F0740220097F4F762
:10E9500013FFAC423068CFD1E6E700BF94500C08FB
:10E960000C760024F0B59B4D85B02868002800F097
:10E970002E81D4228021FEF771FF2868002800F044
:10E98000268180221146FEF769FF2868002800F0E2
:10E990001E81A8228021FEF761FF2868002800F070
:10E9A00016813F228021FEF759FF2868002800F0D9
:10E9B0000E81D3228021FEF751FF2868002800F045
:10E9C000068100228021FEF749FF2868002800F018
:10E9D000FE8040228021FEF741FF2868002800F0D9
:10E9E000F6808D228021FEF739FF2868002800F08C
:10E9F000EE8014228021FEF731FF2868002800F005
:10EA0000E680A1228021FEF729FF2868002800F077
:10EA1000DE80C8228021FEF721FF2868002800F050
:10EA2000D680DA228021FEF719FF2868002800F03E
:10EA3000CE8012228021FEF711FF2868002800F006
:10EA4000C68081228021FEF709FF2868002800F097
:10EA5000BE80CF228021FEF701FF2868002800F049
:10EA6000B680D9228021FEF7F9FE2868002800F040
:10EA7000AE80F1228021FEF7F1FE2868002800F028
:10EA8000A680DB228021FEF7E9FE2868002800F03E
:10EA90009E8040228021FEF7E1FE2868002800F0D9
:10EAA0009680A4228021FEF7D9FE2868002800F075
:10EAB0008E80A6228021FEF7D1FE2868002800F073
:10EAC0008680AF228021FEF7C9FE286800287ED00C
:10EAD000A6228021FEF7C2FE2868002877D0AE2249
:10EAE0008021FEF7BBFE2868002870D020228021FC
:10EAF000FEF7B4FE2868002869D000228021FEF7C6
:10EB0000ADFE2868002862D0B0228021FEF7A6FE64
:10EB1000286800285BD040228021FEF79FFE2868ED
:10EB2000002854D000228021FEF798FE2868002893
:10EB30004DD010228021FEF791FE28684FF48064AA
:10EB400000270DF10F0628B30379012B2BD0022BE0
:10EB500004F1FF3215D094B2002CF6D1812280212D
:10EB6000FEF77CFE286848B1C8228021FEF776FEB9
:10EB7000286818B1AF228021FEF770FE012005B091
:10EB8000F0BD8268402112F0010218BF0022FEF79A
:10EB900007FE2868013CA4B2002CD4D10028DDD1A6
:10EBA000012005B0F0BD8268013C90F910E002F050
:10EBB000010CA4B2417C402270468DF80F70CDE963
:10EBC000006CF4F7D9FD2868002CBCD1E6E70020E2
:10EBD000B4E700BF0C760024FDF7C0BEFDF7BEBE53
:10EBE000FDF7BCBEFDF7BABEFDF7B8BEFDF7B6BE79
:10EBF000FDF7B4BE01207047034620B1026812B190
:10EC0000D26902B1104793ED017AF6EE007A074B14
:10EC1000B8EEC77AD3ED016AE7EE267AFDEEE77A21
:10EC200017EE900A00F30B00704700BF04BD0024EC
:10EC3000034620B1026812B1126A02B1104793ED87
:10EC4000027AF6EE007A074BB8EEC77AD3ED026A85
:10EC5000E7EE267AFDEEE77A17EE900A00F30B0056
:10EC6000704700BF04BD0024034628B102681AB1F2
:10EC7000516A09B19369184793ED037AF6EE007A69
:10EC8000064BB8EEC77AD3ED036AE7EE267AFDEEBF
:10EC9000E77A17EE900A00F30B00704704BD0024DA
:10ECA000D8B10E4B0E4A70B506680D4682B00446C8
:10ECB00033449B0A32F8130066F068FAC5F3810307
:10ECC0000022A1883046CDE90032C5F3411305F09A
:10ECD00013026BF0E3FC02B070BD70470000FEA7AA
:10ECE000DC470C08D0B10E4BF0B5076816460D4A4C
:10ECF0000D463B4483B004469B0A32F8130066F08D
:10ED000045FAC5F38103A188384605F01302CDE921
:10ED100000366B096BF0C2FC03B0F0BD704700BF5A
:10ED20000000FEA7DC470C0810B50409013C042CC8
:10ED300019D80F4A00F00F0332F8140040FA03F21A
:10ED400012F0010211D0012202FA03F3013B184034
:10ED500075F042FA074B084A1B5D184400EB40006F
:10ED600002EB800010BD002010BD104610BD00BF9A
:10ED7000D0470C086C500C08C85F00242DE9F04FF8
:10ED80005422044600218BB0AF4874F09FF9AF4A7B
:10ED9000611EE01C144611F8013F5D1E052D88BF61
:10EDA0000023884244F8043BF5D102F110031146D8
:10EDB00051F8040B012800F038818B42F8D111463C
:10EDC00051F8040B022800F026818B42F8D111463D
:10EDD00051F8040B032800F014818B42F8D111463E
:10EDE00051F8040B042800F002818B42F8D111463F
:10EDF00051F8040B052800F0F0808B42F8D152F84E
:10EE0000041B062900F0DF809342F8D1904F1A26A8
:10EE10004FF0000ADFF8308207F52D75DFF83492E5
:10EE200098F80C4054B32046FFF77EFF20B105232D
:10EE3000C6718371002303720321FFF731FF0023A2
:10EE400002E001331C2B37D015F83320A242F8D151
:10EE500007EBC303D3F8B8420123D9F8BC2106213C
:10EE6000C8F81040D0189A4488F81420C9F8BC019A
:10EE700088F8161088F8153089F8B831013608F18D
:10EE80000C08F6B2202ECBD1BAF1000F11D0DFF86A
:10EE9000DCA14FF0000BDFF8D8919AF8EC306BB999
:10EEA0000BF1010B0AF1F40A09F58C79BBF1030FA0
:10EEB000F3D10BB0BDE8F08F0024CDE7BAF806001F
:10EEC0004FF4403666F062F9BAF8040066F05EF975
:10EED000DAF8F0305F4CF421012BCAF82830DAF868
:10EEE000002001FB0B41D4BF002301230327CAF8F4
:10EEF0001020CAF81C300023CAF838308AF82C30A9
:10EF0000CAF83030CAF820308AF848300493082311
:10EF1000CAE905634FF48063CAF834304FF4807354
:10EF2000AAF824304FF48053CAE90F73D1F8303176
:10EF3000002B00F0848093689D0003D59168464BB8
:10EF40000B4093609368D80013D4444B90681968C1
:10EF5000434B034043F080539360424BB1FBF3F3C8
:10EF60000493049B2BB1049B013B0493049B002B53
:10EF7000F9D19368D90023D4F4234FF0010803FB9F
:10EF80000B43D3F8301141F01001C3F83011D3F81E
:10EF9000341141EA0801C3F83411F423916803FBEA
:10EFA0000B4301F00401D3F8300100F010000143DD
:10EFB00060D0D3F8302142F01002C3F830216FE75F
:10EFC0004FF00008E9E7284B172193F8802183F8D8
:10EFD0007411013283F8802118E72349142491F831
:10EFE000800181F86841013081F8800107E71E49FE
:10EFF000342491F8800181F85C41013081F880016E
:10F00000F5E61949352491F8800181F85041013025
:10F0100081F88001E3E61449312491F8800181F8F8
:10F020004441013081F88001D1E60F49302491F844
:10F03000800181F83841013081F88001BFE6C1F8D4
:10F0400034318AF8603076E7ECEB0024DCEB002406
:10F0500084500C08941B0024C0FFFF5F00000024B4
:10F06000C0FFFF6F400D0300C0EA0024601C0024B5
:10F07000C0300030D3F8301121F4817141F0020129
:10F08000C3F830119368DB0713D47B4B9A4200F02E
:10F09000178303F580739A4200F01283774B9B68C5
:10F0A000DE0706D476498B6823F47C1343F440339F
:10F0B0008B60744B74491B68D368194043F2080392
:10F0C0000B43D3609168936801F0040103F00803D7
:10F0D000194300F05D82DAF81000DAF81C30012BD9
:10F0E00000F05283036B23F00F030363F42303FB4D
:10F0F0000B43D3F8302122F0030242F00102C3F89F
:10F100003021B8F1000F7FF4CBAE9AF86020CDF833
:10F110001480012A3FF4C4AE8268012195078AF861
:10F120006010816802D4CA0700F18282F421574A34
:10F13000574B01FB0B41D1F830512A4042F00202FB
:10F14000C1F830218268134043F000438360836834
:10F15000504A002BC0F2E481F4204F4B4F4D4FF446
:10F16000005600FB0B404E490327D0F8302122F017
:10F17000030242F00102C0F83021DAF80820CAF890
:10F180009C70AA4218BF9A424FF480650CBF0123BD
:10F1900000238A4208BF43F0010318318A4208BFA6
:10F1A00043F0010318318A4208BF43F001031831CC
:10F1B0008A4208BF43F0010318318A4208BF43F076
:10F1C000010318318A4208BF43F0010301F556716B
:10F1D0008A4208BF43F0010318318A4208BF43F056
:10F1E000010318318A4208BF43F0010318318A42F3
:10F1F00008BF43F0010318318A4208BF43F00103FE
:10F2000018318A4208BF43F0010318318A4208BF0F
:10F2100043F0010300218AF86010CAF89810CAE987
:10F220001F11CAE92811DAF80C10CAF878104FF447
:10F230000061CAE921514FF480711A4DCAE9236176
:10F240004FF400315646CAF89410296846F8742FD6
:10F250001BB9154B9A4240F0AC840020F4238AF885
:10F26000A800022003FB0B4383F87501136823F009
:10F27000010313601FE000BF00200240006002583D
:10F28000006302580010005C03C0F0FFFDEEFFFFBA
:10F29000C0FFFE3F00F8C3251000024028000240D6
:10F2A00040000240002F0024B80402402B685B1A83
:10F2B000052B00F2B3811368DB07F7D413683046DF
:10F2C000A2491940A24B0B431360536923F0070373
:10F2D0005361F2F7F1FEDAF8D03003F01F013F235B
:10F2E0008B408360DAF874209A4B9B499B4F8A428B
:10F2F00018BF9A4201F11801A2EB070C0CBF0123C1
:10F3000000238A4208BF43F0010318318A4208BF34
:10F3100043F0010318318A4208BF43F0010318315A
:10F320008A4208BF43F0010318318A4208BF43F004
:10F33000010318318A4208BF43F0010301F55671F9
:10F340008A4208BF43F0010318318A4208BF43F0E4
:10F35000010318318A4208BF43F0010318318A4281
:10F3600008BF43F0010318318A4208BF43F001038C
:10F3700018318A4208BF43F0010318318A4208BF9E
:10F3800043F00103DCF1000701F1180147EB0C0722
:10F390008A4208BF43F001037149501A14313B43BC
:10F3A000D0F1000EA2EB010C4EEB000EDCF10001DF
:10F3B0004EEA030341EB0C010B4301916949501ADA
:10F3C0004142414168480B4302916849A2EB010C5C
:10F3D000DCF1000141EB0C010B430091111A484292
:10F3E00048416349A2EB010C0343DCF1000141EB0E
:10F3F0000C01DFF894C1624514BF4FF0000C4FF0D0
:10F40000010C0B4302D1BCF1000F3ED047EA0E07BE
:10F41000019B3B43029F1F433B46009F1F43D3B2C8
:10F42000384301435CEA010100F039831422083BB0
:10F430000127DFF858C1B3FBF2F34E4A9F401A444C
:10F440009200DAF87C30CAF8DC70802BCAE9352CDF
:10F4500000F00C81DAF87830D8B2013B072B10604D
:10F46000CCF8047000F20881471E002900F09C834C
:10F47000414B424903449B0001220020BA40CAE9A3
:10F480003831CAF8E82018604A60F42301220021CC
:10F49000009503FB0B439646C3F8941183F875213E
:10F4A0000AF110034FFA8BF2CAF85C60CAF8AC306C
:10F4B0009446334B06E00EF1010E0C33BEF1070FFC
:10F4C00000F008815A7D002AF5D093F90D2062459D
:10F4D000F1D100229D7D196906922A4A019502EB1D
:10F4E0008802D2F894039AF86020012A3FF4D8AC3D
:10F4F0004FF001028AF86020DAF8102095686D0755
:10F5000040F10E81F42303FB0B43D3F8302142F08A
:10F510002002C3F830214FF000038AF86030BFE4C6
:10F52000059B01330593059B9342FFF410AEF42233
:10F53000002102FB0B42D2F8303123F0120343F0DA
:10F540001003C2F830318AF86010A9E43F8010FE41
:10F55000002D02001000024028000240085402580A
:10F560001C540258445402586C54025858540258BF
:10F5700080540258009600163F96001640590258D3
:10F58000ECEB002484500C08945402588058025824
:10F59000D068AD4B0340DAF8440043F00303D36076
:10F5A000136923F001031361136923F070430343CC
:10F5B0001361A64B9A427BD003F580739A4277D0B1
:10F5C000A34B9B6813F4403F14BF01230023002B7F
:10F5D00000F0EB80F2F714FEDAF814300146B3F5D0
:10F5E000003F00F01082B3F5403F00F01082B3F509
:10F5F000803F00F00882974BDAF810001A6841F259
:10F600000303B3EB124FC0F0C880934B9942836859
:10F6100000F2158123F4807383605EE5F4232022D9
:10F6200003FB0B43C3F89421032283F8752137E4CD
:10F63000826802F00D02012A24D0D3F83021002183
:10F6400042F01002C3F83021D3F8342142F0010215
:10F65000C3F83421F42303FB0B43D3F8302142F0E9
:10F660001002C3F830218AF8601019E40023CAF8A8
:10F6700078301360CCF804700023CAE93833CAF834
:10F68000E83002E78268754B754D134043F0020382
:10F690008360032303602A688368DF077FF546AD34
:10F6A0002B689B1A022BF7D9F42303FB0B43C4E707
:10F6B0006C4B9B6813F4403F14BF0123002386E783
:10F6C000624B69499B6889680B43DF073FF5F1ACE2
:10F6D0006449E8E4DAF810105C4B009D9942DAF8CE
:10F6E000F0604FD003F5807399424BD05848826840
:10F6F0008B685B073FF5D4AB9AF86030012B3FF481
:10F70000CFAB02F01F0240F221230127D3408AF839
:10F7100060703B4040F0F5808AF86030FFF7C0BB76
:10F72000C1F31305C1F384670295002D78D101253B
:10F73000BD40D6692E43850900F01F00D66105F053
:10F740000C05874002F1300603971F2707FA00F0E7
:10F75000775927EA0000039F3843705195689068F5
:10F7600005F0040500F00800284300F08780906849
:10F77000C0072ED508F1010800225FFA88F88AF840
:10F78000602098E63748B2E7026BDAF8283022F0BA
:10F790000F02013B13430363A8E4344B994247D85B
:10F7A000836823F44073836097E4314A936D03F4D4
:10F7B0004033B3F5803F00F04581B3F5003F00F0E2
:10F7C0003381002B7FF417AF07A8F2F759FD079993
:10F7D00011E7D2F8C0000029029D20EA0500C2F816
:10F7E000C000C7DA1948824200F0318100F580700C
:10F7F000824200F02C8116481E4E8568B668F607D6
:10F8000040F12F81F423002103FB0B43D3F8302177
:10F8100042F02002C3F830218AF86010FFF740BBA5
:10F8200091FAA1F50126B5FA85F506FA05F580E706
:10F83000114B994200F2ED80836823F4407343F446
:10F840008073836049E400BFFCBFFFFF00200240DB
:10F85000006302580010005C002D3101C0FFFF7FE3
:10F86000002F0024002302400021024021BCBE00E2
:10F87000004402580060025841787D01C1F30450F1
:10F88000019FCD0D02F11406874005F00405019794
:10F8900007278740705920EA0700019F38437051BD
:10F8A000AB48006800F07040B0F1805FD06800D0D5
:10F8B000D068106E8D0600F0F840B0EB816F03D178
:10F8C000106E20F000401066506E00F0F840854247
:10F8D00003D1506E20F000405066906E00F0F8406A
:10F8E000854203D1906E20F000409066D06E00F00B
:10F8F000F84085427FF43BAFD06E20F00040D066E8
:10F9000035E78B68DF0723D48F68924B1F4240F0A6
:10F91000D7808F68904B3B4043F001038B602F688A
:10F920008368D80602D08D4B994211D08A480CE0EA
:10F930008B68DB0704D48B68034043F001038B60C2
:10F940002B68DB1B022B00F2BB800B68DB07EFD5BB
:10F95000F420834B814D00FB0B40A942D0F830715D
:10F9600003EA070343F48073C0F8303100D142B991
:10F97000F42303FB0B43D3F8302122F48012C3F8A5
:10F980003021F42303FB0B43D3F8302112F48052CF
:10F9900000F08280D3F8342122F00602C3F834212B
:10F9A000DAF85C0000246F4BDAF83C20C3636E4B3E
:10F9B00003646E4BC3641C230B604B688AF8604081
:10F9C00043F010034B60CB6823F003031343CB6079
:10F9D00090F83430012B0CD0012380F8343090F8AB
:10F9E0003530012B00F036814FF4006380F834404D
:10F9F0004365DAF81020584B91680B4043F004033C
:10FA00009360FFF74DBA1B0CB1FBF3F1F3E58108EE
:10FA1000F1E5574B9942836866D823F4407343F469
:10FA200000738360FFF759BBD36C13F0405360D071
:10FA3000B3F1805F00F0A0814E4AB3F1005F08BFD0
:10FA40001146D8E507A8F2F7B5FC0999D3E54A486D
:10FA50004A4E424F8568B668BF683E43F7073FF598
:10FA6000D1AE474F05F0E076B94244D0454FB94298
:10FA70005ED0454FB9427FF47DAE69023FF57AAE64
:10FA800042498A427FF476AE826822F0E0723243C5
:10FA900042F4800282606DE6C3F8342180E73C487E
:10FAA000103B10441822A828B3FBF2F300D8083307
:10FAB000384A0127DFF8ECC01A449F409200C0E4A6
:10FAC000F42303FB0B43D3F8302142F01002C3F8B8
:10FAD0003021D3F8342142F00102C3F8342100234D
:10FAE0008AF86030FFF7DCB943F440738360FFF7B6
:10FAF000F4BA29497FE52F023FF53CAE23498A42FB
:10FB00007FF438AE254A1168826822F0E0723243F1
:10FB100042F400028260224AB1FBF2F252000692E5
:10FB200002E0069A013A0692069A002AF9D121E6E5
:10FB3000ED013FF51FAE15498A427FF41BAE826886
:10FB400022F0E072324342F08072826012E600BF1F
:10FB50000010005C3F000080C0FFFF7F00210240DA
:10FB6000FEF0FFFF010004085500040859000408D6
:10FB700081F0FA0200127A000023024000200240C5
:10FB8000000084CB000052C70000B8CF00600258CC
:10FB9000F0FBFDBF008200100090D00300000024A5
:10FBA000400D030080080240744B754903449B00DC
:10FBB00062E4744B74498A4218BF9A4201F11401FD
:10FBC0000CBF012300238A4208BF43F00103143114
:10FBD0008A4208BF43F0010314318A4208BF43F050
:10FBE000010314318A4208BF43F0010314318A42F1
:10FBF00008BF43F0010313B9644B9A4223D100209C
:10FC0000F421634B8AF8A800022001FB0B41134446
:10FC100081F875011421B3FBF1F38340106842F2BF
:10FC2000A0516FF31010014330461160CAF8D03074
:10FC3000F2F742FADAF8D03003F01F0101238B40CB
:10FC40004360FFF74FBB4023C0F8943180F87571D3
:10FC5000FFF726B9036840314E4A4F4D876DAB42DE
:10FC600018BF934205F130050CBF01220022AB42C0
:10FC700008BF42F001021835AB4208BF42F0010252
:10FC80001835AB4208BF42F001021835AB4208BF3D
:10FC900042F0010205F55675AB4208BF42F0010281
:10FCA0001835AB4208BF42F001021835AB4208BF1D
:10FCB00042F001021835AB4208BF42F0010218358C
:10FCC000AB4208BF42F001021835AB4208BF42F018
:10FCD00001021835AB4208BF42F00102142505FBB2
:10FCE00006F8022580F8355044652C4C2C4DA34273
:10FCF00008BF42F00102A4F59564AB4218BFA342CD
:10FD00000CBF0124002401D0002A4DD01D6825F02D
:10FD100001051D60002C78D0D0F86CC0D0E91956D0
:10FD20006E60BCF1000F04D0D0E91C566E60002C50
:10FD300073D0C56D05F01F0E3F2505FA0EF5BD60A9
:10FD40001D6825F480251D608568C3F80480402D5A
:10FD500000F0E7809960C3F80C9014B9002A00F015
:10FD60009880196821F01E0141F016011960196888
:10FD700041F008011960BEE00A493CE43F820010EE
:10FD800040090240085402581C5402589454025826
:10FD9000F8ABFDA75800024040000240B804024002
:10FDA0002800024000093D00624DDFF890C1634524
:10FDB00018BFAB420CF1280C0CBF01250025634590
:10FDC00008BF45F001050CF1140C634508BF45F070
:10FDD00001050CF1140C634508BF45F001050CF159
:10FDE000140C634508BF45F00105D3F800C02CF0A2
:10FDF000010CC3F800C0DFF84CC1634508BF45F0F3
:10FE0000010515B94C4DAB4243D1D0F86CC0D0E9D7
:10FE100019566E60BCF1000F86D1002A89D1474D7A
:10FE2000DFF810C1634518BFAB420CF1140C0CBFD6
:10FE300001250025634508BF45F001050CF1140CB0
:10FE4000634508BF45F001050CF1140C634508BF7C
:10FE500045F001050CF1140C634508BF45F00105A0
:10FE60000CF1140C634508BF45F0010515B9324D7E
:10FE7000AB420ED1C56D05F01F0C012505FA0CF53E
:10FE80007D608568C3F80480402D4ED09960C3F82A
:10FE90000C902A49274DAB4218BF8B4205F114053F
:10FEA0000CBF01210021AB4208BF41F001011D68D8
:10FEB00025F00E0545F00A051D60214DAB4208BF37
:10FEC00041F001011435AB4208BF41F00101143586
:10FED000AB4208BF41F001011D6845F004051D60FB
:10FEE000184DAB4208BF41F0010111B912498B42D4
:10FEF00012D1D0F86CC0016E0868C20303D508683F
:10FF000040F480700860BCF1000F05D0DCF80010F0
:10FF100041F48071CCF800101A6842F001021A60B6
:10FF200067E5C3F80890D96017E7C3F80890D9606F
:10FF3000AFE700BF1C5402589454025808540258AA
:10FF40004454025880540258036810B51A79044684
:10FF5000022A03D000232360237110BD987AFEF794
:10FF6000E3FE0028F6D040F61A610022C18020216D
:10FF70000272FEF795FE00232360237110BD00BFBF
:10FF80002DE9F04FBA4E85B0BA4CA64256D21D4666
:10FF900002E00C36A64251D273798B42F9D1337903
:10FFA000834201D00028F4D1F3799342F1D134682F
:10FFB000002C43D0002326606360A360E3602361CC
:10FFC0006361A361E36133792371012B96F806B075
:10FFD000C4F808B0317AE16032D0022B2ED1F07A29
:10FFE000FEF7A2FE96F90970A061B07A2774FEF7B9
:10FFF0009BFE06466061F0B1DFF8948207EB470193
:020000040805ED
:100000007B0058F8319008EBC1010193B9F1000F62
:1000100011D0887DE8B10E2200230D213046F27107
:100020003372B571FEF73CFE3368B2889A612046A0
:1000300005B0BDE8F08F2046FFF786FF0024F6E705
:10004000F07AFEF771FE727AB37AA061227463745B
:10005000EDE7B1F808A0504665F098F801214FEAA5
:100060005A100AF01F0A023801FA0AF1092812D8B8
:10007000DFE810F0F6001100EE0018011001E600B4
:10008000E000D800D0000A007B4BD3F89C0020EAA7
:100090000101C3F89C107B00D91908EBC101487914
:1000A000FEF742FE791CCBB20146019318B10372F0
:1000B00040F60A30C8807B000291D81908EBC000D6
:1000C000C079FEF731FE02990346039020B1019AF0
:1000D000027240F60A50D8807B000291D81908EBD2
:1000E000C0008079FEF720FE0299824628B1019B6C
:1000F000037240F60A40AAF806007B00D8191BF0EC
:10010000040308EBC0000293807A0246084614BF3D
:100110004E212E21FEF7E6FD03987B002E2103EBF6
:10012000070B08EBCB0B9BF80B20FEF7DBFD5046D3
:100130009BF80C200E21FEF7D5FD9BF804A0BAF128
:10014000000F40F0ED80D9F8002022F00102C9F83C
:1001500000204A4A914500F0C180494A914540F04B
:10016000AC80454AD2F8901041F48041C2F890101A
:10017000D2F8901021F48041C2F89010029B002B1D
:1001800040F098804FF000714FF08072D9F80C0069
:1001900040F00040C9F80C00D9F8080020F4F070D5
:1001A000C9F80800D9F80000C00727D4D9F808001A
:1001B000344B034034481843C9F80800D9F80C0000
:1001C000C30005D4D9F8000040F48050C9F80000FD
:1001D000D9F80C0011432D4A02400A4342F08862CC
:1001E000C9F80C20D9F8002022F40062C9F80020D8
:1001F000D9F8502022F00102C9F85020BAF1000FBE
:1002000040F09B807B003B4408EBC308012388F847
:10021000163000E7184BD3F8880020EA0101C3F834
:10022000881038E7144BD3F88C0020EA0101C3F89A
:100230008C1030E7104BD86F20EA0101D9672AE70C
:100240000D4BD3F8940020EA0101C3F8941022E783
:10025000094BD3F8800020EA0101C3F880101AE7A7
:10026000054BD3F8980020EA0101C3F8981012E773
:10027000A00200082C04000800440258003001408D
:1002800000380040E0FFBF8F07000020FFFF39D893
:10029000540300243E4BD3F8900020EA0101C3F838
:1002A0009010F8E63A4BD3F8840020EA0101C3F835
:1002B0008410F0E600210A4668E7364A91451BD1D2
:1002C000334AD2F8901041F40041C2F89010D2F8AD
:1002D000901021F40041C2F890104FE72C4AD2F858
:1002E000981041F48051C2F89810D2F8981021F477
:1002F0008051C2F8981041E7274A914527D0274AF4
:10030000914532D1224AD2F8981041F48011C2F8B6
:100310009810D2F8981021F48011C2F898102DE7A7
:100320005046FEF701FD20B1019B40F60A620372C0
:10033000C2800D21FEF7B4FC05E75046FEF7F4FC41
:1003400000283FF45FAF0268838893615AE7104A40
:10035000D2F8981041F40051C2F89810D2F89810D1
:1003600021F40051C2F8981008E70D4A91457FF436
:1003700005AF02F50C32D2F89C1041F02001C2F812
:100380009C10D2F89C1021F02001C2F89C10F5E6D8
:1003900000440258003C004000340140005001403D
:1003A00000140058084B53F8203029B153B19A88F3
:1003B000196812048A617047002BFCD01A689B8868
:1003C00093617047704700BF78500C0838B5164CE1
:1003D000206820B1154A0321F4F7C8FA20680021EB
:1003E000F4F704F8206800231149426815695A019E
:1003F00001EB431401338A586A4012F47C5F07D042
:10040000102BF4D100220B4BC2604361002038BD99
:100410000849C4604161237F002BF7D140F62B428D
:10042000BDE8384065F09ABB18B70024009F24004F
:10043000540100240000003010B5144C206820B195
:10044000134A6421F4F792FA20680021F3F7CEFFF3
:1004500024682046F4F77AF9226802200D4B52688E
:10046000116882F83D0088680340062B06D0B3F57A
:10047000803F03D00B6843F001030B600123064962
:1004800082F83D3081F8A53210BD00BF18B70024B6
:10049000009F240007000100C0EA00242DE9F04F6E
:1004A000DFF854A283B09AF8A592B9F1000F02D0F8
:1004B00003B0BDE8F08F8B4B1C68237C002BF7D179
:1004C0009AF8A9B2CC469AF8A8720AF52B709AF855
:1004D000AAE201228449CDE90094D9468378C578FF
:1004E000C3F1FF032C469BB293B1B0F80080C3F177
:1004F000FF037E4E05FB03F3A6FB08B61B1276092D
:10050000052E00F2EB80DFE806F0D6BBA2866C4F2A
:10051000AE46AB462B46A1460125274600951E0256
:1005200046EA0446172446EA0B060CEB040802FAD6
:1005300004F5A8EB0403013C35429BB208BF01253A
:1005400003F12A0318BF022541F82350631CEED1A2
:100550000430674B0CF1180C98421FFA8CFCBDD18B
:100560004FF44063CB46DDF80090AAF8AC3480230A
:10057000019CAAF8AE34B9F1000F05D08AF8AAE2BE
:100580008AF8A9B28AF8A8725A4B1B78002B8FD030
:10059000204640F62B41F4F7EBF8524B186803B0B5
:1005A000BDE8F04FF4F75CB9504EEF1A5FFA83F9EB
:1005B0001C462B46A6FB08E56D09C5EB0515A8EB07
:1005C0008505ADB2C5F13C0507FB05F51F46A6FB49
:1005D000056509EB55155FFA85FE0125F346009583
:1005E0009DE7424FEE1AAB465FFA83F91C46A7FB24
:1005F0000853DE465B09C3EB0313A8EB83039BB2EE
:1006000003FB06F6A7FB0637012309EB57170093F8
:10061000FFB23B4683E7354EA5EB030EAB46DFB298
:10062000A6FB08546409C4EB0414A8EB8404A4B228
:10063000C4F13C040EFB04F4DE46A6FB046407EBA5
:1006400054145FFA84F9012400944C4667E7DFF8FC
:100650009CE0EE1AA946DFB2AEFB08B56D09C5EB0A
:100660000515A8EB8505ADB205FB06F6AEFB065EEB
:10067000012507EB5E1E00955FFA8EFEF3464EE7FE
:100680001A4EEF1A5FFA83FEA9469B46A6FB085353
:100690005B09C3EB0313A8EB83039BB2C3F13C03D9
:1006A00003FB07F70123A6FB076700930EEB571721
:1006B000FFB23B4633E7EC1A0C4E5FFA83FE9B46D3
:1006C00008FB04F42B462F46A6FB04640EEB5414DF
:1006D0005FFA84F9012400944C4620E74C463B46DF
:1006E000F3461CE718B7002400000030898888888A
:1006F0006CEF002421B70024C0EA0024F8B53B4C7D
:1007000023687BB13A4A054692F8A5225AB15A6845
:100710005379032B66D8DFE803F056595C0213685F
:1007200040331D60F8BD5A6832491269C2F3032292
:1007300051F82270DA685668EFF31182102181F3C4
:100740001288DFF8BCC059681CF807C02A484F79E6
:1007500030F817000F6800F4F050F96821EA000142
:10076000D868F96056F80C1021F0010146F80C1019
:1007700001691F2930D946682039202000FA01F18B
:10078000F160D2B282F3118800211A681974022331
:100790005268116882F83D30184B88680340062B78
:1007A00006D0B3F5803F03D00B6843F001030B6024
:1007B0000121236882F83D100022DB681A77FFF7D9
:1007C0003BFE2368A3E713683433AAE71368383382
:1007D000A7E713683C33A4E74668202000FA01F13C
:1007E000B160CEE700231B60FFDE00BF18B7002416
:1007F000C0EA002418450C0838450C080700010021
:10080000F8460C0808B5224B1B688BB1214A92F8B8
:10081000A51269B12049097803290AD0022910D00C
:10082000002382F8A532FFF7D1FD08B91B4B1870E1
:1008300008BD5A685379032B27D8DFE803F023203B
:100840001D185A685379032B1FD8DFE803F00D0AEF
:1008500007021368403300221A6008BD13683C3356
:10086000F9E713683833F6E713683433F3E71368AE
:10087000403364221A6008BD13683C33F9E71368FB
:100880003833F6E713683433F3E700231B60FFDEE9
:1008900018B70024C0EA002420B7002421B70024A0
:1008A0002DE9F04F0021A7B04FF00A0A9A4D0C46EF
:1008B0009A4ECDF800A083E0B9F1000F16D14CF0AC
:1008C000400CBEF18C0F86F808C000F2D980621C83
:1008D000983498320DEB040974464FF0040E6A44C4
:1008E00009F88CEC04F1020E02F88CCCBEF18C0FEE
:1008F00040F0020C00F2C48004F198024FF00509A8
:100900006A4402F88BCC04F1040C02F88C9CBCF114
:100910008C0F00F2B5800EF1980E4FF0060B9B0085
:10092000EE44DBB20EF88CBC04EB0B0E02F8897CB3
:10093000BEF18C0F00F2A48004F19C0C4FF0070A6A
:10094000EC440CF88CAC02F8873C04F108038C2BC7
:1009500000F296800EF1980C0DEB0C0E0EF88C9CAC
:1009600002F8850C04F10A008C2800F2898004F159
:10097000A0036B4403F88CBC02F8837C04F10C02E6
:100980008C2A7DD804F1A20004F1A3031446684424
:100990006B4400F88CAC03F88C8C480901F01F07FD
:1009A000012255F82030BA4023EA020345F82030EE
:1009B000009B013B00936DD00131B1F5F07F69D20E
:1009C0003C222846F9F71AFE011E5CDB544BC1F3AA
:1009D000072096F808C0CFB233F8112004F1020EB8
:1009E0000CF040090196D3B24FEA122852073FF5A6
:1009F00063AFB9F1000F03D10CF038029A4217D05F
:100A00000CF0870CBEF18C0F4CEA030C86F808C082
:100A100036D8631C04F1980298330DEB02040422CB
:100A20006B4404F88C2C74460EF1020E03F88CCC47
:100A3000BEF18C0F24D804F198030DEB03020523BB
:100A400002F88C3C231D02F88B0C8C2B18D80EF16D
:100A500098000DEB000E06200EF88C0C201802F802
:100A6000897C8C280CD8621D04F19C030446072065
:100A700098326B446A4403F88C0C02F88C8C8CE737
:100A80006FF0004489E71CB9204627B0BDE8F08F1D
:100A9000224B0193019B23491D6895F91030AA68E8
:100AA00003EB4303920751F8330020D5234603AAF2
:100AB0000021F3F7ABFBAB689B0701D50120E4E70E
:100AC000194A4FF4FA70194B1268194900FB02F2E7
:100AD0004868A3FB023292094B681B1A9A42FBD268
:100AE0006B69002BEAD01A689B889361E6E76B6913
:100AF0001BB11A689B881B0493610B4B0C491A6845
:100B00000A4BD2004E68A3FB023292094B689B1B32
:100B10009A42FBD2CAE700BF70EF00247899002404
:100B200084990024540300245C390024D34D6210BE
:100B3000001000E0F0B5244C83B0206808B1A37920
:100B40000BB103B0F0BD012384210DF10702A371A5
:100B5000FDF7CEF9227A042120680A43FCF77EFED5
:100B60000DF1070284212068FDF7C2F99DF80730D6
:100B700013F00405F4D13C2229461448237272F084
:100B8000A5FA13482A46134F4FF0010E00F5707670
:100B90000E4D30F8023F02F01F014FEA521C0132A5
:100BA0003B400EFA01F19BB223B155F82C300B43B8
:100BB00045F82C30B042ECD1FFF772FE0028FBD193
:100BC000A07103B0F0BD00BF7899002470EF00243D
:100BD0008299002404DFFFFF70B53D4D82B02C6880
:100BE0006CB32B79012B3DD0022B2AD1082294F92A
:100BF00010300021EA718DF8052040F2044203EB29
:100C000043038DF80410ADF80620324A52F8330041
:100C1000A3689A073FD5042300210DEB0302F3F7E5
:100C2000F5FAA3689B071FD53C22FF212A4872F0E2
:100C30004DFA6B791BB9FFF77DFF01236B7102B091
:100C400070BD0DF10302A0212046FDF751F99DF87A
:100C5000033003F00503012B37D0002B2FD12C6874
:100C60000822C4E74822C2E71C4A4FF4FA701C4B22
:100C700012681C4900FB02F24868A3FB0232920989
:100C80004B681B1A9A42FBD26369002BCCD01A68BE
:100C90009B889361C8E763691BB11A689B881B0432
:100CA00093610E4B0F491A680D4BD2004E68A3FB9F
:100CB000023292094B689B1B9A42FBD2ABE70A4A6D
:100CC00040F2DC5312689A42B9D92C6848228EE768
:100CD000789900245403002470EF00245C39002428
:100CE000D34D6210001000E00C3300242DE9F041D8
:100CF0002C4D82B0AB7903B1FEE7012204460E46CB
:100D00002868AA711946EA7902F0F702EA71FCF73D
:100D1000A5FDE2B2074609212868FCF79FFDB4F55E
:100D2000807F38D0DFF88080502208212868FCF7C7
:100D300095FD0DF10702A0212868FDF7D9F850B9FB
:100D4000D8F80C23B8F81033516933EA010108BF11
:100D50001B049361EDE79DF8074014F02004EFD1E8
:100D6000E2B20A212868FCF779FD32190134C0216A
:100D70002868FDF7BDF8362CF2D13FB9EA7939463B
:100D8000286802F0F702EA71FCF768FD0023AB71F6
:100D900002B0BDE8F08140220A212868FCF75EFD20
:100DA000C0E700BF78990024C85F00242DE9F04F08
:100DB0005C4DC3B0AF7907B1FEE7EA790446012381
:100DC0000E4602F0F70239462868EA71AB71FCF76B
:100DD00045FD0923FF2C01AA5470137070D9A40893
:100DE00004F0C0084FF0020C4FF0000E4FF00A0B59
:100DF0000DF1050A4FF00B0911E0B1F5827F02F801
:100E00000CB00AF80C0016F80E0017D80EF1010EFF
:100E100002F804908C46D055BEF1360F17D00CF175
:100E20000204634648EA0E000CF10401B4F5827F27
:100E300003F10307C0B203F10603DED90EF1010E80
:100E40006FF00041384BBEF1360F8C46E7D1B3F559
:100E5000827F64D80823A02053540DF105010CF1C2
:100E6000020301F80C002C68304894F9101001EBD3
:100E7000410150F83100A168890723D50021F3F71B
:100E8000C5F9A3689B0733D5294C0DF10302A021B6
:100E90002868FDF72DF850B9D4F80C23B4F81033B6
:100EA000516933EA010108BF1B049361EDE79DF826
:100EB000033013F02003EFD1AB7143B0BDE8F08FE6
:100EC000B8468FE7616919B18E880F683604BE6134
:100ED0001849194F0E681949F600D7F804C0A1FB4C
:100EE0000616B6097968A1EB0C018E42FAD2C5E765
:100EF000104A4FF4FA70114B12680F4900FB02F2CE
:100F00004868A3FB023292094B681B1A9A42FBD233
:100F10006369002BB8D01A689B889361B4E76FF0BF
:100F20000043A0E7789900240100008054030024C6
:100F3000C85F00245C390024001000E0D34D62102B
:100F4000002A30B501DA10445242002B03EB0105B0
:100F500003DA0C465B4229462546002832DB84181A
:100F6000002901DA2B460021A4F11D0CBCF1000F71
:100F700002DDA2EB0C021418A5F10F02002A01DD1C
:100F80009B1A5D1884421CDBC1F1010CC1EB0113FB
:100F90000E4A0134AC4400EB43034FF0200ECCEB7F
:100FA0000C1C02EB43024FEA4C0C8D4205DB002384
:100FB00022F813E01E339C45FAD101300232A042E0
:100FC000F3D130BD121A00201446C9E784990024D9
:100FD000014B43F820107047504000581648174BFB
:100FE0000168174A41F4807130B4016082B0D3F8CF
:100FF000F410FF24CA2041F48031C3F8F410D3F870
:10100000F41001F4803101915321019D546250622A
:101010005162D3F8D030DB0107D4094B0021094AD3
:1010200059651A6502B030BC7047126D054B9A4283
:10103000F3D102B030BC7047004802580044025857
:101040000040005876614E6970B50546BDF81060E5
:101050000C46016019B119462046F3F787FC31466A
:101060002046F3F7C3F92046F3F770FB226802230A
:101070005268116882F83D30194B88680340062B8E
:1010800006D0B3F5803F03D00B6843F001030B603B
:10109000012382F83D3062685379032B1BD8DFE8C7
:1010A00003F0140E0802136800224033AB601A608C
:1010B00070BD136800223C33AB601A6070BD1368CA
:1010C00000223833AB601A6070BD136800223433DD
:1010D000AB601A6070BD0023AB601B60FFDE00BF19
:1010E000070001002DE9F04F85B0064689461746F6
:1010F0009846BDF838B09DF83CA0F3F7F5F8002805
:101100005DD0304D95F8EC340F2B53D85A1C2E4C33
:1011100002905C20D2B200FB034004F5527485F8C3
:10112000EC2403EB43050392C3EBC50304EB8304F8
:101130000023C0F8483380F84C333079FDF7F4FDD4
:101140000299054620B3039A434680F8069002723E
:1011500002203A46E8712046CDF800B0FFF774FF50
:10116000BAF1000F08D0327A02212846FDF7BAFD05
:10117000204605B0BDE8F08F28461121FDF790FD0F
:10118000AB882A6820461B04936105B0BDE8F08F48
:1011900043463A462046CDF800B0FFF755FFBAF176
:1011A000000FE0D150461121FDF77AFD204605B031
:1011B000BDE8F08F054A00210420F9F771FF0024F3
:1011C000D6E700BFC0EA0024C0300030E4F10C08CC
:1011D000F0B5064600680D4617462DED028B83B02C
:1011E000F0EE408AB0EE608AF3F776FB0446002307
:1011F0003046022100934FF6FF730197B4FBF5F2DE
:1012000013441B0CB4FBF3F4B4FBF5F52246ABB26C
:10121000FFF768FFC0B1B5EE408A07EE904AF8EEDE
:10122000677AF1EE10FA13D028EE278A9FED0B7A39
:101230000123C8EE076A037127EE667AC0ED046ADF
:10124000A8EEA77A80ED037A03B0BDEC028BF0BD67
:1012500007EE105AB8EE478AE8E700BF00007A446C
:101260002DE9F04FB04B0027B04EB14DBA4606F510
:101270008C78B146DFF8D4B22DED028BA7B01B7885
:101280000293D9F80040002355F83320944203D04C
:1012900001330E2BF8D1FF235B4493F8F034022B7B
:1012A00000F09480032B00F08880012B09D1D9F83D
:1012B0000C3023F0807323F0080343F00403C9F8D3
:1012C0000C304846FBF73EF950B90AEB8A03974ABF
:1012D00002EB8303D96801F00C03042B00F081803A
:1012E00009F114090AF1010AC145CAD18F4C029DC6
:1012F0000AE00146E0602068FBF730FA09EB0002E3
:10130000D7B2143444451FD02046FBF71BF9002800
:10131000F7D1E368590703F00C02F2D5042AF0D0A4
:1013200023F008007A1C23F00403BD4240F00400BF
:101330005FFA82F91946DCD82068143444F8083C76
:10134000FBF70CFA4445DFD100247A4F2546A2462C
:10135000A1460AE053074CD4D10100F19B8014361A
:1013600009F10109143746456AD03046FBF7EAF81F
:10137000002858D1F268530703D5029B534500F269
:10138000AD801107E6D5002D57F80CEC40F3B38083
:101390000DF1140C0023614602E0AB4200F0AB807B
:1013A00051F8040F013300688645F6D1530720D465
:1013B000D201D4D557F80C0C72E0D9F80C3023F0D8
:1013C0000C0343F08073C9F80C307AE7D9F80C307D
:1013D00023F0807323F0040343F00803C9F80C30B2
:1013E0006FE701372046FBF7B9F9FFB20744FFB2B8
:1013F00076E7002C57F80CCC40F389800DF1540EA1
:101400000023714602E0A34200F0818051F8040FEE
:10141000013300688445F6D1D201A0D5002D57F8DC
:101420000C0C3BDC4AE014364B46434A01210420B5
:1014300009F10109F9F734FE464507F1140794D183
:10144000394B93F80090B9F10C0F00F37A813B4BC4
:101450001A79032A8BF8FF247AD9111F022900F286
:10146000C881052A00F0AA81062A0CBF4FF47A50E1
:101470004FF47A60324900260027B1FBF0F10020DA
:10148000CBF800152F49486001F110002E4940E9C2
:1014900002675EE0002D57F80C0C0BDD0DF1140C0B
:1014A00000235CF8042F0133126882423FF457AFE7
:1014B000AB42F6D1002C0BDD0DF1540E00235EF88B
:1014C000042F0133126890423FF449AFA342F6D192
:1014D0004FF08071F160FBF741F940E722F008011D
:1014E0000AF1010AF1605FFA8AFA57F80C0CFBF76F
:1014F00035F9F26845E726AB0821704603EB840313
:10150000F160013443F8406CFBF728F927E726AB7C
:101510000421604603EB8503F160013543F8806CDC
:10152000FBF71CF91BE700BF74740024B40300240C
:10153000E0450C08C003002420F20C085C74002471
:1015400040420F00C0EF002495C70408C0EA002401
:10155000B749CBF81015B74901EB420292F8D423F2
:10156000002A00F040814D45C0F24581B9F1000FDD
:101570005AD005AF9FEDB08A0025DFF82483AF4E27
:101580000294D8F800209BF8FF3457F8040FC2F3F8
:101590000072062B00F24681DFE803F061586A34DE
:1015A00004040400052B00F0F680A549A54C062B89
:1015B00018BF21460024019214230A4600940221F8
:1015C000FFF790FD8246002800F0FB80234604468A
:1015D00054F814CBDCF8042010695A0106EB4311CF
:1015E0000133B258424012F47C5F00F0B680102BF9
:1015F000F3D10023CCF81440CCF80C30924B43F8D4
:1016000035A00DE0DFED910A914BB0EE600A5988EC
:10161000FFF7DEFD8C4B43F83500002800F0008119
:101620000135A945ADD1029C9BF814354BBB894AC5
:1016300002210420F9F734FD9BF8FE04B0FA80F093
:10164000400927B0BDEC028BBDE8F08FDFED820AC8
:101650004FF47A71B0EE600AFFF7BAFDDAE7F0EE08
:10166000480A9FED750A4FF4C871FFF7B1FDD1E745
:10167000DFED7A0A4FF4FA619FED790AFFF7A8FDD2
:10168000C8E79BF815959BF8163509F10109A9EBF8
:101690000309B9F1120F0BDD122002214B46714AEA
:1016A000009004208BF8FE140021F9F7F9FCC3E741
:1016B0009BF82035012B00F09280022B6DD166F053
:1016C0002BFE694A9BF82035CBF8242513F0FD0F3B
:1016D00069D1022B6DD023469BB24B45C0F2968058
:1016E000A145A8BFA146B9F1000FA5DD15AD5F4E1C
:1016F0000024DFF8AC815E4F04E0013446F8040BAF
:101700004C4599D0BBF81A35D8F80010BBF818052D
:10171000C1F30071564AB7FBF3F3CDE900019BB268
:10172000032155F8040FFFF7DDFC0028E5D105255E
:10173000014623464F4A04208BF8FE54F9F7B0FCCB
:101740007AE70C2201214B46042000928BF8FE140C
:101750000021494AF9F7A4FC66E7CCF80C10CCF854
:1017600014400B7F002B7FF449AF604612222146C4
:10177000039364F0F3F900283FF440AF039B204645
:101780004822194671F0A2FC01238AF804302E4B3E
:1017900043F835A044E739490CE7394A13F0FD0F07
:1017A000CBF8242597D0374A02210420F9F778FC9A
:1017B00042E7122C2346B8BF12238DE74FF4FA50AC
:1017C00058E6214B029C43F8350005212B462E4A52
